:020000040800F2
:1080000000800120854A0208C94A0208C94A0208BC
:10801000C94A0208C94A0208C94A02080000000009
:10802000000000000000000000000000C94A020833
:10803000C94A020800000000C94A0208C1BF01087D
:10804000C94A0208C94A0208C94A0208C94A0208BC
:10805000C94A0208C94A02085DE60108C5E60108E6
:10806000C94A0208C94A0208C94A0208C94A02089C
:10807000C94A0208C94A0208C94A0208C94A02088C
:10808000C94A0208C94A0208C94A0208C94A02087C
:10809000C94A0208C94A0208C94A0208C94A02086C
:1080A000C94A0208C94A0208C94A0208C94A02085C
:1080B000FDEF0108C94A0208C94A0208C94A020874
:1080C000C94A0208C94A0208C94A0208C94A02083C
:1080D000C94A0208C94A0208E5D5010879D201084F
:1080E000C94A0208C94A0208C94A0208C94A02081C
:1080F000C94A0208C94A0208C94A0208C94A02080C
:10810000C94A0208C94A02082DE70108C94A0208FB
:10811000C94A0208C94A0208C94A0208C94A0208EB
:10812000C94A0208C94A0208C94A0208C94A0208DB
:10813000C94A0208C94A0208C94A0208C94A0208CB
:10814000C94A0208C94A0208C94A0208A3CB010861
:10815000C94A0208C94A0208C94A0208E9CF010807
:10816000C94A0208C94A0208C94A0208C94A02089B
:10817000C94A0208C94A0208C94A0208C94A02088B
:04818000C94A0208DE
:1081880010B5054C237833B9044B13B10448AFF349
:1081980000800123237010BD781F0020000000001C
:1081A800204E02080C4B43B10C4810B50C49AFF3F4
:1081B80000800C48036823B910BD0A48036833B926
:1081C8007047094B002BF7D0BDE810401847064B05
:1081D800002BF5D0184700BF00000000204E020811
:1081E8007C1F0020741F0020000000000000000019
:1081F800074B10B51B6898470022064B1A70064BB0
:108208001B689847BDE81040044B9B695B69184799
:10821800181A0020341A0020C41000208C4D0208BF
:108228002DE9F84F924B1446421ED3F8D450052A34
:1082380000F24081DFE812F006000C000C00560046
:108248008100D800FFF7D4FF47F6A853236046E023
:10825800884B894E022816BFB2469A461E464FF0F2
:10826800FF374FF000094FF0010B844BAAF1040AC5
:10827800D3F80C80043ED8F80030DAF804001B6903
:108288009847D8F800307068DB689847D8F800300D
:1082980070685B699847D8F80030DAF804001B6A00
:1082A800984718B90BFA09F327EA0307D8F80030FA
:1082B80056F8040F9B699847D8F800305AF8040F0D
:1082C8001B6A984718B10BFA09F327EA030709F163
:1082D8000109B9F1110FCED1C7F31007276028465D
:1082E800BDE8F88F216003292DD8DFE801F0021BD3
:1082F8001F23624BDB691B68188880B21BF0DCFD0A
:1083080057A3D3E900231BF067FF57A3D3E9002342
:108318001BF038FE00225A4B1BF034FE1CF044F8C8
:108328002060DCE7554BDB695B68E5E7534BDB69AD
:108338009B68E1E7534B1B6988E70129216022D03C
:1083480005D3022935D0D3F8DC301D43C7E74B4BA2
:10835800DC686068236820309B68984760682368F9
:108368003C30DB689847606823685830DB6898477A
:10837800236860685B693C309847236860685B697C
:1083880058309847ABE73D4BDC68606823683C3061
:108398009B689847606823682030DB689847606866
:1083A80023685830DB6898476068236820305B6929
:1083B800E2E7324BDC686068236858309B6898476E
:1083C800606823682030DB689847606823683C3021
:1083D800DB6898476068236820305B6998472368A2
:1083E80060685B693C30CCE7012921604CD01BD325
:1083F8000229A8D1214BDC686068236858309B6843
:108408009847606823682030DB689847606823686D
:108418003C30DB6898476068236820305B69984780
:10842800236860689B69DDE7144BDC686068236833
:1084380020309B689847606823683C30DB68984721
:10844800606823685830DB689847236860685B6910
:108458003C309847236860689B6991E7AFF30080D8
:108468000000000000FEAF40AAF1D24D6210144097
:1084780004000020184D0020D44C00208C4D020828
:1084880000002440341A00200C4BDC686068236824
:108498003C309B689847606823682030DB689847C1
:1084A800606823685830DB68984760682368203024
:1084B8005B69CEE7D3F8E03047E700BF8C4D020890
:1084C8003B4B3C4ADB685B6803F5B871116003F10C
:1084D800AC01516003F1E401916003F58E71D16044
:1084E80003F5AA71116103F5D471516103F5F071B7
:1084F800916103F50671D16103F51471116203F5F9
:108508002271516203F53071916203F53E71D162B7
:1085180003F54C71116303F55A71516303F56871E2
:10852800916303F57671D16303F582611164224A80
:1085380003F17401116003F19001516003F1C80166
:10854800916003F58071D16003F59C71116103F5A9
:10855800C671516103F5E271916103F5FE71D16154
:1085680003F50D71116203F51B71516203F5297151
:10857800916203F53771D16203F54571116303F513
:108588005371516303F56171916303F56F7103F5DD
:108598007D731364D1630122084B1A70084B094A92
:1085A8001A65094ADA65094A5A6518F03FB900BFE1
:1085B8008C4D0208D44C0020184D0020341A00209D
:1085C8000400002029820008F9810008D9850008E4
:1085D80038B5084C05462368C31A002BB8BF5B4260
:1085E800B3F5FA7F04DB044B9B699B6998472560C8
:1085F80038BD00BF941F00208C4D0208704770479B
:10860800014BD3F8DC00704704000020014BD3F87D
:10861800DC0070470400002070477047014BD3F816
:10862800DC00704704000020014BD3F8DC007047E1
:1086380004000020014BD3F8DC0070470400002040
:10864800012070477047704743691449144A10B5B0
:10865800C3F80412C3F80822C3F80C12C3F8102296
:10866800104B1149C365114B114A8361836203633F
:10867800C361104B104C4364104B41628364104B30
:1086880010494363C36303640F4B4265C16284634B
:108698000465C1640266436610BD00BF49860008D0
:1086A8000786000805860008098600081586000860
:1086B8004F860008218600083D86000823860008AA
:1086C80031860008258600084D86000800230948E1
:1086D800094A80F87930C26713705370074A4367B4
:1086E800C0F8C0204FF0FF32C36602676830FFF75A
:1086F800ABBF00BF04000020A41F0020D5860008DF
:1087080000230748074A4374426113705370064AAE
:10871800C36082654FF0FF3243608260FFF794BF09
:1087280004000020C421002009870008830C2DE9DB
:10873800F0410446294D0CD0C0F34243062B08D122
:108748006B7B20F01F04002B3FD02B7903F01F0315
:108758001C432B69224E9B680021C4F307406F69B4
:1087680096F80080984732786B6907EB880778603D
:1087780003EB82035A68002112025A602B69C4F382
:1087880007209B68984733786A69012102EB8302C6
:10879800536818432B69000250609B68E0B2984701
:1087A8006A69317802EB81014B6818430011A30C08
:1087B800486010610BD0C4F34243072B02D1C4F3C5
:1087C8000111317043F0080302E0EB7BBEE7082398
:1087D80002EB83035C60BDE8F08100BF300100203C
:1087E800E423002038B50C4B04461B6C0F20984737
:1087F8000323B4FBF3F3054603EB4303E41A240114
:1088080004F0300420F030002043FFF78FFF2846A3
:10881800BDE838408AE700BF300100200346C1F3B5
:108828001300820C10B40B4A05D0440C062C04BF6C
:1088380001F01F01D173516903F0770343F0080376
:1088480001EB83035860937B0BB910BC6EE710BC37
:10885800704700BF3001002038B5074D0446AA7B99
:108868001AB9030701D4FFF7BDFF6B6904F07F0451
:1088780003EB8404606838BD30010020002038B55F
:108888000C4CA57BE36BA073A1699847E36BA16AC5
:1088980004209847E36BE16A05209847E36B216B56
:1088A80006209847E36B616B07209847A573012062
:1088B80038BD00BF3001002010B50E4C00206269A1
:1088C800E36B516A98476269E36B516B04209847E0
:1088D8006269E36B916B052098476269E36BD16B22
:1088E800062098476269E36B116C072098470120BE
:1088F80010BD00BF30010020084B70B51B6C054649
:1089080040F008000C461646984720EA040040EA62
:1089180006012846BDE8704080E700BF300100200E
:10892800F8B5284D0646AB7B002B45D0264C607821
:10893800FFF758FF03226378013393FBF2F202EB4F
:1089480042029B1AA27863706B6942F0080203EB3B
:1089580082035868FFF7EAFEA37873B3013303F084
:108968000703A3706368F31A002BB8BF5B42092B97
:1089780022DD2B6C03209847030620D5134B9B78E8
:10898800EBB9E97B2A792372914218D901210A2788
:10899800E06829734218E260AA68B2FBF7F29042D5
:1089A80001D96973E360237A012B04D100232B7367
:1089B8006B73E36023726660F8BD0423D1E701237B
:1089C8002372F0E730010020E4230020341A00204D
:1089D8002DE9F843894690461E460746154C002166
:1089E800236840F080009B689DF8205098472368D2
:1089F80000219B6848469847236800219B684046A9
:108A08009847236800219B68304698472368284682
:108A18009B680121984748EA0928D4F89C3246EA1D
:108A2800082607F07F0703EB870745EA06257D60E0
:108A3800BDE8F8838001002007B5CBB20093C1F3ED
:108A48000742C1F30723090EFFF7C2FF03B05DF821
:108A580004FB70B5284D00F07F06AB1993F80C3273
:108A680013F0050F05D1D5F89C3203EB8606706824
:108A780070BD2B6800219B683046984700212B6801
:108A880008469B68984700212B6808469B689847CA
:108A980000212B6808469B6898472B6801219B6832
:108AA800002098472B6800219B6830469847002192
:108AB8002B6808469B68984700212B6804029B682E
:108AC8000846984700212B6804439B680846984746
:108AD8002B68240204439B68012100209847240244
:108AE800222E40EA040001D0422E03D1030248BFDF
:108AF80040F07F4070BD00BF80010020054BD3F8D7
:108B08009C321A781AB901205A70187070470020E0
:108B1800704700BF80010020054BD3F89C321A78BB
:108B280022B902215A70197001207047002070473D
:108B3800800100202DE9F0474A4C8046D4F89C5229
:108B48002B7883B3022B0CBF2B1D04F10C03687820
:108B5800221892F80C2212F0020F42B20BD0002A0F
:108B68000EDB53F82010D4F8942290476B78013329
:108B78006B70BDE8F087002AF1DB01306870E6E72A
:108B8800D4F89C321A78D10708D5D3F80832984718
:108B98000022D4F89C321A70BDE8F0879207F7D506
:108BA800D3F81032F3E7304D2E68861B002EB8BF7D
:108BB8007642042E53DD16F03BF92120FFF749FFDA
:108BC8002A4F8246BB781BB9D4F89C32C3F8880078
:108BD80030461BF013FD81466868AAEB00000028A8
:108BE800B8BF40421BF00AFD49461BF00FFE204962
:108BF8001BF058FD1BF01CFF60602220FFF729FFC7
:108C08000028B8BF63684FF04100BCBF5B42636097
:108C1800C5F804A0FFF71DFFBB7806461BB9D4F8BA
:108C28009C32C3F80801A868301A0028B8BF40422F
:108C38001BF0E4FC49461BF0E9FD0D491BF032FD31
:108C48001BF0F6FEA0604220FFF703FF0028B8BF24
:108C5800A368AE60BCBF5B42A360C5F80080BDE8F6
:108C6800F08700BF8001002000240020341A002073
:108C78006F1283442DE9F843894690461E460746FD
:108C8800154C0021236840F080009B689DF8205017
:108C98009847236800219B68484698472368002125
:108CA8009B6840469847236800219B683046984750
:108CB800236828469B680121984748EA0928D4F880
:108CC8009C3246EA082607F07F0703EB870745EA48
:108CD80006257D60BDE8F8832804002007B5CBB2DF
:108CE8000093C1F30742C1F30723090EFFF7C2FF40
:108CF80003B05DF804FB70B5284D00F07F06AB1992
:108D080093F80C3213F0050F05D1D5F89C3203EB1C
:108D18008606706870BD2B6800219B6830469847AE
:108D280000212B6808469B68984700212B68084655
:108D38009B68984700212B6808469B6898472B68D2
:108D480001219B68002098472B6800219B683046CA
:108D5800984700212B6808469B68984700212B6894
:108D680004029B680846984700212B6804439B68C7
:108D7800084698472B68240204439B680121002079
:108D880098472402222E40EA040001D0422E03D143
:108D9800030248BF40F07F4070BD00BF2804002098
:108DA800054BD3F89C321A781AB901205A701870FA
:108DB80070470020704700BF28040020054BD3F8F7
:108DC8009C321A7822B902215A7019700120704712
:108DD80000207047280400202DE9F047414C074641
:108DE800D4F89C522B7883B3022B0CBF2B1D04F1B3
:108DF8000C036878221892F80C2212F0020F42B283
:108E08000BD0002A0EDB53F82010D4F89422904798
:108E18006B7801336B70BDE8F087002AF1DB013015
:108E28006870E6E7D4F89C321A78D10708D5D3F8E9
:108E3800083298470022D4F89C321A70BDE8F087AF
:108E48009207F7D5D3F81032F3E7274D2E68861B23
:108E5800002EB8BF7642042E41DD15F0E9FF21202F
:108E6800FFF749FF214B82469A7899461AB9D4F8F8
:108E78009C32C3F8880030461BF0C0FB8046686807
:108E8800AAEB00000028B8BF40421BF0B7FB4146E0
:108E98001BF0BCFC16491BF005FC1BF0C9FD60600B
:108EA8004120C5F804A0FFF726FF99F802300646CE
:108EB8001BB9D4F89C32C3F80801A868301A0028F6
:108EC800B8BF40421BF09AFB41461BF09FFC084983
:108ED8001BF0E8FB1BF0ACFDAE60A0602F60BDE8A6
:108EE800F08700BF2804002018240020341A00202E
:108EF8006F1283440023184610B5064C1A5D5900BA
:108F080002F0030201338A40072B40EA0200F5D140
:108F180010BD00BF30240020002304495A5C02F031
:108F28000302C2540133072BF8D1704730240020C4
:108F3800074B1A7802705A7842709A788270DA78F9
:108F4800C2701A7902715A7942719B79837170479C
:108F580030240020F8B50024074B084D084FDE6880
:108F6800E15D336801F00301DB6955F8040F013452
:108F78009847072CF4D1F8BD8C4D02081007002043
:108F8800302400200023054A00F0030199540133DE
:108F9800072B4FEA9000F7D1DCE700BF3024002010
:108FA800014B586AEEE700BFD006002000230449B1
:108FB800C25C02F003025A540133072BF8D1C9E707
:108FC800302400200278074B1A7042785A70827851
:108FD8009A70C278DA7002791A7142795A71827974
:108FE8009A71B7E7302400202DE9F8438946904666
:108FF8001E460746154C0021236840F080009B68F8
:109008009DF820509847236800219B684846984758
:10901800236800219B6840469847236800219B6885
:1090280030469847236828469B680121984748EAB4
:109038000928D4F8983246EA082607F07F0703EB98
:10904800870745EA06257D60BDE8F88368070020A4
:1090580007B5CBB20093C1F30742C1F30723090E4A
:10906800FFF7C2FF03B05DF804FB70B5274D00F0B1
:109078007F06AB1993F8083213F0050F05D1D5F820
:10908800983203EB8606706870BD2B6800219B68D8
:109098003046984700212B6808469B68984700216E
:1090A8002B6808469B68984700212B6808469B68F0
:1090B80098472B6801219B68002098472B6800215E
:1090C8009B683046984700212B6808469B6898475C
:1090D80000212B6804029B680846984700212B68EA
:1090E80004439B68084698472B68240204439B68FE
:1090F8000121002098472402222E40EA040003D1CF
:10910800030248BF40F07F4070BD00BF68070020E1
:10911800054BD3F898321A781AB901205A7018708A
:1091280070470020704700BF68070020054BD3F840
:1091380098321A7822B902215A70197001207047A2
:10914800002070476807002038B5184CD4F89852AA
:109158002B7853B3022B0CBF2B1D04F1080368783E
:10916800221892F8082212F0020F42B20AD0002AFE
:109178000DDB53F82010D4F8902290476B78013318
:109188006B7038BD002AF2DB01306870E7E7D4F86D
:1091980098321A78012A0CBFD3F80832D3F8103263
:1091A80098470022D4F898321A7038BD6807002012
:1091B8002DE9F843894690461E460746154C00217E
:1091C800236840F080009B689DF8205098472368EA
:1091D80000219B6848469847236800219B684046C1
:1091E8009847236800219B6830469847236828469B
:1091F8009B680121984748EA0928D4F8983246EA3A
:10920800082607F07F0703EB870745EA06257D60F8
:10921800BDE8F883100A002007B5CBB20093C1F36C
:109228000742C1F30723090EFFF7C2FF03B05DF839
:1092380004FB70B5274D00F07F06AB1993F8083290
:1092480013F0050F05D1D5F8983203EB8606706840
:1092580070BD2B6800219B683046984700212B6819
:1092680008469B68984700212B6808469B689847E2
:1092780000212B6808469B6898472B6801219B684A
:10928800002098472B6800219B68304698470021AA
:109298002B6808469B68984700212B6804029B6846
:1092A8000846984700212B6804439B68084698475E
:1092B8002B68240204439B6801210020984724025C
:1092C800222E40EA040003D1030248BF40F07F4049
:1092D80070BD00BF100A0020054BD3F898321A78E9
:1092E8001AB901205A70187070470020704700BFE3
:1092F800100A0020054BD3F898321A7822B90221B7
:109308005A7019700120704700207047100A002019
:109318002DE9F843304B80461B78304C052B29D17A
:109328002F4D2E68861B002EB8BF7642042E21DDF5
:1093380015F07EFD2120FFF77CFF2A4B07469B781E
:109348001BB9D4F89832C3F888006868381A1BF03B
:1093580055F9814630461BF051F9014648461BF045
:1093680055FA21491BF09EF91BF062FB6F606060A3
:10937800C5F80080D4F898522B7853B3022B14BF49
:109388001A4B2B1D6878221892F8082212F0020F47
:1093980042B20BD0002A0EDB53F82010D4F89022EA
:1093A80090476B7801336B70BDE8F883002AF1DBD6
:1093B80001306870E6E7D4F898321A78012A0CBFB1
:1093C800D3F80832D3F8103298470022D4F89832EC
:1093D8001A70BDE8F88300BF04000020100A0020BE
:1093E80044240020341A00206F128344180A0020F5
:1093F8002DE9F843894690461E460746154C00213C
:10940800236840F080009B689DF8205098472368A7
:1094180000219B6848469847236800219B6840467E
:109428009847236800219B68304698472368284658
:109438009B680121984748EA0928D4F8983246EAF7
:10944800082607F07F0703EB870745EA06257D60B6
:10945800BDE8F883B80C002007B5CBB20093C1F380
:109468000742C1F30723090EFFF7C2FF03B05DF8F7
:1094780004FB70B5274D00F07F06AB1993F808324E
:1094880013F0050F05D1D5F8983203EB86067068FE
:1094980070BD2B6800219B683046984700212B68D7
:1094A80008469B68984700212B6808469B689847A0
:1094B80000212B6808469B6898472B6801219B6808
:1094C800002098472B6800219B6830469847002168
:1094D8002B6808469B68984700212B6804029B6804
:1094E8000846984700212B6804439B68084698471C
:1094F8002B68240204439B6801210020984724021A
:10950800222E40EA040003D1030248BF40F07F4006
:1095180070BD00BFB80C0020054BD3F898321A78FC
:109528001AB901205A70187070470020704700BFA0
:10953800B80C0020054BD3F898321A7822B90221CA
:109548005A7019700120704700207047B80C00202D
:109558002DE9F843304B80461B78304C102B29D12D
:109568002F4D2E68861B002EB8BF7642042E21DDB3
:1095780015F05EFC2120FFF77CFF2A4B07469B78FD
:109588001BB9D4F89832C3F888006868381A1BF0F9
:1095980035F8814630461BF031F8014648461BF045
:1095A80035F921491BF07EF81BF042FA6F606060C4
:1095B800C5F80080D4F898522B785BB3022B14BFFF
:1095C8001A4A2A1D6878231893F8083203F00A0308
:1095D800022B43B20BD1002B0EDBD4F8903252F899
:1095E800201098476B7801336B70BDE8F883002B27
:1095F800F1DB01306870E5E7D4F898321A78012A6F
:109608000CBFD3F80832D3F8103298470022D4F8A8
:1096180098321A70BDE8F88304000020B80C0020C6
:1096280058240020341A00206F128344C00C0020F4
:109638002DE9F843184C1E462368894607469B685F
:10964800002140F0800090469DF8205098472368FC
:1096580084F8A6009B6800214846984723680021A3
:109668009B6840469847236800219B683046984786
:10967800236828469B680121984748EA0928D4F8B6
:10968800A83046EA082607F07F0703EB870745EA74
:1096980006257D60BDE8F883600F002007B5CBB2D2
:1096A8000093C1F30742C1F30723C0B2090EFFF7C5
:1096B800BFFF03B05DF804FB38B5244C00F07F050C
:1096C80063191B7ADB073AD5236800219B68284673
:1096D80098470021236808469B689847002123681B
:1096E80008469B6898470021236808469B68984766
:1096F800236801219B6800209847236800219B6804
:10970800284698470021236884F8A6009B680846E5
:1097180098470021236805029B680846984700215E
:10972800236805439B680846984723682D0205432C
:109738009B680121002098472D02284338BDD4F8A2
:10974800A83003EB8505686838BD00BF600F0020AE
:10975800F8B50027364C94E86000330243EA1563F5
:10976800C6B22A0232433B43C4E90023237A226962
:10977800013323726369180E1B0243EA1263120253
:10978800207663612261002950D012F039FC054629
:1097980012F036FC401B0028B8BF40420A28F7DC0C
:1097A800237A244D042B04D9D5F8903061686D20B4
:1097B8009847D5F8903021686C20984712F020FC23
:1097C800064612F01DFC801B0028B8BF4042322814
:1097D800F7DCD5F8903021686C20984700230022E8
:1097E800C4E90023C4E90423237A042B0AD9D5F851
:1097F80094306F209847D4E90423002342EA0006F6
:1098080066612361D5F894306E209847D4E90467DF
:109818000346227A47EAE371C2F10802D2003043D4
:109828001AF0ECF90023C4E904012372207EF8BD84
:1098380070240020600F002038B52220FFF73CFF7D
:10984800A8B904212020FFF729FF0B492420FFF79E
:1098580025FF7920FFF730FFC0B2D0F1800508D08E
:109868002120FFF729FF29183720FFF717FF0020CD
:1098780038BD012038BD00BF0010270038B50546A7
:10988800334C18B1637E0BB901236376637E013BC9
:10989800042B34D8DFE803F0032837415700282089
:1098A800FFF70AFFE0612920FFF706FF0421206285
:1098B8002020FFF7F3FEE1692820B1F57A7F38BF51
:1098C8004FF47A71FFF7EAFE216A2920B1F57A7F11
:1098D80038BF4FF47A71FFF7E1FE00212420FFF72B
:1098E800DDFE022363760AE00720FFF7E5FE20F09D
:1098F800E0710720FFF7D2FEFFF79EFF08B90025A9
:109908001FE00323EEE70720FFF7D6FE40F0807143
:109918000720FFF7C3FE0423E4E7002DEFD107205B
:10992800FFF7CAFE20F080710720FFF7B7FE072077
:10993800FFF7C2FE40F480010720FFF7AFFE0523C2
:109948006376284638BD002301256376F9E700BF12
:109958007024002038B5054C0546636A834203D05D
:109968000020FFF78BFF656238BD00BF7024002020
:1099780000207047012070470022014B5A60704751
:109988000400002038B50A4C05462368C31A002B8A
:10999800B8BF5B42B3F57A7F05DB606815F0E0FC81
:1099A80000232560636063680133636038BD00BFCE
:1099B800A424002010B50C4612F082FE206010BDD1
:1099C80012F0AABE70B51E46C24B19B1D3F8E840D2
:1099D800204670BD4B2AD3F8D44000F0058300F22E
:1099E80091803B2A00F0208246D82E2A00F0AF81D1
:1099F8001ED82A2A00F050810BD8282A00F01A8194
:109A080000F23181272A00F00681D3F8E0000443F0
:109A1800DEE72C2A00F0718140F25381002840F0E3
:109A28008581112012F04CFEC0F380703060CFE7C2
:109A3800332A00F0C9810FD8302A00F0AF81C0F076
:109A48009C81312AE1D1002840F0B58101461320DC
:109A580012F0C1FE3060BBE7392A00F0C98100F27C
:109A6800D581342AD1D1002840F0BA81014601209D
:109A780012F0B1FE3060ABE7432A00F0478220D8ED
:109A88003F2A00F00B820ED83D2A00F0ED8140F20B
:109A9800DA81002840F0F9810146072012F09BFE88
:109AA80000B2306094E7412A00F0178240F2058244
:109AB800002840F0228201460B2012F08CFE306014
:109AC80086E7472A00F059820ED8452A00F03C82E2
:109AD80040F22A82002840F0478201460F2012F007
:109AE8007AFE00B2306073E7492A00F0648240F2DF
:109AF8005482002840F06F820146132012F06BFE5A
:109B0800306065E75B2A00F0318342D8532A00F0C1
:109B1800CB8220D84F2A00F097820ED84D2A00F029
:109B28007D8240F26E82002840F087820146212023
:109B380012F051FE00B230604AE7512A00F09F82CD
:109B480040F28F82002840F0A8820146252012F0BA
:109B580042FE30603CE7572A00F0D6820CD8552ADE
:109B680000F0BC8240F2AD82002840F0C58231206E
:109B780012F0A6FD30602BE7592A00F0E18240F28E
:109B8800D182002840F0EA82352012F099FD306039
:109B98001EE7632A00F04F831DD85F2A00F0168362
:109BA8000CD85D2A00F0FE8240F2EE82002840F0D8
:109BB8000683392012F084FD306009E7612A00F03D
:109BC800238340F21283002840F02D833D2012F0B9
:109BD80077FD3060FCE6672A00F062830CD8652ABE
:109BE80000F0478340F23683002840F05183772005
:109BF80012F066FD3060EBE6692A00F06F83C0F072
:109C08005E83FF2A7FF401AF00287FF4E1AE15F0F0
:109C18006BFB3060DCE630B90146142012F0DBFD46
:109C280000B23060D4E601287FF4D2AED3F8E00069
:109C38000443CDE630B9112012F042FDC0F30240D2
:109C48003060C5E601287FF4C3AE112012F038FD5C
:109C5800336820F4E0211B0403F4E02319431120A6
:109C680012F05AFDB4E630B9112012F029FDC0F304
:109C7800C4403060ACE601287FF4AAAE112012F08F
:109C88001FFD336820F47801DB0403F478031943DB
:109C9800112012F041FD9BE628B9112012F010FDA9
:109CA80080B2306094E601287FF492AE112012F061
:109CB80007FD3188000C00040143112012F02CFD2F
:109CC80086E648B9112012F0FBFCC0F30260306050
:109CD8007EE600BF0400002001287FF479AE112041
:109CE80012F0EEFC336820F0E0611B0603F0E0633D
:109CF8001943112012F010FD6AE630B9112012F054
:109D0800DFFCC0F3C260306062E601287FF460AE19
:109D1800112012F0D5FC336820F06051DB0603F007
:109D280060531943112012F0F7FC51E601287FF423
:109D38004FAE112012F0C4FC336820F080419B071D
:109D480003F080431943112012F0E6FC40E628B9DD
:109D5800112012F0B5FCC00F306039E601287FF4FD
:109D680037AE112012F0ACFC316820F0004040EA18
:109D7800C171112012F0D0FC2AE630B90146122038
:109D880012F029FD00B2306022E601287FF420AEEF
:109D980032880021122012F04FFD19E620B9152053
:109DA80012F08EFC306013E601287FF411AED3F870
:109DB800E00004430CE601287FF40AAE3288002153
:109DC800132012F039FD03E618B912F004FD3060D3
:109DD800FEE501287FF4FCADD3F8E0000443F7E585
:109DE80001287FF4F5AD3288002112F025FDEFE55A
:109DF80028B90146022012F0EEFC3060E8E501289F
:109E08007FF4E6ADD3F8E0000443E1E520B9032090
:109E180012F056FC3060DBE501287FF4D9AD3168DB
:109E2800032012F079FCD3E528B9042012F0D3FC02
:109E380000B23060CCE501287FF4CAAD3288042036
:109E480012F0FAFCC4E530B90146052012F0C3FC53
:109E580000B23060BCE501287FF4BAAD3288002139
:109E6800052012F0E9FCB3E530B90146062012F0EE
:109E7800B2FC00B23060ABE501287FF4A9AD3288AE
:109E88000021062012F0D8FCA2E501287FF4A0AD3D
:109E980032880021072012F0CFFC99E520B908206C
:109EA80012F099FC306093E501287FF491AD328877
:109EB8000021082012F0C0FC8AE528B901460920D3
:109EC80012F089FC306083E501287FF481AD328887
:109ED8000021092012F0B0FC7AE528B901460A20D1
:109EE80012F079FC306073E501287FF471AD328897
:109EF80000210A2012F0A0FC6AE501287FF468AD71
:109F0800328800210B2012F097FC61E520B90C2063
:109F180012F061FC30605BE501287FF459AD3288AE
:109F28000C2012F089FC53E528B901460D2012F0E7
:109F380052FC30604CE501287FF44AAD328800219C
:109F48000D2012F079FC43E528B901460E2012F0E5
:109F580042FC30603CE501287FF43AAD32880021AC
:109F68000E2012F069FC33E501287FF431AD328808
:109F780000210F2012F060FC2AE528B9102012F009
:109F88002AFC00B2306023E501287FF421AD328835
:109F98000021102012F050FC1AE520B9112012F00F
:109FA8008FFB306014E501287FF412AD3168112071
:109FB80012F0B2FB0CE528B90146122012F00BFC96
:109FC800306005E501287FF403AD328800211220B6
:109FD80012F032FCFCE401287FF4FAAC328800214C
:109FE800132012F029FCF3E420B9142012F0F3FB3B
:109FF8003060EDE401287FF4EBACD3F8E0000443D3
:10A00800E6E420B9152012F05BFB3060E0E401289B
:10A018007FF4DEACD3F8E0000443D9E430B901465C
:10A02800202012F0D8FB00B23060D1E401287FF480
:10A03800CFACD3F8E0000443CAE401287FF4C8ACED
:10A04800D3F8E0000443C3E420B9222012F0C3FB94
:10A058003060BDE401287FF4BBACD3F8E0000443D2
:10A06800B6E428B90146232012F0B5FB3060AFE40E
:10A0780001287FF4ADACD3F8E0000443A8E428B984
:10A088000146242012F0A7FB3060A1E401287FF4E8
:10A098009FACD3F8E00004439AE401287FF498AC1D
:10A0A800D3F8E000044393E420B9262012F008FB1B
:10A0B80030608DE401287FF48BACD3F8E0000443D2
:10A0C80086E420B9272012F0FBFA306080E40128EA
:10A0D8007FF47EACD3F8E000044379E420B9302063
:10A0E80012F0EEFA306073E401287FF471AC316845
:10A0F800302012F011FB6BE401287FF469AC316861
:10A10800312012F009FB63E420B9322012F0D8FAAA
:10A1180030605DE401287FF45BAC3168322012F0D6
:10A12800FBFA55E420B9332012F0CAFA30604FE444
:10A1380001287FF44DAC3168332012F0EDFA47E482
:10A1480020B9342012F0BCFA306041E401287FF4D1
:10A158003FAC3168342012F0DFFA39E401287FF48B
:10A1680037AC3168352012F0D7FA31E420B93620FF
:10A1780012F0A6FA30602BE401287FF429AC31688C
:10A18800362012F0C9FA23E420B9372012F098FAE1
:10A1980030601DE401287FF41BAC3168372012F0D1
:10A1A800BBFA15E420B9382012F08AFA30600FE4BF
:10A1B80001287FF40DACD3F8E000044308E401283B
:10A1C8007FF406ACD3F8E000044301E428B93A2050
:10A1D80012F076FA3060FFF7FBBB01287FF4F8AB8A
:10A1E800D3F8E0000443FFF7F3BB28B93B2012F093
:10A1F80067FA3060FFF7ECBB01287FF4E9ABD3F8CE
:10A20800E0000443FFF7E4BB28B93C2012F058FAF9
:10A218003060FFF7DDBB01287FF4DAABD3F8E0004C
:10A228000443FFF7D5BB01287FF4D2ABD3F8E00095
:10A238000443FFF7CDBB28B93E2012F041FA306045
:10A24800FFF7C6BB01287FF4C3ABD3F8E000044393
:10A25800FFF7BEBB28B93F2012F032FA3060FFF793
:10A26800B7BB01287FF4B4ABD3F8E0000443FFF791
:10A27800AFBB28B9762012F023FA3060FFF7A8BBED
:10A2880001287FF4A5ABD3F8E0000443FFF7A0BB97
:10A2980001287FF49DABD3F8E0000443FFF798BB97
:10A2A80028B97C2012F00CFA3060FFF791BB012826
:10A2B8007FF48EABD3F8E0000443FFF789BB28B9DD
:10A2C8007D2012F0FDF93060FFF782BB01287FF492
:10A2D8007FABD3F8E0000443FFF77ABB28B97E20B0
:10A2E80012F0EEF93060FFF773BB01287FF470AB12
:10A2F800D3F8E0000443FFF76BBB07B502AB43F8A4
:10A30800042D02460120FFF75DFB03B05DF804FB56
:10A31800134602460020FFF755BB0F4B9A7882423E
:10A3280004BF0E4A92F8D1001A78824206D10C4B2B
:10A33800DB681B689B690B4A106818475B78834287
:10A3480009D1064B93F8D130834204D1044BDB6822
:10A358001B685B69EFE77047781A0020040000204B
:10A368008C4D0208604D002010B50020FFF7D5FF86
:10A37800BDE81040034B044ADB6810681B689B6803
:10A38800184700BF8C4D0208604D002038B51C4BA3
:10A398001C4DDC6860682368C8302860DB68984713
:10A3A800236828685B699847174B18495A69012040
:10A3B8000A601749C2F804121649C2F80C120021A3
:10A3C80011705170144A58749A63144A83F8D00073
:10A3D8005A63134A9A64134A5A64134A5A65134AC9
:10A3E8001A65134A5A66134A1A66134ADA653222FC
:10A3F800DA604FF48C729A60BDE838408DE700BF90
:10A408008C4D0208604D0020040000205C4D0020A7
:10A4180045A400087D99000819A3000803A30008B3
:10A42800C9990008BD9900088D9900087999000814
:10A4380023A300088199000871A300080120704730
:10A4480012F03EB912F068B912F0C5B912F0F4B9B9
:10A45800084B93F87920824289BF074AD3F8E8006D
:10A4680052F82020002082BF1076D160D3F8D400A3
:10A47800704700BF0400002010100020E8E74942A0
:10A48800E6E70021E4E72DE9F3411D46B24B93F8D6
:10A4980079401E468C4205D8D3F8E840204602B0E1
:10A4A800BDE8F081A32AD3F8D44000F0558265D8DE
:10A4B800072A00F0448126D8032A00F0FC800DD832
:10A4C800012A00F0DF8040F2CD80002840F0EA80C9
:10A4D800A24B53F82130DB682B60DFE7052A00F038
:10A4E800068140F2F180002840F0118120209C4B29
:10A4F800884040F01000D3F89832C0B29847C0F3B3
:10A5080007202860CAE7182A00F081810BD8162A8C
:10A5180000F0498100F26181082A00F03C81D6F8F8
:10A52800E0000443BAE71D2A00F0A28111D81C2AD2
:10A53800F5D1002840F085810801894B40F06C0076
:10A54800D3F8983200F0FC009847C0F380402860A8
:10A55800A4E78C2A00F09481A22AE0D1002840F0D8
:10A56800E38108017E4B40F06C00D3F8983200F08C
:10A57800FC009847C0F3C13028608FE7AC2A00F090
:10A588007D833AD8A72A00F0CB821CD8A52A00F0F0
:10A598002D8240F20682002840F096820E01704F0C
:10A5A80046F06C06F6B2D7F898323046984710F461
:10A5B800804FD7F89832304600F077829847C0F33A
:10A5C800021028606AE7A92A00F0F482C0F0CD8260
:10A5D800AA2A00F01583AB2AA1D1002840F03683BF
:10A5E80008015F4B40F06D00D3F8983200F0FD0091
:10A5F8009847C0F34110286050E7B42A00F0D5838B
:10A6080016D8AE2A00F08783C0F05E83B32A86D1BD
:10A61800002840F0B2830801514B40F06C00D3F899
:10A62800983200F0FC009847C0F34040286035E7B6
:10A63800B62A00F0FD83C0F0C883B82A00F014845D
:10A64800CE2A7FF46CAF00287FF428AF0801444B72
:10A6580040F06F00D3F89832C0B29847C0F30900B1
:10A6680028601BE728B93D4B53F821301B692B6044
:10A6780014E701287FF412AF384B2A6853F82130C9
:10A688001A610BE728B9354B53F821309B682B60CA
:10A6980004E701287FF402AF304B2A6853F82130D1
:10A6A8009A60FBE601287FF4F9AE2C4B2A6853F830
:10A6B8002130DA60F2E600287FF4F0AE274B53F839
:10A6C80021301B682B60E9E628B9244B53F8213068
:10A6D8005B692B60E2E601287FF4E0AE1F4B53F87C
:10A6E80021202B68002BB8BF5B425361D6E628B9FE
:10A6F8001A4B53F821305B682B60CFE601287FF4B2
:10A70800CDAE164B2A6853F821305A60C6E60128A8
:10A718007FF4C4AE20268E40114F46F01006F6B2E4
:10A72800D7F8983230469847C2B22B780092D7F8BB
:10A738009052C0F3074200213046A847AEE688B9D8
:10A748002020074B884040F01000D3F89832C0B260
:10A758009847C0B22860A1E604000020101000202D
:10A768002804002001287FF499AE20268E40AA4FA5
:10A7780046F01006F6B2D7F89832304698472B784C
:10A78800C0F307420093D7F89052C0F30723002183
:10A798003046A84782E600287FF480AE9F4B1B68AE
:10A7A8005B7E2B607AE650B920209B4B884040F0B6
:10A7B8001100D3F89832C0B2984728606EE6012895
:10A7C8007FF46CAE2020944B884040F01100D3F801
:10A7D80094322968C0B2984760E650B920208E4B61
:10A7E800884040F01200D3F89832C0B298472860E9
:10A7F80054E601287FF452AE2020874B884040F071
:10A808001200D3F894322968C0B2984746E650B986
:10A818002020814B884040F01300D3F89832C0B212
:10A82800984728603AE601287FF438AE20207A4B12
:10A83800884040F01300D3F894322968C0B2984792
:10A848002CE601287FF42AAE0E0146F06C06724F02
:10A85800F6B2D7F89832304698472B6820F4802112
:10A868000BB141F48021D7F894323046984715E669
:10A8780000287FF413AE6A4B1B681B682B600DE63B
:10A8880060B90801644B40F06C00D3F8983200F0CE
:10A89800FC009847C0F303602860FFE501287FF4B7
:10A8A800FDAD2B68102B23D00DDC022B1CD004DC53
:10A8B800012B16D04FF0FF3314E0042B16D0082BD1
:10A8C800F8D105230EE0402B14D003DC202BF1D166
:10A8D800032307E0802B0FD0B3F5807FEAD1002354
:10A8E80000E008232B6008E00723FBE70623F9E7CD
:10A8F8000423F7E70223F5E728602B6801333FF4C8
:10A90800CDAD0E01444F46F06C06F6B2D7F898323A
:10A9180030469847296820F0706040EA0161D7F80E
:10A92800943230469847B9E501287FF4B7AD0E0157
:10A93800394F46F06C06F6B2D7F898323046984749
:10A948002B6820F4C031DB0303F4C033D7F894221A
:10A95800194330469047A1E560B908012E4B40F0F5
:10A968006C00D3F8983200F0FC009847C0F38030B0
:10A97800286093E501287FF491AD0E0146F06C063E
:10A98800254FF6B2D7F89832304698472B6820F40E
:10A9980080410BB141F48041D7F894323046984752
:10A9A8007CE560B908011C4B40F06C00D3F8983284
:10A9B80000F0FC009847C0F3003028606EE50128DD
:10A9C8007FF46CAD0E0146F06C06134FF6B2D7F863
:10A9D8009832304698472B6820F480510BB141F4E7
:10A9E8008051D7F894323046984757E548BB0E0156
:10A9F800094F46F06C06F6B2D7F8983230469847B9
:10AA080010F4804FD7F8983230460BD09847C0F3EF
:10AA1800C310286042E500BF280400201010002061
:10AA2800641A00209847D7F89832804630469847ED
:10AA380018F4006FC0F3021018BF40F00800286037
:10AA48002CE501287FF42AAD0E0146F06C06BD4FB7
:10AA5800F6B2D7F898323046984710F4804F0FD0A6
:10AA6800D7F89832304698472B6820F4F061DB011C
:10AA780003F4F063D7F894221943304690470DE564
:10AA8800D7F898323046984729680B074CBF40F4EE
:10AA9800006020F40060090120F07000C9B2014391
:10AAA800D7F8943230469847F8E49847D7F8983260
:10AAB80080463046984718F4006FC0F3C31018BF9B
:10AAC80040F008002860E9E401287FF4E7AC0E01B3
:10AAD8009C4F46F06C06F6B2D7F898323046984745
:10AAE80010F4804FD7F8983230460CD098472B682E
:10AAF80020F070011B0103F07003D7F8942219436A
:10AB080030469047CAE498472B6820F4F061DB018F
:10AB180003F4F063D7F89422194330469047BDE414
:10AB280060B90801874B40F06C00D3F8983200F008
:10AB3800FC00984700F00F002860AFE401287FF47C
:10AB4800ADAC0E017F4F46F06C06F6B2D7F89832DE
:10AB5800304698472B6820F00F0103F00F03D7F811
:10AB6800942219433046904798E460B90801754B20
:10AB780040F06D00D3F8983200F0FD009847C0F31C
:10AB8800C03028608AE401287FF488AC0E0146F0C2
:10AB98006D066C4FF6B2D7F89832304698472B6856
:10ABA80020F400410BB141F40041D7F8943230460B
:10ABB800984773E460B90801624B40F06D00D3F820
:10ABC800983200F0FD009847C0F34130286065E4F2
:10ABD80001287FF463AC0E015A4F46F06D06F6B2B9
:10ABE800D7F89832304698472B6820F4C0415B0369
:10ABF80003F4C043D7F894221943304690474DE4F4
:10AC080060B908014F4B40F06D00D3F8983200F05E
:10AC1800FD009847C0F3032028603FE401287FF433
:10AC28003DAC0E01474F46F06D06F6B2D7F89832A4
:10AC3800304698472B6820F470611B0203F4706358
:10AC4800D7F8942219433046904727E401287FF427
:10AC580025AC0E013B4F46F06D06F6B2D7F8983298
:10AC6800304698472B6820F060015B0103F06003D1
:10AC7800D7F894221943304690470FE460B9080189
:10AC8800304B40F06D00D3F8983200F0FD00984743
:10AC980000F00F00286001E401287FF4FFAB0E01EB
:10ACA800284F46F06D06F6B2D7F8983230469847E6
:10ACB8002B6820F00F0103F00F03D7F894221943F3
:10ACC80030469047FFF7EABB68B908011D4B40F0D2
:10ACD8006D00D3F8983200F0FD009847C0F300608B
:10ACE8002860FFF7DBBB01287FF4D8AB0E0146F0E4
:10ACF8006D06144FF6B2D7F89832304698472B684D
:10AD080020F080710BB141F08071D7F89432304651
:10AD18009847FFF7C3BBB8B908010A4B40F06D006C
:10AD2800D3F8983200F0FD009847001410F0800F17
:10AD380014BF6FF0FF030023C2B213432B60FFF769
:10AD4800ADBB00BF2804002001287FF4A7AB0E018B
:10AD5800594F46F06D06F6B2D7F898323046984704
:10AD68002B6820F4FE011B0403F4FE03D7F8942299
:10AD7800194330469047FFF791BB01287FF48EAB0B
:10AD88000E0146F06C064C4FF6B2D7F898323046B2
:10AD980098472B6820F400310BB141F40031D7F803
:10ADA800943230469847FFF779BB00287FF476AB9A
:10ADB8000801414B40F06F00D3F89832C0B2984771
:10ADC800C0F307402860FFF769BB30B93B4B53F825
:10ADD8002130DB692B60FFF761BB01287FF45EAB94
:10ADE800202606FA01F0344F46B246F0110046F02C
:10ADF80014062968F6B2D7F89432C0B29847D7F843
:10AE080098323046984720F480684146D7F8943203
:10AE1800304698472B683046002B14BF4FF48061AA
:10AE28000021D7F8943241EA08019847FFF736BB6A
:10AE380058B92020204B884040F01100D3F89832B0
:10AE4800C0B298472860FFF729BB01287FF426ABDA
:10AE58002020194B884040F01100D3F8943229681B
:10AE6800C0B29847FFF71ABB68B90801124B40F007
:10AE78006C00D3F8983200F0FC009847C0F34030DB
:10AE88002860FFF70BBB01287FF408AB0E0146F0E2
:10AE98006C06094FF6B2D7F89832304698472B68B7
:10AEA80020F400510BB141F40051D7F894323046E8
:10AEB8009847FFF7F3BA00BF2804002010100020BD
:10AEC80007B502AB43F8042D02460120FFF7DBFA71
:10AED80003B05DF804FB134602460020FFF7D3BA1F
:10AEE800014BD3F89432184728040020034B10B5BF
:10AEF800D3F898320C469847206010BD28040020EB
:10AF0800014BD3F88C321847280400200022014B4B
:10AF1800DA667047040000200B4B70B5DD680B4CF7
:10AF28002B6820699B6898472B68206A9B6898471C
:10AF38002B68606A9B689847054BDB689847BDE8B3
:10AF48007040044B5B6818478C4D0208B8240020F9
:10AF5800641A0020AC190020074A10B1D2F8E800A2
:10AF68007047064B1B6819610121197683F84C005C
:10AF7800D2F8D400704700BF040000201010002051
:10AF8800034B0A681B689B6813440B601946E3E788
:10AF98001010002010B50B4A10B1D2F8E80010BD0F
:10AFA8000124094B1B681C7683F84C00074800688D
:10AFB80080685864586C1861996483F84C40D2F8DA
:10AFC800D40010BD0400002010100020641A0020D6
:10AFD800084B93F87920824202D8D3F8E8007047EA
:10AFE8000028FAD1044A126812680A60D3F8D4001B
:10AFF800704700BF04000020641A0020012810B523
:10B00800144605D0022810D00B4BD3F8E00010BD31
:10B018000A4B0B4ADB68106A1B681B6A98470030AA
:10B0280018BF01202060002010BD044B044ADB68D3
:10B03800506A1B681B6AF1E7040000208C4D020867
:10B04800B824002038B50D4B0D4C987820B92368EA
:10B058001A688AB91B687BB90A4B0B4DD3F8A03222
:10B068009847AB6898470120084A2B685168D2680E
:10B078002360636059629A6238BD00BF341A0020A9
:10B088001010002028040020641A0020B824002092
:10B09800022804BF0B4B93F8D10030B90A4BDB6888
:10B0A8001B685B69094A10691847012809D1054BD3
:10B0B80093F8D130012B04D1034BDB681B689B69E3
:10B0C800F0E77047040000208C4D0208B8240020E7
:10B0D80070B5544E544CF5686B6803F1C802226190
:10B0E80003F59C72626203F5AA72226203F5C672C6
:10B0F800A26003F5D47203F5B870626003F5E272DA
:10B1080003F53773A3622B68E260DB682060984719
:10B118002B68A068DB6898472B686068DB689847ED
:10B128002B68E068DB6898472B682069DB689847DC
:10B138002B68A06ADB6898473C4DA26A33690020F7
:10B148005A602B603A4BD5F89462C5F89C32D5F812
:10B158009832984740F006010020B047354EB36852
:10B16800984733682168344A5962A1681360996224
:10B17800736832495360626802205A62E2680024A8
:10B188009A622F4BDA6FC2F80412D5F8A412147021
:10B198005470C2F80C122B4A2B4DC3F888202B4A46
:10B1A800C3F884202A4AC3F880202A4AC3F88C208E
:10B1B800294AC3F8A020294AC3F89C20284AC3F882
:10B1C8009020284AC3F89420274AC3F89820274A91
:10B1D800C3F8B020264AC3F8AC20264AC3F8BC20DE
:10B1E800254AC3F8B820254AC3F8B420244AC3F82E
:10B1F800CC20244A83F87900C3F8C82032225A6741
:10B208004FF48C721A67204A83F8D000C3F8C42020
:10B21800FFF73EFF2B689847AB682046BDE87040B3
:10B22800184700BF8C4D0208B824002028040020CD
:10B23800A41F0020641A0020101000204DB0000840
:10B248000400002059A40008AC19002085A40008B7
:10B2580087A400088BA40008DFAE0008C9AE000868
:10B2680061AF000889AF00089DAF0008E9AE00088B
:10B27800F5AE000809AF000805B00008D9AF00080E
:10B2880099B0000815AF000821AF0008084B93F8E3
:10B298007920824289BF074AD3F8E80052F8202073
:10B2A800002082BF1076D160D3F8D400704700BF69
:10B2B800040000201C100020E8E74942E6E70021CE
:10B2C800E4E7024B0846DB6B184700BFD0060020B6
:10B2D800034B10B51B6C0C469847206010BD00BF8F
:10B2E800D0060020364B0628F7B505460C46D3F89D
:10B2F800D4701A4605D9D3F8E0301F43384603B056
:10B30800F0BD022906D9012801D10F2902DDD2F8A2
:10B31800EC30F2E72B4E6846336B98473346052DE1
:10B3280006D8DFE805F003094144474A8DF8004094
:10B33800DB6A68469847E1E7082CF9D8DFE804F0AB
:10B34800050C11161B20252A2F00F2788DF80120F4
:10B35800327B8DF80220EBE732798DF80120727B81
:10B36800F7E772798DF80120B27BF2E7B2798DF8B0
:10B378000120F27BEDE7F2798DF80120327CE8E7D5
:10B38800727A8DF80120B27CE3E7B27A8DF8012059
:10B39800F27CDEE7327A8DF80120727CD9E7F27A06
:10B3A8008DF80120327DD4E78DF80340C0E78DF891
:10B3B8000440BDE78DF80540BAE78DF80640B7E7C9
:10B3C80004000020D0060020464B06282DE9F34152
:10B3D80004460E46D3F8D470984606D9D3F8E03020
:10B3E8001F43384602B0BDE8F0813F4D68462B6BDD
:10B3F800013C98472B46052C70D8DFE804F003631E
:10B4080066696C6F9DF80120E978914207D19DF833
:10B418000200297B884202D100233360E1E71979D1
:10B42800914206D19DF80200597B884201D101233F
:10B43800F3E75979914206D19DF80200997B884239
:10B4480001D10223E9E79979914206D19DF80200DA
:10B45800D97B884201D10323DFE7D979914206D10C
:10B468009DF80200197C884201D10423D5E7597A56
:10B47800914206D19DF80200997C884201D10523AA
:10B48800CBE7997A914206D19DF80200D97C88428F
:10B4980001D10623C1E7197A914206D19DF802002D
:10B4A800597C884201D10723B7E7D97A914206D15E
:10B4B8009DF802201B7D9A4201D10823ADE7D8F8F8
:10B4C800EC308DE79DF80330A7E79DF80430A4E73A
:10B4D8009DF80530A1E79DF806309EE79DF80030FD
:10B4E8009BE700BF04000020D006002007B5034BEF
:10B4F80068461B6B984703B05DF804FBD006002034
:10B5080070B50020FFF7F2FF1F4B204CDD68206B61
:10B518002B689B6898472B68E06A9B6898472B685C
:10B52800E0689B6898472B68A0689B6898472B68D9
:10B5380060689B6898472B6820689B6898472B68C9
:10B54800A0699B6898472B68E0699B6898472B68B7
:10B55800A06A9B6898472B6860699B6898472B6826
:10B56800206A9B6898472B68606A9B6898472B6895
:10B5780020699B689847064BDB689847BDE8704090
:10B58800044B5B68184700BF8C4D0208F02400206C
:10B59800641A0020AC190020604B2DE9F041DF68E7
:10B5A8005F4C78685F4E00F5FE73236300F5F07317
:10B5B800E36200F52973E36000F53073A36000F5DA
:10B5C8002273636000F50D73236000F55A73A3615D
:10B5D80000F55373E36100F1C803A36200F5C67375
:10B5E800636100F56873236200F56F7363623B68FB
:10B5F80000F5B870DB68206198473B686069DB68D4
:10B6080098473B68206BDB6898473B68E06ADB68D3
:10B6180098473B68206A1B6998473B68606A1B69C2
:10B628009847E26806F140057264A26806F15C0872
:10B63800B2646268F26422683265A2697265E2697E
:10B64800B265A26AF2653B686868DB6898473B6840
:10B6580055F8040F9B6998474545F4D10022324DAF
:10B66800DFF80481EB6F1A70D8F808309847D8F8DB
:10B6780004302269DFF8F4805A626269C8F8003041
:10B688009A622A4B0220C5F88830294BC5F88430C5
:10B69800284BC5F88030284BC5F88C30274BC5F8A7
:10B6A800A030274BC5F89C30264BC5F89030264B68
:10B6B800C5F89430254BC5F8B030254BC5F8AC30EB
:10B6C800244BC5F8CC30012385F8793085F8D03083
:10B6D800214BC5F8C030214BC5F8C430FFF706FF31
:10B6E800D8F800301B6813B11D4B9B780BB1B36AB7
:10B6F80098470222236B197C5A741868012215F0A6
:10B708000DFA3B68206B174C1B68984723689847CD
:10B71800A3680020BDE8F041184700BF8C4D02081F
:10B72800F0240020D00600200400002095B2000874
:10B73800C1B20008C3B20008C7B20008BDB700080C
:10B7480091B8000879B70008A9B70008CBB200087B
:10B75800D9B20008F5B40008A1B5000809B5000879
:10B76800341A0020AC190020641A00201C10002094
:10B77800094B93F87920824202D8D3F8E800704741
:10B78800064A52F82020116101211176002182F821
:10B798004C10D3F8D4007047040000201C1000207F
:10B7A800034B0A681B689B6813440B601946DFE764
:10B7B8001C10002038B5304B154693F879208A4282
:10B7C8001A4603D8D3F8E840204638BD0B28D3F8EA
:10B7D800D44011D8062837D202282BD005D800B378
:10B7E800012823D0D2F8E00019E00428234B28D000
:10B7F80024D91B685B6817E013280CD80E2835D2AB
:10B808000C2827D00D28EDD11D4B1E4ADB68106B84
:10B818001B681B6A24E08C28E4D1D3F8E0000443B9
:10B82800D2E7164B1B681B692B60CDE7134B1B68CF
:10B838009B68F9E7114B1B68DB68F5E71B681B6819
:10B84800F2E71B685B69EFE70828E6D10B4B1B683A
:10B858005B7EE9E70A4B0B4ADB68D06A1B681B6A08
:10B868009847003018BF01202860ADE70E382946F8
:10B87800C0B2FFF7A9FDA7E7040000201C100020B4
:10B888008C4D0208F02400201FB5364B019293F826
:10B8980079408C42194604D8D3F8E840204604B0D1
:10B8A80010BD0B28D3F8D44011D8062840D202285E
:10B8B80031D005D838B3012829D0D1F8E00014E0F8
:10B8C8000428294B2ED02AD91B685A60E6E713288A
:10B8D8000DD80E2844D20C2830D00D28EDD142F2D4
:10B8E80010718A4237D9D3F8E0000443D6E78C2890
:10B8F800E3D101A90120FFF767FD1C4B04439B6BB3
:10B9080002A89847CAE7184B1B681A61C6E7164B86
:10B918001B689A60C2E7144B1B68DA60BEE71B68B5
:10B928001A60BBE71B68002AB8BF52425A61B5E7E4
:10B9380006381146C0B2FFF7D5FCD6E70C4B0D49C7
:10B948002AB1CA6812685269D86A9047A6E7CA68D5
:10B9580012689269F8E7084B90B29B6898479DE790
:10B968000E38E6E7040000201C100020D006002056
:10B97800F02400208C4D0208AC190020084B93F8E5
:10B988007920824289BF074AD3F8E80052F820207C
:10B99800002082BF1076D160D3F8D400704700BF72
:10B9A8000400002024100020E8E74942E6E70021CF
:10B9B800E4E7F7B5B84E1D4696F879308B42334622
:10B9C80004D8D6F8E840204603B0F0BDA62AD6F839
:10B9D800D44000F0548300F28B80172A00F0D881FD
:10B9E80033D8042A00F06E810ED8012A00F038817D
:10B9F800C0F02881022A00F04181032A00F0548116
:10BA0800D3F8E0000443DEE7072A00F08D8110D860
:10BA1800052A00F06881062AF2D1002840F07181D9
:10BA28009E4B1020D3F894329847C0F30720286023
:10BA3800C9E7082A00F09581152AE1D1002840F0CD
:10BA48009D81D6F8E0000443BDE71D2A00F021825D
:10BA58001FD81A2A00F0D0810BD8182AD0D1002874
:10BA680040F0C0818D4B3320D3F89432984728603A
:10BA7800A9E71B2A00F0DD811C2AC1D1002840F06B
:10BA8800F581864BD3F894329847C0F3400028607C
:10BA980099E7A32A00F07B8210D88C2A00F006824E
:10BAA800A22AADD1002840F05E827C4B6C20D3F8EE
:10BAB80094329847C0F3C130286084E7A42A00F084
:10BAC8008382A52A9CD1002840F0A982734E6C205D
:10BAD800D6F89432984710F4804FD6F894324FF045
:10BAE8006C0000F08E829847C0F3C31028606AE7A4
:10BAF800B52A00F01E8442D8AB2A00F0768316D807
:10BB0800A82A00F02283C0F00383A92A00F03A8310
:10BB1800AA2A7FF475AF002840F052835F4B6D204E
:10BB2800D3F894329847C0F3032028604BE7AE2A35
:10BB380000F0B08311D8AC2A00F07983AD2A7FF4E5
:10BB48005FAF002840F09283544B6D20D3F89432B5
:10BB58009847C0F30060286035E7B32A00F0C28335
:10BB6800B42A7FF44DAF002840F0DB834B4B6F20A5
:10BB7800D3F894329847C0F30440286023E7BB2ADF
:10BB880000F05B8436D8B82A00F0008417D8B62AAB
:10BB98007FF436AF002840F0E383404B1420D3F8FD
:10BBA800943298474FF08073002808BF012093FB18
:10BBB800F0F03B4B9842D4BF28602B6003E7B92ACA
:10BBC80000F00384BA2A7FF41BAF002840F01D84DC
:10BBD800324B1320D3F8943298474FF080730028E3
:10BBE80008BF012093FBF0F02D4B9842D4BF28608A
:10BBF8002B60E8E6C02A00F0968411D8BC2A00F031
:10BC08004C84BF2A7FF4FCAE002840F06D84234B9F
:10BC18007020D3F894329847C0F301402860D2E6E8
:10BC2800CC2A00F0AA84CE2A7FF4EAAE002840F09D
:10BC3800C6841A4B6F20D3F894329847C0F3090092
:10BC48002860C0E620B9174B1B681B692B60BAE651
:10BC580001287FF4B8AE134B2A681B681A61B2E654
:10BC680020B9104B1B689B682B60ACE601287FF459
:10BC7800AAAE0C4B2A681B689A60A4E620B9094B47
:10BC88001B68DB682B609EE601287FF49CAE054BA1
:10BC98002A681B68DA6096E604000020680700201E
:10BCA800FFFF0F002410002020B99E4B1B681B6863
:10BCB8002B6088E601287FF486AE9A4B2A681B68B9
:10BCC8001A6080E620B9974B1B685B692B607AE69F
:10BCD80001287FF478AE934B1A682B68002BB8BF05
:10BCE8005B4253616FE620B98E4B1B685B682B6023
:10BCF80069E601287FF467AE8A4B2A681B685A6098
:10BD080061E601287FF45FAE874E1020D6F89432A2
:10BD18009847C2B22B780092D6F88C52C0F30742EB
:10BD280000211020A8474EE638B97F4B1020D3F8E1
:10BD380094329847C0B2286045E601287FF443AEA4
:10BD4800794E1020D6F8943298472B78C0F30742E2
:10BD58000093D6F88C52C0F3072300211020A8477F
:10BD680031E620B96F4B1B685B7E2B602BE6012800
:10BD78007FF429AED6F8E000044324E601287FF4D6
:10BD880022AE694B2968D3F89032112098471AE6F9
:10BD980088B9654B1520D3F8943298474FF08073D3
:10BDA800002808BF012093FBF0F0604B9842D4BFF5
:10BDB80028602B6007E601287FF405AE2B684FF05A
:10BDC8008076002B08BF012396FBF3F6574B15200E
:10BDD8009E42A8BF1E46544B3146D3F8903298472E
:10BDE8002E60F0E501287FF4EEAD4F4B2968D3F8BB
:10BDF800903233209847E6E540B94B4B6C20D3F896
:10BE080094329847C0F380402860DCE501287FF42D
:10BE1800DAAD454E6C20D6F8943298472B6820F45A
:10BE280080210BB141F48021D6F890326C209847DC
:10BE3800C9E540B93C4B6C20D3F894329847C0F31D
:10BE4800C0402860BFE501287FF4BDAD364E6C20A8
:10BE5800D6F8943298472B6820F400210BB141F4AE
:10BE68000021D6F890326C209847ACE501287FF481
:10BE7800AAAD2D4E6C20D6F8943298472B6820F442
:10BE880080210BB141F48021D6F890326C2098477C
:10BE980099E520B9264B1B681B682B6093E50128A0
:10BEA8007FF491ADD6F8E00004438CE560B91E4BF1
:10BEB8006C20D3F8943298474FF48073C0F3036032
:10BEC80043FA00F028607EE501287FF47CAD2A68FB
:10BED800102A23D00DDC022A1CD004DC012A16D03B
:10BEE8004FF0FF3214E0042A16D0082AF8D10522B0
:10BEF8000EE0402A14D003DC202AF1D1032207E007
:10BF0800802A17D0B2F5807FEAD1002200E008220B
:10BF18002A6010E00722FBE70622F9E70422F7E788
:10BF28000222F5E72410002068070020FFFF0F0019
:10BF3800641A002028602A68013210D0B04E6C20A4
:10BF4800D6F8943298472B6820F070611B0603F0EE
:10BF58007063D6F8902219436C20904733E5D3F8E4
:10BF6800EC0004432FE501287FF42DADA44E6C208E
:10BF7800D6F8943298472B6820F4C031DB0303F4D9
:10BF8800C033D6F8902219436C2090471BE540B97E
:10BF98009B4B6C20D3F894329847C0F380302860CC
:10BFA80011E501287FF40FAD954E6C20D6F8943238
:10BFB80098472B6820F480410BB141F48041D6F8B2
:10BFC80090326C209847FEE440B98D4B6C20D3F832
:10BFD80094329847C0F300302860F4E401287FF4D5
:10BFE800F2AC874E6C20D6F8943298472B6820F430
:10BFF80080510BB141F48051D6F890326C209847AB
:10C00800E1E49847D6F8943207466C2098473905FA
:10C01800C0F3021048BF40F008002860D3E40128AC
:10C028007FF4D1AC764E6C20D6F89432984710F451
:10C03800804F0FD0D6F894326C2098472B6820F4A4
:10C04800F061DB0103F4F063D6F8902219436C2009
:10C058009047B8E4D6F894326C2098472968D6F807
:10C0680090320A074CBF40F4006020F400600901D8
:10C0780020F07000C9B201436C209847A3E4F0B9DE
:10C088005F4E6C20D6F89432984710F4804FD6F85B
:10C0980094324FF06C0004D09847C0F30210286027
:10C0A80091E49847D6F8943207466C2098473B05A8
:10C0B800C0F3C31048BF40F00800286083E401289B
:10C0C8007FF481AC4E4E6C20D6F89432984710F429
:10C0D800804FD6F894324FF06C000CD098472B68FC
:10C0E80020F070011B0103F07003D6F89022194369
:10C0F8006C20904767E498472B6820F4F061DB01D7
:10C1080003F4F063D6F8902219436C2090475AE460
:10C1180040B93B4B6C20D3F89432984700F00F009D
:10C12800286050E401287FF44EAC354E6C20D6F8D8
:10C13800943298472B6820F00F0103F00F03D6F8CC
:10C14800902219436C2090473DE440B92C4B6D2058
:10C15800D3F894329847C0F3C030286033E40128FC
:10C168007FF431AC264E6D20D6F8943298472B6870
:10C1780020F400410BB141F40041D6F890326D2013
:10C18800984720E440B91E4B6D20D3F89432984765
:10C19800C0F34130286016E401287FF414AC184E2F
:10C1A8006D20D6F8943298472B6820F4C0415B0381
:10C1B80003F4C043D6F8902219436D20904702E457
:10C1C80001287FF400AC0E4E6D20D6F894329847C3
:10C1D8002B6820F470611B0203F47063D6F8902278
:10C1E80019436D209047FFF7EEBB58B9044B6D20FB
:10C1F800D3F894329847C0F341102860FFF7E3BBA7
:10C208006807002001287FF4DEABB34E6D20D6F816
:10C21800943298472B6820F060015B0103F06003BB
:10C22800D6F8902219436D209047FFF7CCBB48B948
:10C23800A94B6D20D3F89432984700F00F0028607E
:10C24800FFF7C1BB01287FF4BEABA34E6D20D6F823
:10C25800943298472B6820F00F0103F00F03D6F8AB
:10C26800902219436D209047FFF7ADBB01287FF45A
:10C27800AAAB994E6D20D6F8943298472B6820F0D7
:10C2880080710BB141F08071D6F890326D209847DB
:10C29800FFF799BB88B9904B6D20D3F89432984733
:10C2A800001410F0400F14BF6FF07F03002300F05C
:10C2B8007F0213432B60FFF786BB01287FF483AB13
:10C2C800854E6D20D6F8943298472B6820F4FE01ED
:10C2D8001B0403F4FE03D6F8902219436D209047FF
:10C2E800FFF771BB48B97C4B6C20D3F89432984760
:10C2F800C0F340402860FFF766BB01287FF463ABBA
:10C30800754E6C20D6F8943298472B6820F400318B
:10C318000BB141F40031D6F890326C209847FFF702
:10C3280052BB01287FF44FABD6F8E0000443FFF777
:10C338004ABB30B9694B53F82130DB692B60FFF7F2
:10C3480042BB01287FF43FAB644B2A6853F8213085
:10C35800DA610022624B1B6883F83020FFF733BB99
:10C3680001287FF430AB2A685E4E32B14FF08073FB
:10C3780093FBF2F39E42A8BF1E46574B3146D3F8B3
:10C388009032142098472E60FFF71DBB48B9524BD6
:10C398006C20D3F894329847C0F340302860FFF7F8
:10C3A80012BB01287FF40FAB4B4E6C20D6F89432A9
:10C3B80098472B6820F400510BB141F40051D6F88E
:10C3C80090326C209847FFF7FEBA48B9424B6C2070
:10C3D800D3F894329847C0F303502860FFF7F3BAB4
:10C3E80001287FF4F0AA3C4E6C20D6F89432984786
:10C3F8002B6820F470011B0503F47003D6F8902213
:10C4080019436C209047FFF7DEBA01287FF4DBAAB6
:10C418002B684FF08076002B08BF012396FBF3F6BC
:10C42800304B13209E42A8BF1E462B4B3146D3F8F3
:10C43800903298472E60FFF7C6BA48B9264B70204D
:10C44800D3F894329847C0F307202860FFF7BBBAA7
:10C4580001287FF4B8AA204E7020D6F89432984765
:10C46800296820F47F4040EA0121D6F890327020F4
:10C478009847D6F89432002098472A6833464AB13C
:10C4880040F00406D3F890323146002098472E60D9
:10C49800FFF799BA20F00406F4E740B90E4B702074
:10C4A800D3F894329847C0B22860FFF78CBA0128B5
:10C4B8007FF489AA084F7020D7F8943298472E78CD
:10C4C80020F0FF000643D7F8903231467020984795
:10C4D8002E60FFF778BA00BF6807002024100020FC
:10C4E800641A0020FFFF0F0001287FF46CAA2A6855
:10C4F800032A13D8364F7020D7F8943298472B6800
:10C5080020F440301E0406F440360643D7F8903233
:10C518003146702098472E60FFF755BAD6F8EC00E0
:10C528000443FFF750BA48B9294B7020D3F8943226
:10C538009847C0F380402860FFF745BA01287FF488
:10C5480042AA2A68012A13D8214F7020D7F89432BA
:10C5580098472B6820F480209E0406F48026064322
:10C56800D7F890323146702098472E60FFF72BBAE3
:10C57800D6F8EC000443FFF726BA48B9144B7020EC
:10C58800D3F894329847C0F301502860FFF71BBADC
:10C5980001287FF418AA0E4F7020D7F894329847D4
:10C5A8002B6820F440101E0506F440160643D7F801
:10C5B80090323146702098472E60FFF704BA012860
:10C5C8007FF401AAD6F8E0000443FFF7FCB900BFE6
:10C5D8006807002007B502AB43F8042D0246012086
:10C5E800FFF7E7F903B05DF804FB134602460020A5
:10C5F800FFF7DFB9014BD3F89032184768070020DE
:10C60800034B10B5D3F894320C469847206010BD00
:10C618006807002070B50D46144604287CD8DFE86A
:10C6280000F0032536424D0044F6206314689C420E
:10C6380018D842F210713A4B3A4ADB688C421B68B0
:10C64800106ADB6994BF00210121984742F21173F7
:10C65800B4FBF3F003FB1040334B80B29B68984760
:10C66800002070BD314BD3F8EC0070BD2C4B146822
:10C67800DB6858681B682CB10021DB6900F506707F
:10C688009847EDE79B6800F506709847E8E7284E5D
:10C698001168D6F8903228469847D6F8943228463A
:10C6A80098472060DCE71E4B1168DB681D4A1B6851
:10C6B8000031DB6918BF01211069E1E711681D4BE2
:10C6C800002203291BD8DFE801F002060C121B68C0
:10C6D80083F84C20C4E7184A1B68126892685A64A9
:10C6E800BEE7154A1B68126892689A64B8E7012287
:10C6F8001B6883F84C20596C19611A76B0E71B68DF
:10C7080083F84C200C4A126892685A6422689A642A
:10C718005A6C1A610122DBE7044BD3F8E00070BDC4
:10C728008C4D020830250020AC19002004000020A0
:10C738006807002024100020641A00201B4B70B5E5
:10C74800DD681B4C2B68A0685B6998472B682068DC
:10C758009B6898472B6860689B6898472B68206A95
:10C768009B6898472B68606A9B6898472B68E068C5
:10C778009B6898472B6820699B6898472B68606975
:10C788009B6898472B68A0699B6898472B68E06965
:10C798009B6898472B68A0689B689847054BDB689F
:10C7A8009847BDE87040044B5B6818478C4D0208F9
:10C7B80030250020641A0020AC19002038B50B4C35
:10C7C8002268126812B10A4B987870B1094B0A4D69
:10C7D800D3F89C329847AB6898470120074A2B68E2
:10C7E80011685268236059629A6238BD241000208B
:10C7F800341A002068070020641A00203025002021
:10C80800094B93F87920824202D8D3F8E8007047A0
:10C81800064A52F82020116101211176002182F880
:10C828004C10D3F8D40070470400002024100020D6
:10C83800034B0A681B689B6813440B601946DFE7C3
:10C848002410002010B50D4A92F87930834202D89E
:10C85800D2F8E80010BD01200024094B1B681876A7
:10C8680083F84C40074C2468A4685C645C6C1C61C9
:10C87800996483F84C00D2F8D40010BD040000205D
:10C8880024100020641A002038B50D4C0D4DD4F842
:10C89800883298472B6893F8302082B993F8403053
:10C8A8006BB1D4F894326F209847D4F894326F2043
:10C8B8009847C30142BF01222B6883F8302038BD56
:10C8C80068070020641A0020084B93F879208242F8
:10C8D80002D8D3F8E80070470028FAD1044A126851
:10C8E80012680A60D3F8D400704700BF0400002023
:10C8F800641A0020022804BF0B4B93F8D10030B90A
:10C908000A4BDB681B685B69094A9068184701286D
:10C9180009D1054B93F8D130012B04D1034BDB68C7
:10C928001B689B69F0E77047040000208C4D0208E3
:10C93800302500202DE9F041694D6A4CEE686A4FB8
:10C948007368DFF8FC8103F1C802A26003F5B872CE
:10C95800226003F5C672626003F5F072226203F585
:10C96800FE72626203F55372E26003F55A7203F5D0
:10C978006870226103F5617203F56F73E3613368D0
:10C9880062611B69A06198473368E0691B69984731
:10C99800336860691B69984733682068DB68984783
:10C9A80033686068DB6898473368A068DB68984735
:10C9B80033682069DB6898473368E068DB68984724
:10C9C8003368606ADB6898473368206ADB68984791
:10C9D8003368606A9B6998473368206A9B699847FF
:10C9E800336860699B6998473368E0689B69984732
:10C9F8002A693E4D02F110033B60736803F50D731D
:10CA08005361EB6FC7F89832D8F808309847D8F8D0
:10CA18000030374A4FF001081360226802205A623A
:10CA280062689A62EB6F334AC3F80422D7F8A022EF
:10CA38000027C3F80C221F705F702F4B85F8798090
:10CA4800C5F888302D4B85F8D080C5F884302C4B3C
:10CA5800C5F880302B4BC5F88C302B4BC5F8A0306F
:10CA68002A4BC5F89C302A4BC5F89030294BC5F89D
:10CA78009430294BC5F89830284BC5F8B030284B6E
:10CA8800C5F8AC30274BC5F8BC30274BC5F8B830D3
:10CA9800264BC5F8B430264BC5F8CC3032236B672B
:10CAA8004FF4F0732B67234BC5F8C030224BC5F801
:10CAB800C430FFF71FFF0222636A197C5A74186892
:10CAC800424614F02BF83368606A1C4C1B68984780
:10CAD80023689847A3683846BDE8F041184700BF67
:10CAE8008C4D020830250020680700200400002033
:10CAF80024100020C5C7000885B90008B1B900088E
:10CB0800B3B90008B7B90008F3C50008DDC50008C7
:10CB180009C8000839C800084DC80008FDC5000844
:10CB280009C6000891C800081DC60008D1C8000839
:10CB3800FDC800083DC9000845C70008AC19002019
:10CB4800641A00200FF0C4BD0FF0EEBD0FF04CBE0C
:10CB58000FF07CBE084B93F87920824289BF074AC0
:10CB6800D3F8E80052F82020002082BF1076D16068
:10CB7800D3F8D400704700BF040000202C10002018
:10CB8800E8E74942E6E70021E4E7084B93F8792013
:10CB9800824289BF064AD3F8E80052F82020D3F829
:10CBA800D40082BF11610121117670470400002072
:10CBB8002C100020034B0A681B689B6813440B6009
:10CBC8001946E2E72C10002010B5194B044693F8DB
:10CBD80079008842194602D8D3F8E80010BDD3F886
:10CBE800D400052C1FD8DFE804F003070B0F131A35
:10CBF800104B1B681A6110BD0E4B1B689A6010BD64
:10CC08000C4B1B68DA6010BD0A4B1B681A6010BD1C
:10CC1800084B002A1B68B8BF52425A6110BD054B29
:10CC28001B685A6010BDD1F8E030184310BD00BF32
:10CC3800040000202C1000200022014BDA66704707
:10CC48000400002000207047044B9B691A781AB929
:10CC580001205A701870704700207047B84D0020A6
:10CC6800054B9B691A7822B902215A701970012064
:10CC780070470020704700BFB84D0020022804BF4D
:10CC88000B4B93F8D10030B90A4BDB681B685B6922
:10CC9800094A10681847012809D1054B93F8D13083
:10CCA800012B04D1034BDB681B689B69F0E77047D5
:10CCB800040000208C4D02086425002070B54C4EFD
:10CCC8004C4CF5686B6803F5B872626003F5C67280
:10CCD800A26003F58E72E26003F59C7203F1C8004E
:10CCE800226103F1E40203F58073A3612B6862619A
:10CCF800DB68206098472B686068DB6898472B687A
:10CD0800A068DB6898472B68E068DB6898472B6861
:10CD18002069DB6898472B6860691B6998472B680E
:10CD2800A0691B699847F56A334E2B689847334BBF
:10CD38003349DA6F0D608A614FF4F851E165314982
:10CD48000125C4F8CC113049C4F8DC112F49C2F8C8
:10CD580004122F49C2F80C12002111702D4A83F8D1
:10CD68007950C3F888202C4A83F8D050C3F884201F
:10CD78002A4AC3F880202A4AC3F88C20294AC3F8D3
:10CD8800A020294AC3F89C20284AC3F89020284AA2
:10CD9800C3F89420274AC3F8B020274AC3F8AC2028
:10CDA800264AC3F8B820264AC3F8CC20254AC3F837
:10CDB800C82032225A674FF4C3721A67224AC3F84E
:10CDC800C020224AC3F8C420214AC3F8BC20B36853
:10CDD800984733681F4A2846136062685A62A268F7
:10CDE800BDE870409A624FF448425A615A6045E77C
:10CDF8008C4D020864250020641A002004000020DD
:10CE0800B84D00205300001024000DC151CC00087B
:10CE180069CC00085DCB000889CB00088BCB0008E3
:10CE28008FCB0008C5D10008D1CB000893CB0008F0
:10CE3800BDCB0008B9D00008ABCE00084DCC000827
:10CE480085CC000841CC0008C5CC000861CE00089C
:10CE580065D100082C10002010B50020FFF70EFF48
:10CE6800BDE81040034B044ADB6810681B689B68E8
:10CE7800184700BF8C4D020864250020072310B511
:10CE880001FA03F200F0800402F08002A2424FEAA5
:10CE9800400018BF80F0070013F1FF33C0B2EFD293
:10CEA80010BD804B2DE9F34100F07F07DB5D0E4696
:10CEB80013F0010F7C4C06D104EB8704E3690B6087
:10CEC80002B0BDE8F08105210020FFF7D7FF00215F
:10CED800FFF7D4FF3946FFF7D1FF8046734D2B6823
:10CEE8009B6998472B6805209B6898472B6800200A
:10CEF8009B6898472B6838469B6898472B6840463C
:10CF08009B6898470FF07CF8C4F81C022B680DF159
:10CF18000700DB689847002871D09DF80730052B7B
:10CF28006DD10FF06DF8C4F81C022B680DF10700E5
:10CF3800DB68984700286ED00FF062F8C4F81C022E
:10CF48002B680DF10700DB68984700286FD00FF0B9
:10CF580057F8C4F81C022B680DF10700DB689847E6
:10CF6800002870D09DF8073033600FF049F8C4F8F6
:10CF78001C022B680DF10700DB68984700286ED06B
:10CF880032689DF8073043EA022333600FF038F81F
:10CF9800C4F81C022B680DF10700DB6898470028CD
:10CFA80069D032689DF8073043EA022333600FF0F6
:10CFB80027F8C4F81C022B680DF10700DB689847B6
:10CFC800002863D032689DF8073043EA02233360B3
:10CFD8000FF016F8C4F81C022B680DF10700DB6887
:10CFE800984700287FF46CAF0FF00AF8D4F81C3289
:10CFF800C01A0028B8BF40420A28EDDD60E70EF0ED
:10D00800FFFFD4F81C32C01A0028B8BF40420A28D3
:10D018007FF77CAF54E70EF0F3FFD4F81C32C01A48
:10D028000028B8BF40420A287FF77FAF48E70EF0D4
:10D03800E7FFD4F81C32C01A0028B8BF40420A28BB
:10D048007FF77EAF3CE70EF0DBFFD4F81C32C01A46
:10D058000028B8BF40420A287FF77DAF30E70EF0BE
:10D06800CFFFD4F81C32C01A0028B8BF40420A28A3
:10D078007FF77FAF24E70EF0C3FFD4F81C32C01A45
:10D088000028B8BF40420A2884DD19E70EF0B8FF2F
:10D09800D4F81C32C01A0028B8BF40420A288ADDDA
:10D0A8000EE700BF804C020864250020B84D002020
:10D0B8002DE9F74F06460D4600200521FFF7DEFE55
:10D0C80046F0800B0021FFF7D9FE4FEA156A594652
:10D0D800FFF7D4FEC5F307495146FFF7CFFEC5F366
:10D0E80007284946FFF7CAFEEFB24146FFF7C6FEDA
:10D0F8003946FFF7C3FE174C0190236806F07F06F8
:10D108009B699847236805209B68984723680020F7
:10D118009B689847236858469B68984723685046F9
:10D128009B689847236848469B6898472368404609
:10D138009B689847236838469B6898472368019AF4
:10D148009B6810469847044B03EB8606F56103B0CD
:10D15800BDE8F08FB84D00206425002070B5144D4F
:10D168000646AA69137813B3124CD4F82032C31AAE
:10D17800002BB8BF5B42022B19DD0F4901E00130DB
:10D188005070507803060FD40B5C023B012BF6D885
:10D1980004EB8003D969FFF78BFFAA695378013341
:10D1A8005370C4F8206270BD00231370F9E770BD96
:10D1B800B84D002064250020804C020810B5184B9B
:10D1C800044693F879008842194602D8D3F8E80053
:10D1D80010BDD3F8D400052C1DD8DFE804F00308EF
:10D1E8000C1014180F4B1B681B69136010BD0D4BF6
:10D1F8001B689B68F9E70B4B1B68DB68F5E7094B75
:10D208001B681B68F1E7074B1B685B69EDE7054B7B
:10D218001B685B68E9E7D1F8E030184310BD00BF30
:10D22800040000202C100020084B93F8792082423B
:10D2380089BF074AD3F8E80052F82020002082BFAF
:10D248001076D160D3F8D400704700BF04000020E6
:10D2580034100020E8E74942E6E70021E4E7084BFC
:10D2680093F87920824289BF064AD3F8E80052F839
:10D278002020D3F8D40082BF1161012111767047B4
:10D288000400002034100020034B0A681B689B68C8
:10D2980013440B601946E2E73410002010B5194B0F
:10D2A800044693F879008842194602D8D3F8E80072
:10D2B80010BDD3F8D400052C1FD8DFE804F003070D
:10D2C8000B0F131A104B1B681A6110BD0E4B1B680D
:10D2D8009A6010BD0C4B1B68DA6010BD0A4B1B68C6
:10D2E8001A6010BD084B002A1B68B8BF52425A6129
:10D2F80010BD054B1B685A6010BDD1F8E0301843CB
:10D3080010BD00BF04000020341000200022014B93
:10D31800DA6670470400002000207047044B9B69C0
:10D328001A781AB901205A7018707047002070478F
:10D33800B84D0020054B9B691A7822B902215A7012
:10D348001970012070470020704700BFB84D0020B9
:10D35800022804BF0B4B93F8D10030B90A4BDB68A5
:10D368001B685B69094A10681847012809D1054BF1
:10D3780093F8D130012B04D1034BDB681B689B6900
:10D38800F0E77047040000208C4D02089427002025
:10D3980070B54C4E4C4CF5686B6803F5B87262601A
:10D3A80003F5C672A26003F58E72E26003F59C7203
:10D3B80003F1C800226103F1E40203F58073A3615D
:10D3C8002B686261DB68206098472B686068DB68BF
:10D3D80098472B68A068DB6898472B68E068DB688B
:10D3E80098472B682069DB6898472B6860691B6938
:10D3F80098472B68A0691B699847F56A334E2B68D4
:10D408009847334B3349DA6F0D608A614FF4F8510E
:10D41800E16531490125C4F8CC113049C4F8DC1163
:10D428002F49C2F804122F49C2F80C1200211170BA
:10D438002D4A83F87950C3F888202C4A83F8D050B5
:10D44800C3F884202A4AC3F880202A4AC3F88C20CB
:10D45800294AC3F8A020294AC3F89C20284AC3F8BF
:10D468009020284AC3F89420274AC3F8B020274AB6
:10D47800C3F8AC20264AC3F8B820264AC3F8CC2003
:10D48800254AC3F8C82032225A674FF4C3721A6774
:10D49800224AC3F8C020224AC3F8C420214AC3F84C
:10D4A800BC20B368984733681F4A284613606268EF
:10D4B8005A62A268BDE870409A624FF448425A61C5
:10D4C8005A6045E78C4D020894270020641A002012
:10D4D80004000020B84D00205300001024000DC1A6
:10D4E80025D300083DD3000831D200085DD20008DA
:10D4F8005FD2000863D2000899D80008A5D20008B6
:10D5080067D2000891D200088DD700087FD500089F
:10D5180021D3000859D3000815D3000899D300086F
:10D5280035D5000839D800083410002010B500207F
:10D53800FFF70EFFBDE81040034B044ADB68106894
:10D548001B689B68184700BF8C4D02089427002071
:10D55800072310B501FA03F200F0800402F08002FC
:10D56800A2424FEA400018BF80F0070013F1FF33D2
:10D57800C0B2EFD210BD804B2DE9F34100F07F0718
:10D58800DB5D0E4613F0010F7C4C06D104EB8704DB
:10D59800E3690B6002B0BDE8F08105210020FFF7C8
:10D5A800D7FF0021FFF7D4FF3946FFF7D1FF8046A8
:10D5B800734D2B689B6998472B6805209B68984793
:10D5C8002B6800209B6898472B6838469B689847CB
:10D5D8002B6840469B6898470EF012FDC4F81C0261
:10D5E8002B680DF10700DB689847002871D09DF87B
:10D5F8000730052B6DD10EF003FDC4F81C022B6813
:10D608000DF10700DB68984700286ED00EF0F8FC93
:10D61800C4F81C022B680DF10700DB689847002846
:10D628006FD00EF0EDFCC4F81C022B680DF107005A
:10D63800DB689847002870D09DF8073033600EF0FB
:10D64800DFFCC4F81C022B680DF10700DB68984763
:10D6580000286ED032689DF8073043EA0223336011
:10D668000EF0CEFCC4F81C022B680DF10700DB6835
:10D678009847002869D032689DF8073043EA0223AA
:10D6880033600EF0BDFCC4F81C022B680DF10700D6
:10D69800DB689847002863D032689DF8073043EA72
:10D6A800022333600EF0ACFCC4F81C022B680DF1A9
:10D6B8000700DB68984700287FF46CAF0EF0A0FCE9
:10D6C800D4F81C32C01A0028B8BF40420A28EDDD41
:10D6D80060E70EF095FCD4F81C32C01A0028B8BFD9
:10D6E80040420A287FF77CAF54E70EF089FCD4F853
:10D6F8001C32C01A0028B8BF40420A287FF77FAF03
:10D7080048E70EF07DFCD4F81C32C01A0028B8BFD8
:10D7180040420A287FF77EAF3CE70EF071FCD4F850
:10D728001C32C01A0028B8BF40420A287FF77DAFD4
:10D7380030E70EF065FCD4F81C32C01A0028B8BFD8
:10D7480040420A287FF77FAF24E70EF059FCD4F84F
:10D758001C32C01A0028B8BF40420A2884DD19E7E5
:10D768000EF04EFCD4F81C32C01A0028B8BF404254
:10D778000A288ADD0EE700BF004D02089427002022
:10D78800B84D00202DE9F74F06460D46002005212B
:10D79800FFF7DEFE46F0800B0021FFF7D9FE4FEAC7
:10D7A800156A5946FFF7D4FEC5F307495146FFF7F6
:10D7B800CFFEC5F307284946FFF7CAFEEFB2414638
:10D7C800FFF7C6FE3946FFF7C3FE174C01902368E2
:10D7D80006F07F069B699847236805209B68984751
:10D7E800236800209B689847236858469B68984799
:10D7F800236850469B689847236848469B68984723
:10D80800236840469B689847236838469B68984732
:10D818002368019A9B6810469847044B03EB8606D9
:10D82800F56103B0BDE8F08FB84D002094270020C3
:10D8380070B5144D0646AA69137813B3124CD4F880
:10D848002032C31A002BB8BF5B42022B19DD0F49E7
:10D8580001E001305070507803060FD40B5C023B96
:10D86800012BF6D804EB8003D969FFF78BFFAA696F
:10D87800537801335370C4F8206270BD00231370CD
:10D88800F9E770BDB84D002094270020004D02082C
:10D8980010B5184B044693F879008842194602D807
:10D8A800D3F8E80010BDD3F8D400052C1DD8DFE864
:10D8B80004F003080C1014180F4B1B681B69136045
:10D8C80010BD0D4B1B689B68F9E70B4B1B68DB68A9
:10D8D800F5E7094B1B681B68F1E7074B1B685B6999
:10D8E800EDE7054B1B685B68E9E7D1F8E0301843C2
:10D8F80010BD00BF040000203410002028B101280A
:10D908000AD0094BD3F8E00070471368074AB3FA06
:10D9180083F35B09937370471368054AB3FA83F37B
:10D928005B091360002070470400002030010020CC
:10D938003C100020084B93F87920824289BF074A9F
:10D94800D3F8E80002EB8000426881BFD3F8D40026
:10D958001161012111767047040000203C1000205D
:10D96800034B0A685B689B6813440B601946E1E740
:10D978003C10002070B51D46A54B93F879408C42A9
:10D98800194603D8D3F8E840204670BDA82AD3F832
:10D99800D44000F0488264D81D2A00F04F8124D872
:10D9A800042A00F0FE800ED8012A00F0D080C0F0D2
:10D9B800C080022A00F0D980032A00F0E480D1F860
:10D9C800E0000443E0E7062A00F00A81C0F0FA808C
:10D9D800072A00F01881082AF1D1002840F0278191
:10D9E8008C4B5B685B7E2B60CEE7A32A00F0B4818A
:10D9F80022D8A02A00F074810ED88C2ADFD1002802
:10DA080040F02981844B08201B6C984700F00F00D8
:10DA1800C0F108002860B7E7A12A00F07881A22A9F
:10DA2800CDD1002840F08A817B4B0C201B6C984795
:10DA3800C0F3C1302860A7E7A52A00F0BB81C0F079
:10DA4800A281A62A00F0CD81A72AB8D1002840F0EB
:10DA5800DE81714B0C201B6C984700F00F0028608A
:10DA680092E7B22A00F0B5822AD8AD2A00F04282A5
:10DA780011D8AA2A00F00582C0F0EC81AB2A00F088
:10DA88001B82AC2A9BD1002840F02C82634B1B6878
:10DA98005B6B2B6078E7AF2A00F05F82C0F04182B1
:10DAA800B02A00F07182B12A89D1002840F083821F
:10DAB800594B0F201B6C9847C0F38020286063E700
:10DAC800B72A00F0DC8212D8B42A00F0AF82C0F086
:10DAD8009782B52A00F0BA82B62A7FF470AF002880
:10DAE80040F0C5824B4B5B681B6A2B604CE7CE2A23
:10DAF80000F0008310D8B82A00F0D782B92A7FF442
:10DB08005EAF002840F0E882434B0F201B6C98471B
:10DB1800C0F30040286037E7D02A00F00483D62AF3
:10DB28007FF44DAF002840F013833B4B9B682B607C
:10DB38002AE720B9374B5B681B692B6024E701286B
:10DB48007FF422AF334B2A685B681A611CE720B95F
:10DB5800304B5B689B682B6016E701287FF414AF95
:10DB68002C4B2A685B689A600EE720B9294B5B68E2
:10DB7800DB682B6008E701287FF406AF254B2A688D
:10DB88005B68DA6000E720B9224B5B681B682B6092
:10DB9800FAE601287FF4F8AE1E4B2A685B681A6023
:10DBA800F2E620B91B4B5B685B692B60ECE6012849
:10DBB8007FF4EAAE174B5A682B68002BB8BF5B425C
:10DBC8005361E1E620B9134B5B685B682B60DBE6C9
:10DBD80001287FF4D9AE0F4B2A685B685A60D3E6F8
:10DBE80018B90D4BDB7B2B60CEE601287FF4CCAE59
:10DBF8002A68094B1F21DA732A68DB6C02F01F02BE
:10DC080006209847C0E658B9034B1B792B60BBE642
:10DC1800040000203C10002030010020641A00207D
:10DC280001287FF4B1AE2A68A14B1A71ACE601282D
:10DC38007FF4AAAED3F8E0000443A5E620B99D4BD3
:10DC48005B681B682B609FE601287FF49DAED3F8C4
:10DC5800E000044398E601287FF496AE2B68102B69
:10DC680023D00DDC022B1CD004DC012B16D04FF086
:10DC7800FF3314E0042B16D0082BF8D105230EE04F
:10DC8800402B14D003DC202BF1D1032307E0802B99
:10DC98000FD0B3F5807FEAD1002300E008232B6082
:10DCA80008E00723FBE70623F9E70423F7E7022345
:10DCB800F5E728602A687E4E501C0DD0F36C02F000
:10DCC8000F020F21002098472A68F36C02F00F0218
:10DCD8000F210020984757E6D1F8EC301C43F3E7B2
:10DCE80038B9734B08201B6C9847C0F34020286054
:10DCF8004AE601287FF448AE2A686D4B5202DB6C75
:10DD080002F400724FF40071002098473CE638B9DD
:10DD1800674B08201B6C9847C0F30020286033E647
:10DD280001287FF431AE2A68614B1202DB6C02F4E1
:10DD380080724FF480710020984725E601287FF40F
:10DD480023AE2A685A4BD203DB6C02F4C0324FF47C
:10DD5800C0310420984717E638B9554B0C201B6C86
:10DD68009847C0F3803028600EE601287FF40CAE97
:10DD78002A684F4B9203DB6C02F480424FF48041D7
:10DD88000420984700E638B9494B0C201B6C98478B
:10DD9800C0F3C1202860F7E501287FF4F5AD2A68B3
:10DDA800434BD202DB6C02F4C0524FF4C051042042
:10DDB8009847E9E538B93E4B0C201B6C9847C0F3EF
:10DDC800C3102860E0E501287FF4DEAD2A68384BEF
:10DDD800D201DB6C02F4F0624FF4F0610420984742
:10DDE800D2E538B9324B0C201B6C9847C0F30210AF
:10DDF8002860C9E501287FF4C7AD2A682C4B1201B9
:10DE0800DB6C02F07002702104209847BCE5012801
:10DE18007FF4BAAD2A68264B02F00F02DB6C0F21A3
:10DE280004209847B0E538B9214B0D201B6C984762
:10DE3800C0F3C0302860A7E501287FF4A5AD2A68A3
:10DE48001B4BD203DB6C02F400424FF40041052067
:10DE5800984799E538B9164B0D201B6C9847C0F3C5
:10DE68004130286090E501287FF48EAD2A68104B78
:10DE78005203DB6C02F4C0424FF4C04105209847BE
:10DE880082E538B90A4B0D201B6C9847C0F3032074
:10DE9800286079E501287FF477AD2A68044B1202DF
:10DEA800DB6C02F470624FF47061052098476BE5F3
:10DEB800300100203C10002038B9A24B0D201B6C0B
:10DEC8009847C0F3411028605EE501287FF45CADF7
:10DED8002A689C4B5201DB6C02F06002602105202D
:10DEE800984751E501287FF44FAD974B2A681B6886
:10DEF8005A6349E538B9934B0E201B6C9847C0F319
:10DF08000040286040E501287FF43EAD2A688D4B2B
:10DF18001204DB6C02F480324FF4803106209847FB
:10DF280032E560B9874B0E201B6C9847000A00F059
:10DF38007F03420648BF63F07F032B6024E5012876
:10DF48007FF422AD2A687F4B1202DB6C02F4FE429A
:10DF58004FF4FE410620984716E538B9794B0F2053
:10DF68001B6C9847C0F3813028600DE501287FF4C9
:10DF78000BAD2A68734B9203DB6C02F440424FF4FA
:10DF8800404107209847FFE438B96E4B0F201B6CBF
:10DF98009847C0F301302860F6E401287FF4F4AC18
:10DFA8002A68684B1203DB6C02F440524FF440516C
:10DFB80007209847E8E401287FF4E6AC2A68614B1B
:10DFC8009202DB6C02F480624FF48061072098476C
:10DFD800DAE438B95B4B0F201B6C9847C0F301207B
:10DFE8002860D1E401287FF4CFAC2A68554B12028F
:10DFF800DB6C02F440724FF4407107209847C3E489
:10E0080038B9504B0F201B6C9847C0F3801028601C
:10E01800BAE401287FF4B8AC2A684A4B9201DB6C59
:10E0280002F04002402107209847ADE438B9454B3B
:10E0380002201B6C9847C0F384202860A4E40128C0
:10E048007FF4A2ACD3F8E00004439DE420B93F4B31
:10E058005B68DB692B6097E401287FF495AC3B4B48
:10E068002A685B68DA61002283F830208CE4012892
:10E078007FF48AAC354B2A685B681A6284E438B945
:10E08800304B0F201B6C9847C0F3C01028607BE40E
:10E0980001287FF479AC2A682A4BD201DB6C02F0A4
:10E0A80080028021072098476EE438B9254B0C2060
:10E0B8001B6C9847C0F34030286065E401287FF462
:10E0C80063AC2A681F4B5203DB6C02F400524FF416
:10E0D80000510420984757E401287FF455AC2A687A
:10E0E800184B1204DB6C02F480324FF480310720A5
:10E0F800984749E480B9154B1A68124B1B6C32B12A
:10E1080002209847800A00F4787028603CE40120D7
:10E118009847C0F38920F8E701287FF435ACD3F895
:10E12800E000044330E430B9064B03201B6C9847E9
:10E13800C0B2286028E401287FF426ACD3F8E000B8
:10E14800044321E430010020641A00203C10002020
:10E1580001287FF419AC2A68014B9A6014E400BFC7
:10E168003001002007B502AB43F8042D0246012018
:10E17800FFF700FC03B05DF804FB134602460020DD
:10E18800FFF7F8BB014BDB6B184700BF30010020DD
:10E19800034B10B51B6C0C469847206010BD00BFA0
:10E1A80030010020034B00F00F02DB6C0F2105202B
:10E1B800184700BF3001002010B50B4CA36B9847DF
:10E1C800237B0A4A43B1D36E43F00103617B39B123
:10E1D80043F00203D36610BDD36E23F00103F5E7C5
:10E1E80023F00203F6E700BF3001002004000020FE
:10E1F80010B50A4B93F87920824202D8D3F8E80088
:10E2080010BD0022064C62732273064C04EB80009A
:10E2180040680276C160D3F8D40010BD0400002025
:10E22800300100203C100020E2E74942E0E70021ED
:10E23800DEE7084B93F87920824202D8D3F8E80049
:10E2480070470028FAD1044A126812680A60D3F8A5
:10E25800D400704704000020641A0020022804BF7C
:10E268000B4B93F8D10030B90A4BDB681B685B692C
:10E27800094AD0681847012809D1054B93F8D130CD
:10E28800012B04D1034BDB681B689B69F0E77047DF
:10E29800040000208C4D0208C42900202DE9F84311
:10E2A8000126DFF88C814C4DD8F80C404B4F636841
:10E2B8003E6003F1C802EA6003F1E40203F5B870B6
:10E2C8002A6103F5C67203F50D732B602368AA60F3
:10E2D800DB68686098472368A868DB689847236804
:10E2E800E868DB689847236828691B6998472368AA
:10E2F8002868DB6898476068236820309B686861F5
:10E308009847D8F810204FF00008354B02F110015B
:10E31800344C19612968DFF81C915161E26F996CDE
:10E328005A61C2F80C12304982F8008082F80180E4
:10E33800C2F8041205221A714FF47A729A60D9F859
:10E3480008309847D9F800306A68C3F838805A62AC
:10E35800AA687B609A622A690220DA62234A1A65EF
:10E36800234B84F87960C4F88830224B84F8D06055
:10E37800C4F88430204BC4F88030204BC4F88C306B
:10E388001F4BC4F8A0301F4BC4F89C301E4BC4F878
:10E3980090301E4BC4F894301D4BC4F8B0301D4B60
:10E3A800C4F8AC301C4BC4F8BC301C4BC4F8B830B3
:10E3B8001B4BC4F8B4301B4BC4F8CC303223636712
:10E3C80040F225132367184BC4F8C030174BC4F824
:10E3D800C430BDE8F84341E7C42900203C100020C0
:10E3E800300100200400002095E40008ADE1000899
:10E3F800F9E1000831E2000833E2000837E20008DA
:10E4080083E100086DE100083DD9000869D90008DA
:10E418008DE1000899E10008C1E1000805D900086C
:10E428003BE2000865E20008A5E2000841E40008B4
:10E438008C4D0208641A002070B50020FFF70EFF0B
:10E448000F4B104CDD68E0682B685B6998472B68B8
:10E4580020689B6898472B68A0689B6898472B683A
:10E46800E0689B6898472B6820699B6898472B68E9
:10E4780060689B689847BDE87040034BDB681847A5
:10E488008C4D0208C4290020641A002038B50A4DB2
:10E498006B681B6813B1094B987860B1084B01246D
:10E4A8005B6C984700226B68022083F830202C6050
:10E4B800FFF7D4FE204638BD3C100020341A002057
:10E4C80030010020014BD3F890301847600F00202E
:10E4D800034B10B5D3F894300C469847206010BD14
:10E4E800600F00200022014B5A6070470400002092
:10E4F80070B5434E434CF5686B6803F59C72E26156
:10E5080003F5AA72A26103F55372626103F55A72A8
:10E51800226103F5617203F57670E26003F56872B3
:10E5280003F57D7323602B68A260DB686060984701
:10E538002B686069DB6898472B682069DB68984717
:10E548002B68E068DB6898472B68A068DB68984709
:10E558002B6860685B6998472B6860695B699847B6
:10E568002B6820695B6998472B68E0685B69984766
:10E578002B68A0685B6998472B68E0691B69984716
:10E588002B68A0691B6998472B6820681B69984706
:10E598006B681D4A316903F537734B6011600121BF
:10E5A8001A4B82F8A51058695974C2F8A800184A7D
:10E5B800C0F80422174A1A62174ADA61174A9A61A0
:10E5C800174A5A62174A9A63174A5A63174A9A624D
:10E5D800174ADA62174A9A64174A5A64174A5A65F8
:10E5E800174A1A65174A1A6693F8D020002A08BFF6
:10E5F8000A4683F8D020144A9A65144ADA6570BD31
:10E608008C4D0208E8290020600F0020040000203B
:10E61800CDE7000881E80008DDE80008DFE8000829
:10E62800E3E80008E7E8000859EA00086DE7000891
:10E63800A9E70008CDE40008D9E4000861E800086B
:10E6480059E60008EDE40008F9E4000809E70008C5
:10E658000128F8B5144633D005D3FF28254C40D0FF
:10E66800D4F8E000F8BD136833F0030224D113F0A6
:10E67800010F214D214E0FD0F3681B681B692869D3
:10E688009847246814F002040ED0F3681B681B69CD
:10E69800686998470020F8BDF76828693B68DB6817
:10E6A80098473B689B69EAE7F66868693368DB68FE
:10E6B800984733689B69EBE70E4BD3F8EC00F8BD3D
:10E6C80014680D4D0D4B24B1DB681B681B69E868A5
:10E6D800DFE7DE68E8683368DB68984733689B697A
:10E6E800F5E7E36FD3F8043298476369D3F8043247
:10E6F8009847CFE704000020E82900208C4D020845
:10E7080070B5164E164CF56860682B689B6998477B
:10E718002B6860699B6898472B6820699B689847B5
:10E728002B68E0689B6898472B68A0689B689847A7
:10E738002B68E0699B6898472B68A0699B68984795
:10E748002B6820689B6898472B6860689B68984787
:10E758003369BDE87040DB69184700BF8C4D02087B
:10E76800E829002070B50C4C0E46637C834202D821
:10E77800D4F8E80070BD094D202095F8A510D5F80B
:10E78800903041F004019847D5F890303146372051
:10E798009847D4F8D40070BD04000020600F002012
:10E7A80038B5074B0C460546D3F8942093F8A400D7
:10E7B80090472368C11821602846BDE83840D1E752
:10E7C800600F002038B5204C204AD4F8A830D26811
:10E7D800197825461E4B126841B9926958689047C6
:10E7E8000122D4F8A8301A70012038BD194C52699A
:10E7F8005868904794F86820012A1ED0032A20D030
:10E80800012A4FF00F0319D04FF4A02143F0884399
:10E8180043F04013D5F89020194304209047D5F8C9
:10E8280090300421102098470022D5F8A8301A709B
:10E83800E36FD3F804329847D6E70B234FF420311F
:10E84800E4E70D23E0E700BF600F00208C4D0208CD
:10E85800E82900200400002010B5064CD4F88830C0
:10E868009847D4F8A8301B7813B1BDE81040A9E741
:10E8780010BD00BF600F002070B5124B0C465A7CCB
:10E888001E46824202D8D3F8E80070BD0E4D202003
:10E89800D5F8903095F8A510984784EAE4710B4BA9
:10E8A800A1EBE4719942D5F8902004DD084911EAFA
:10E8B800240438BF1C46210224209047D6F8D400EF
:10E8C80070BD00BF04000020600F002000127A0015
:10E8D80000EE85FFD0E74942CEE70021CCE738B506
:10E8E800594B15465A7C8A421A4603D8D3F8E84051
:10E8F800204638BD1128D3F8D4407DD025D8042827
:10E9080060D00AD8012853D04CD302285AD0032803
:10E9180053D0D2F8E0000443EAE70E2861D00BD8C0
:10E92800052857D00828F4D1484B0F20D3F8943045
:10E93800984700F001004BE00F2858D01028E8D184
:10E94800424B2A20D3F8943048E0172868D014D8CE
:10E9580014285BD008D8122853D01328D9D13B4BA0
:10E968002B20D3F8943039E0152854D01628D0D16C
:10E97800364B2D20D3F8943018E01A285AD008D8EE
:10E98800182852D01928C4D1304B3020D3F89430ED
:10E998000CE01B2853D0D628BBD12C4B1520D3F81C
:10E9A800943003E03720294BD3F8943098470FE090
:10E9B800264B2120D3F89430F8E7244B2220D3F8B3
:10E9C8009430F3E7214B2420D3F894309847001271
:10E9D80028608DE728201D4BD3F894309847801085
:10E9E800F6E71A4B93F8A5305B002B6080E7174BCE
:10E9F8002520D3F89430D9E7144B2920D3F8943044
:10EA0800ECE7124B2720D3F89430CFE70F4B2620A2
:10EA1800D3F89430CAE70D4B2C20D3F89430C5E7CF
:10EA28000A4B2E20D3F89430C0E7084B2F20D3F898
:10EA38009430BBE7054B3320D3F89430B6E7034B4B
:10EA48003420D3F89430B1E704000020600F002090
:10EA580038B5744B5C7C8C42194603D8D3F8E8402F
:10EA6800204638BD1128D3F8D44000F0A28020D821
:10EA780004286BD009D801285CD054D3022865D06B
:10EA880003285DD0D1F8E00011E00E287DD004D82D
:10EA980005286ED00828E3D0F4E70F287DD0102889
:10EAA800F0D1930D9B05002B7DD0D1F8EC000443E9
:10EAB800D6E7172800F09D801BD8142800F089801D
:10EAC8000DD812287FD01328DCD1930D9B05002B7D
:10EAD800EBD1554B9100D3F890302B2028E0152826
:10EAE8007DD01628CED1504B1146D3F890302D202A
:10EAF8001EE01A2800F0898009D818287FD0192824
:10EB0800C0D1494B1146D3F89030302010E01B2873
:10EB180000F08180D628B5D1434B4449D3F89030D2
:10EB28005143152004E0114637203F4BD3F890306D
:10EB3800984795E73C4B1146D3F890302120F7E7EA
:10EB4800394B1146D3F890302220F1E7364B82EA50
:10EB5800E271D3F89050364BA1EBE271994204DD93
:10EB6800344911EA220238BF1A4611022420A84764
:10EB780076E7910D890511B1D3F8EC0097E72A4B98
:10EB88009100D3F890302820D2E7002A14BF02223F
:10EB98000122254B83F8A52062E7234B1146D3F8C1
:10EBA80090302520C4E7204B9100D3F890302A20DC
:10EBB800BEE7910D89050029DED11B4B9100D3F8E2
:10EBC80090302920B4E7184B1146D3F8903027200D
:10EBD800AEE7154B1146D3F890302620A8E7910DE3
:10EBE80089050029C8D1104B1146D3F890302C2044
:10EBF8009EE70D4B1146D3F890302E2098E70A4B2C
:10EC08001146D3F890302F2092E7074B1146D3F8DE
:10EC1800903033208CE7044B1146D3F890303420E1
:10EC280086E700BF04000020600F0020007102008A
:10EC380000127A0000EE85FF014BD3F89030184798
:10EC4800600F0020034B10B5D3F894300C4698475A
:10EC5800206010BD600F00200022014B5A607047F1
:10EC68000400002070B5494E494CF5686B6803F5FF
:10EC78009C72226203F5AA72E26103F55372A261E3
:10EC880003F55A72626103F56172226103F56872D5
:10EC980003F57670E26003F56F7203F57D73236008
:10ECA8002B68A260DB68606098472B68A069DB6806
:10ECB80098472B686069DB6898472B682069DB6890
:10ECC80098472B68E068DB6898472B68A068DB6882
:10ECD80098472B6860685B6998472B68A0695B69EF
:10ECE80098472B6860695B6998472B6820695B695E
:10ECF80098472B68E0685B6998472B68A0685B6950
:10ED080098472B68206A1B6998472B68E0691B693C
:10ED180098472B6820681B6998476B681D4A3169BA
:10ED280003F537734B60116001211B4B82F8A51066
:10ED380058695974C2F8A800184AC0F80422184A39
:10ED48001A62184ADA61184A9A61184A5A62184AC5
:10ED58009A63184A5A63184A9A62184ADA62184A31
:10ED68009A64184A5A64184A5A65184A1A65184A19
:10ED78001A6693F8D020002A08BF0A4683F8D020E4
:10ED8800144A9A65144ADA6570BD00BF8C4D0208B2
:10ED9800142A0020600F002004000020A9EF0008BA
:10EDA8005DF00008B9F00008BBF00008BFF00008EB
:10EDB800E7FA0008D1FA000849EF000885EF0008D3
:10EDC80041EC00084DEC00083DF00008E5ED0008B6
:10EDD80061EC00086DEC0008DDEE00080228F8B5CB
:10EDE80014464FD006D898B101283AD0354BD3F8FD
:10EDF800E000F8BD032856D0FF28F7D1314CE36F67
:10EE0800D3F8043298476369D3F80432984716E078
:10EE1800136833F00302ECD113F0010F2A4D2B4E87
:10EE28000FD0F3681B681B6968699847246814F059
:10EE380002040ED0F3681B681B69A8699847002074
:10EE4800F8BDF76868693B68DB6898473B689B6969
:10EE5800EAE7F668A8693368DB68984733689B690E
:10EE6800EBE71468184D194B24B1DB681B681B6964
:10EE78002869E3E7DE6828693368DB689847336800
:10EE88009B69F5E71468104D104B24B1DB681B68CB
:10EE98001B69A868D2E7DE68A8683368DB6898470A
:10EEA80033689B69F5E70A4B0120D3F8A0309847EF
:10EEB800034620B9034AD2F8F0002360F8BD0020C9
:10EEC800FBE700BF04000020142A00208C4D020834
:10EED800600F002070B5184E184CF56860682B68F4
:10EEE8009B6998472B68A0699B6898472B6860695D
:10EEF8009B6898472B6820699B6898472B68E0684F
:10EF08009B6898472B68A0689B6898472B68206A7D
:10EF18009B6898472B68E0699B6898472B6820682E
:10EF28009B6898472B6860689B6898473369BDE879
:10EF38007040DB69184700BF8C4D0208142A002076
:10EF480070B50C4C0E46637C834202D8D4F8E800B6
:10EF580070BD094D202095F8A510D5F8903041F0E6
:10EF680004019847D5F89030314637209847D4F8AF
:10EF7800D40070BD04000020600F002038B5074B96
:10EF88000C460546D3F8942093F8A40090472368CC
:10EF9800C11821602846BDE83840D1E7600F00203D
:10EFA80038B5204C204AD4F8A830D26819782546BC
:10EFB8001E4B126841B99269586890470122D4F8EB
:10EFC800A8301A70012038BD194C5269586890470A
:10EFD80094F86820012A1ED0032A20D0012A4FF075
:10EFE8000F0319D04FF4A02143F0884343F0401396
:10EFF800D5F89020194304209047D5F89030042183
:10F00800102098470022D5F8A8301A70E36FD3F87B
:10F0180004329847D6E70B234FF42031E4E70D2359
:10F02800E0E700BF600F00208C4D0208142A002082
:10F038000400002010B5064CD4F888309847D4F85E
:10F04800A8301B7813B1BDE81040A9E710BD00BF78
:10F05800600F002070B5124B0C465A7C1E46824247
:10F0680002D8D3F8E80070BD0E4D2020D5F89030B6
:10F0780095F8A510984784EAE4710B4BA1EBE4716D
:10F088009942D5F8902004DD084911EA240438BFD4
:10F098001C46210224209047D6F8D40070BD00BF3A
:10F0A80004000020600F002000127A0000EE85FFA7
:10F0B800D0E74942CEE70021CCE7F8B51D46BB4B67
:10F0C8005C7C1E468C4203D8D3F8E8402046F8BD45
:10F0D8006F2AD3F8D44000F0088300F29280122AF5
:10F0E80000F01A8243D8052A00F0A4811DD8022A0C
:10F0F80000F0528109D8002A00F02A81012A00F084
:10F108003981D6F8E0000443E0E7032A00F069817A
:10F11800042AF6D1002840F07681A54B2420D3F8A4
:10F128009430984700122860D0E70F2A00F0B58184
:10F138000DD8082A00F099810E2AE2D1002840F063
:10F14800A0819B4B93F8A5305B002B60BEE7102A8B
:10F1580000F0B581112AD4D1002840F0CB81944B1E
:10F168002920D3F89430984780102860AEE7182AF1
:10F1780000F03E8221D8152A00F005820ED8132A05
:10F1880000F0DC81142ABCD1002840F0F281884BC1
:10F198002620D3F894309847286097E7162A00F07D
:10F1A8000B82172AADD1002840F01882804B2E2000
:10F1B800D3F894309847286088E71B2A00F04C82DF
:10F1C8000ED8192A00F026821A2A9AD1002840F06F
:10F1D8003382774B3320D3F894309847286075E70B
:10F1E8006D2A00F0558200F265826C2A89D10028C8
:10F1F80040F044826E4B6020D3F8943098472860E2
:10F2080064E77D2A00F05C834CD8752A00F0E5821B
:10F2180024D8722A00F0A88210D8702A00F08182BF
:10F22800712A7FF46EAF002840F08D82604B062073
:10F23800D3F894309847C0B2286047E7732A00F0A3
:10F24800B082742A7FF45DAF002840F0BC82584B2E
:10F25800D3F8A830D3F870312B6037E7782A00F05C
:10F2680001830FD8762A00F0D782772A7FF449AF36
:10F27800002840F0ED824E4B5E20D3F8943098473A
:10F28800286023E7792A00F0FF827C2A7FF439AFCF
:10F29800002840F00B83464B5C20D3F89430984705
:10F2A800286013E7882A00F074832AD8842A00F09B
:10F2B8004A8316D87E2A00F01783812A7FF421AF6B
:10F2C80001287FF403AF2B68394F002B00F02F8300
:10F2D800D7F8A030984710B9D6F8F0301C4328600A
:10F2E800F4E6852A00F03A83862A7FF40AAF0028DC
:10F2F80040F044832E4BD3F8A830D3F84C312B6020
:10F30800E4E6C82A00F097830FD8892A00F05E83C4
:10F318008A2A7FF4F6AE002840F07883244BD3F88D
:10F32800A83093F892312B60D0E6D42A00F09F835E
:10F33800D62A00F0AF83D12A7FF4E3AE00287FF409
:10F34800C5AE1B4B5020D3F8943098472860BDE6D3
:10F3580030B9174B3720D3F8943098472860B5E672
:10F3680001287FF4B3AE124B2968D3F890303720C8
:10F378009847ABE630B90E4B2120D3F89430984724
:10F388002860A3E601287FF4A1AE094B2968D3F8C9
:10F3980090302120984799E660B9054B2420D3F88E
:10F3A800943098470012286090E600BF04000020BF
:10F3B800600F002001287FF489AEA44B2968D3F898
:10F3C800902081EAE170A24BA0EBE170984204DD45
:10F3D800A04833EA210128BF0146090224209047AA
:10F3E80074E630B9994B2220D3F8943098472860B6
:10F3F8006CE601287FF46AAE944B2968D3F8903004
:10F408002220984762E601287FF460AE8F4B296876
:10F41800D3F8902081EAE1708D4BA0EBE17098421F
:10F4280004DD8C4833EA210128BF01460902242063
:10F4380090474BE638B9854B2820D3F89430984745
:10F448008010286042E601287FF440AE29688A0DC2
:10F4580092051AB1D3F8EC00044337E67B4B8900D8
:10F46800D3F890302820984730E600287FF42EAE55
:10F47800764B0F20D3F89430984700F001002860AD
:10F4880024E601287FF422AE2B68002B0CBF012252
:10F4980002226E4B83F8A52018E630B96B4B252065
:10F4A800D3F894309847286010E601287FF40EAE10
:10F4B800664B2968D3F890302520984706E638B976
:10F4C800624B2A20D3F89430984780102860FDE5D5
:10F4D80001287FF4FBAD29688B0D9B051BB1D6F87D
:10F4E800EC000443F2E5594B8900D3F890302A2008
:10F4F8009847EBE501287FF4E9AD29688B0D9B055A
:10F508001BB1D6F8EC000443E0E5504B8900D3F872
:10F51800903029209847D9E530B94C4B2720D3F8AB
:10F52800943098472860D1E501287FF4CFAD474B48
:10F538002968D3F8903027209847C7E538B9434B56
:10F548002B20D3F89430984780102860BEE5012816
:10F558007FF4BCAD29688B0D9B051BB1D6F8EC0078
:10F568000443B3E5394B8900D3F890302B209847F2
:10F57800ACE501287FF4AAAD344B2968D3F8903064
:10F5880026209847A2E530B9304B2C20D3F8943088
:10F59800984728609AE501287FF498AD29688B0D73
:10F5A8009B051BB1D6F8EC0004438FE5274B2C20B4
:10F5B800D3F89030984789E530B9244B2D20D3F8FB
:10F5C80094309847286081E501287FF47FAD1F4B70
:10F5D8002968D3F890302D20984777E501287FF4E3
:10F5E80075AD1A4B2968D3F890302E2098476DE5F1
:10F5F80030B9164B2F20D3F894309847286065E52A
:10F6080001287FF463AD114B2968D3F890302F207F
:10F6180098475BE530B90D4B3020D3F894309847C4
:10F62800286053E501287FF451AD084B2968D3F8C9
:10F6380090303020984749E501287FF447AD034BC7
:10F648002968D3F89030332098473FE5600F0020B1
:10F6580000127A0000EE85FF30B9A94B3420D3F8A8
:10F6680094309847286031E501287FF42FADA44BEA
:10F678002968D3F890303420984727E501287FF48B
:10F6880025AD9F4B2968D3F89030602098471DE539
:10F6980030B99B4B6120D3F894309847286015E522
:10F6A80001287FF413AD964B2968D3F89030612078
:10F6B80098470BE538B9924B1C20D3F894309847FB
:10F6C8000014286002E501287FF400AD8C4E1C2050
:10F6D800D6F8943098472968C0F3080040EA0141F9
:10F6E800D6F890301C209847F0E438B9844B1C2099
:10F6F800D3F894309847C0B22860E7E401287FF433
:10F70800E5AC7F4E1C20D6F8943098472B6800F45F
:10F718007F01C3F30803D6F8902019431C209047B3
:10F72800D4E430B9764B5920D3F894309847286000
:10F73800CCE401287FF4CAAC714B2968D3F8903027
:10F7480059209847C2E401287FF4C0AC6C4E0620CB
:10F75800D6F894309847297820F0FF000143D6F86E
:10F76800903006209847B1E440B9654B0620D3F89D
:10F7780094309847C0F307202860A7E401287FF455
:10F78800A5AC5F4E0620D6F8943098472B6820F435
:10F798007F411B029BB2D6F8902019430620904760
:10F7A80094E430B9564BD3F8A830D3F86C312B60B9
:10F7B8008CE401287FF48AAC514B2968D3F8903047
:10F7C8005A20984782E401287FF480AC4C4B296882
:10F7D800D3F890305B20984778E440B9484BD3F889
:10F7E800A830D3F87031C3F30E032B606EE4012800
:10F7F8007FF46CAC424A2968D2F8A830C1F30E01F4
:10F80800D3F87031D2F8902023F4FF4323F07F031C
:10F8180019435B20904759E430B9394BD3F8A830E5
:10F8280093F872312B6051E401287FF44FAC344ACD
:10F838005B20D2F8A830D2F89020D3F870112B684A
:10F8480021F47F011B0403F47F03194390473DE42F
:10F8580001287FF43BAC2A4B2968D3F890305E200E
:10F86800984733E430B9264B1820D3F8943098479A
:10F8780028602BE401287FF429AC214B2968D3F8B0
:10F8880090301820984721E430B91D4B1920D3F83F
:10F8980094309847286019E401287FF417AC184B76
:10F8A8002968D3F89030192098470FE401287FF48D
:10F8B8000DAC134B2968D3F890305C20984705E4C9
:10F8C80038B90F4B5F20D3F8943098472860FFF77A
:10F8D800FDBB01287FF4FAAB094B2968D3F89030B7
:10F8E8005F209847FFF7F2BB60B9054B0620D3F8B5
:10F8F80094309847C0F307402860FFF7E7BB00BF84
:10F90800600F002001287FF4E1AB6D4E0620D6F889
:10F91800943098472B6820F47F011B0403F47F037D
:10F92800D6F89020194306209047FFF7CFBBD7F8A9
:10F93800943007209847D7F8903020F480010720AA
:10F948009847FFF7C3BB00287FF4C0AB5C4B65202A
:10F95800D3F8943098472860FFF7B8BB00287FF4A5
:10F96800B5AB574B0720D3F894309847C0F3815074
:10F97800431E584258412860FFF7A8BB01287FF46E
:10F98800A5AB4F4B2968D3F8903052209847FFF722
:10F998009DBB38B94A4BD3F8A83093F890312B6007
:10F9A800FFF794BB01287FF491AB454A2968D2F848
:10F9B800A83001F00F01D3F89031D2F8902023F04D
:10F9C800FF03194363209047FFF780BB48B93C4BBE
:10F9D800D3F8A830D3F89031C3F303232B60FFF793
:10F9E80075BB01287FF472AB354A6320D2F8A83082
:10F9F800D2F89020D3F890112B6821F470611B0283
:10FA080003F4706319439047FFF760BB01287FF444
:10FA18005DAB2B4A6320D2F8A830D2F89020D3F8F7
:10FA280090112B6821F47F011B0403F47F03194311
:10FA38009047FFF74BBB40B9214B0620D3F89430D1
:10FA48009847C0B22860FFF741BB01287FF43EAB5E
:10FA58001B4E0620D6F894309847297820F0FF00EE
:10FA68000143D6F8903006209847FFF72FBB30B9EE
:10FA7800134BD3F8A830DB692B60FFF727BB0128AD
:10FA88007FF424AB0E4B2968D3F890305320984765
:10FA9800FFF71CBB38B90A4B1520D3F894309847A8
:10FAA8002860FFF713BB01287FF410AB2A68044BCA
:10FAB8000449D3F89030514315209847FFF706BB07
:10FAC800600F00200071020007B502AB43F8042D57
:10FAD80002460120FFF7F1FA03B05DF804FB134674
:10FAE80002460020FFF7E9BA014BD3F890301847D7
:10FAF800600F0020034B10B5D3F894300C4698479C
:10FB0800206010BD600F00200022014B5A60704732
:10FB18000400002070B5494E494CF5686B6803F540
:10FB28009C72226203F5AA72E26103F55372A26124
:10FB380003F55A72626103F56172226103F5687216
:10FB480003F57670E26003F56F7203F57D73236049
:10FB58002B68A260DB68606098472B68A069DB6847
:10FB680098472B686069DB6898472B682069DB68D1
:10FB780098472B68E068DB6898472B68A068DB68C3
:10FB880098472B6860685B6998472B68A0695B6930
:10FB980098472B6860695B6998472B6820695B699F
:10FBA80098472B68E0685B6998472B68A0685B6991
:10FBB80098472B68206A1B6998472B68E0691B697E
:10FBC80098472B6820681B6998476B681D4A3169FC
:10FBD80003F537734B60116001211B4B82F8A510A8
:10FBE80058695974C2F8A800184AC0F80422184A7B
:10FBF8001A62184ADA61184A9A61184A5A62184A07
:10FC08009A63184A5A63184A9A62184ADA62184A72
:10FC18009A64184A5A64184A5A65184A1A65184A5A
:10FC28001A6693F8D020002A08BF0A4683F8D02025
:10FC3800144A9A65144ADA6570BD00BF8C4D0208F3
:10FC4800442A0020600F00200400002059FE00080C
:10FC58000DFF000869FF00086BFF00086FFF000830
:10FC68009709010881090108F9FD000835FE000817
:10FC7800F1FA0008FDFA0008EDFE000895FC0008FE
:10FC880011FB00081DFB00088DFD00080228F8B5CF
:10FC980014464FD006D898B101283AD0354BD3F83E
:10FCA800E000F8BD032856D0FF28F7D1314CE36FA8
:10FCB800D3F8043298476369D3F80432984716E0BA
:10FCC800136833F00302ECD113F0010F2A4D2B4EC9
:10FCD8000FD0F3681B681B6968699847246814F09B
:10FCE80002040ED0F3681B681B69A86998470020B6
:10FCF800F8BDF76868693B68DB6898473B689B69AB
:10FD0800EAE7F668A8693368DB68984733689B694F
:10FD1800EBE71468184D194B24B1DB681B681B69A5
:10FD28002869E3E7DE6828693368DB689847336841
:10FD38009B69F5E71468104D104B24B1DB681B680C
:10FD48001B69A868D2E7DE68A8683368DB6898474B
:10FD580033689B69F5E70A4B0120D3F8A030984730
:10FD6800034620B9034AD2F8F0002360F8BD00200A
:10FD7800FBE700BF04000020442A00208C4D020845
:10FD8800600F002070B5184E184CF56860682B6835
:10FD98009B6998472B68A0699B6898472B6860699E
:10FDA8009B6898472B6820699B6898472B68E06890
:10FDB8009B6898472B68A0689B6898472B68206ABF
:10FDC8009B6898472B68E0699B6898472B68206870
:10FDD8009B6898472B6860689B6898473369BDE8BB
:10FDE8007040DB69184700BF8C4D0208442A002088
:10FDF80070B50C4C0E46637C834202D8D4F8E800F8
:10FE080070BD094D202095F8A510D5F8903041F027
:10FE180004019847D5F89030314637209847D4F8F0
:10FE2800D40070BD04000020600F002038B5074BD7
:10FE38000C460546D3F8942093F8A400904723680D
:10FE4800C11821602846BDE83840D1E7600F00207E
:10FE580038B5204C204AD4F8A830D26819782546FD
:10FE68001E4B126841B99269586890470122D4F82C
:10FE7800A8301A70012038BD194C5269586890474B
:10FE880094F86820012A1ED0032A20D0012A4FF0B6
:10FE98000F0319D04FF4A02143F0884343F04013D7
:10FEA800D5F89020194304209047D5F890300421C4
:10FEB800102098470022D5F8A8301A70E36FD3F8BD
:10FEC80004329847D6E70B234FF42031E4E70D239B
:10FED800E0E700BF600F00208C4D0208442A002094
:10FEE8000400002010B5064CD4F888309847D4F8A0
:10FEF800A8301B7813B1BDE81040A9E710BD00BFBA
:10FF0800600F002070B5124B0C465A7C1E46824288
:10FF180002D8D3F8E80070BD0E4D2020D5F89030F7
:10FF280095F8A510984784EAE4710B4BA1EBE471AE
:10FF38009942D5F8902004DD084911EA240438BF15
:10FF48001C46210224209047D6F8D40070BD00BF7B
:10FF580004000020600F002000127A0000EE85FFE8
:10FF6800D0E74942CEE70021CCE7F8B51D46BB4BA8
:10FF78005C7C1E468C4203D8D3F8E8402046F8BD86
:10FF88006F2AD3F8D44000F0088300F29280122A36
:10FF980000F01A8243D8052A00F0A4811DD8022A4D
:10FFA80000F0528109D8002A00F02A81012A00F0C5
:10FFB8003981D6F8E0000443E0E7032A00F06981BC
:10FFC800042AF6D1002840F07681A54B2420D3F8E6
:10FFD8009430984700122860D0E70F2A00F0B581C6
:10FFE8000DD8082A00F099810E2AE2D1002840F0A5
:08FFF800A0819B4B93F8A5309A
:020000040801F1
:100000005B002B60BEE7102A00F0B581112AD4D125
:10001000002840F0CB81944B2920D3F894309847A6
:1000200080102860AEE7182A00F03E8221D8152AF9
:1000300000F005820ED8132A00F0DC81142ABCD10E
:10004000002840F0F281884B2620D3F8943098475E
:10005000286097E7162A00F00B82172AADD10028F6
:1000600040F01882804B2E20D3F8943098472860B7
:1000700088E71B2A00F04C820ED8192A00F026824D
:100080001A2A9AD1002840F03382774B3320D3F8D4
:1000900094309847286075E76D2A00F0558200F289
:1000A00065826C2A89D1002840F044826E4B602022
:1000B000D3F894309847286064E77D2A00F05C8389
:1000C0004CD8752A00F0E58224D8722A00F0A88264
:1000D00010D8702A00F08182712A7FF46EAF002858
:1000E00040F08D82604B0620D3F894309847C0B220
:1000F000286047E7732A00F0B082742A7FF45DAF6E
:10010000002840F0BC82584BD3F8A830D3F87031A7
:100110002B6037E7782A00F001830FD8762A00F0A9
:10012000D782772A7FF449AF002840F0ED824E4B0A
:100130005E20D3F894309847286023E7792A00F0AE
:10014000FF827C2A7FF439AF002840F00B83464BB6
:100150005C20D3F894309847286013E7882A00F091
:1001600074832AD8842A00F04A8316D87E2A00F0A5
:100170001783812A7FF421AF01287FF403AF2B6816
:10018000394F002B00F02F83D7F8A030984710B9D3
:10019000D6F8F0301C432860F4E6852A00F03A8354
:1001A000862A7FF40AAF002840F044832E4BD3F810
:1001B000A830D3F84C312B60E4E6C82A00F09783CE
:1001C0000FD8892A00F05E838A2A7FF4F6AE0028D1
:1001D00040F07883244BD3F8A83093F892312B6009
:1001E000D0E6D42A00F09F83D62A00F0AF83D12A2C
:1001F0007FF4E3AE00287FF4C5AE1B4B5020D3F84C
:10020000943098472860BDE630B9174B3720D3F8B3
:10021000943098472860B5E601287FF4B3AE124BBE
:100220002968D3F8903037209847ABE630B90E4BA9
:100230002120D3F8943098472860A3E601287FF462
:10024000A1AE094B2968D3F890302120984799E650
:1002500060B9054B2420D3F89430984700122860E9
:1002600090E600BF04000020600F002001287FF40A
:1002700089AEA44B2968D3F8902081EAE170A24BA3
:10028000A0EBE170984204DDA04833EA210128BFC9
:10029000014609022420904774E630B9994B222088
:1002A000D3F89430984728606CE601287FF46AAE52
:1002B000944B2968D3F890302220984762E60128B1
:1002C0007FF460AE8F4B2968D3F8902081EAE1700B
:1002D0008D4BA0EBE170984204DD8C4833EA21019C
:1002E00028BF01460902242090474BE638B9854BC8
:1002F0002820D3F8943098478010286042E60128DF
:100300007FF440AE29688A0D92051AB1D3F8EC004B
:10031000044337E67B4B8900D3F890302820984778
:1003200030E600287FF42EAE764B0F20D3F89430C1
:10033000984700F00100286024E601287FF422AEEF
:100340002B68002B0CBF012202226E4B83F8A520E4
:1003500018E630B96B4B2520D3F8943098472860C5
:1003600010E601287FF40EAE664B2968D3F8903072
:100370002520984706E638B9624B2A20D3F89430F6
:10038000984780102860FDE501287FF4FBAD2968BF
:100390008B0D9B051BB1D6F8EC000443F2E5594BDD
:1003A0008900D3F890302A209847EBE501287FF4A4
:1003B000E9AD29688B0D9B051BB1D6F8EC00044311
:1003C000E0E5504B8900D3F8903029209847D9E5D3
:1003D00030B94C4B2720D3F8943098472860D1E5AA
:1003E00001287FF4CFAD474B2968D3F89030272000
:1003F0009847C7E538B9434B2B20D3F8943098473A
:1004000080102860BEE501287FF4BCAD29688B0D03
:100410009B051BB1D6F8EC000443B3E5394B8900CA
:10042000D3F890302B209847ACE501287FF4AAAD93
:10043000344B2968D3F8903026209847A2E530B98C
:10044000304B2C20D3F89430984728609AE5012847
:100450007FF498AD29688B0D9B051BB1D6F8EC0095
:1004600004438FE5274B2C20D3F89030984789E53B
:1004700030B9244B2D20D3F894309847286081E57B
:1004800001287FF47FAD1F4B2968D3F890302D20D1
:10049000984777E501287FF475AD1A4B2968D3F8A2
:1004A00090302E2098476DE530B9164B2F20D3F8A9
:1004B00094309847286065E501287FF463AD114BBF
:1004C0002968D3F890302F2098475BE530B90D4B61
:1004D0003020D3F894309847286053E501287FF402
:1004E00051AD084B2968D3F890303020984749E542
:1004F00001287FF447AD034B2968D3F890303320AF
:1005000098473FE5600F002000127A0000EE85FF5B
:1005100030B9A94B3420D3F894309847286031E59E
:1005200001287FF42FADA44B2968D3F890303420F4
:10053000984727E501287FF425AD9F4B2968D3F81C
:100540009030602098471DE530B99B4B6120D3F86F
:1005500094309847286015E501287FF413AD964B39
:100560002968D3F89030612098470BE538B9924B51
:100570001C20D3F8943098470014286002E5012825
:100580007FF400AD8C4E1C20D6F894309847296833
:10059000C0F3080040EA0141D6F890301C2098478B
:1005A000F0E438B9844B1C20D3F894309847C0B29B
:1005B0002860E7E401287FF4E5AC7F4E1C20D6F8E4
:1005C000943098472B6800F47F01C3F30803D6F8F2
:1005D000902019431C209047D4E430B9764B592021
:1005E000D3F8943098472860CCE401287FF4CAAC53
:1005F000714B2968D3F8903059209847C2E40128FC
:100600007FF4C0AC6C4E0620D6F894309847297819
:1006100020F0FF000143D6F8903006209847B1E45F
:1006200040B9654B0620D3F894309847C0F30720B3
:100630002860A7E401287FF4A5AC5F4E0620D6F819
:10064000943098472B6820F47F411B029BB2D6F868
:10065000902019430620904794E430B9564BD3F8C4
:10066000A830D3F86C312B608CE401287FF48AAC7D
:10067000514B2968D3F890305A20984782E40128DA
:100680007FF480AC4C4B2968D3F890305B209847BE
:1006900078E440B9484BD3F8A830D3F87031C3F3AD
:1006A0000E032B606EE401287FF46CAC424A29688B
:1006B000D2F8A830C1F30E01D3F87031D2F89020EF
:1006C00023F4FF4323F07F0319435B20904759E451
:1006D00030B9394BD3F8A83093F872312B6051E41C
:1006E00001287FF44FAC344A5B20D2F8A830D2F80E
:1006F0009020D3F870112B6821F47F011B0403F4C0
:100700007F03194390473DE401287FF43BAC2A4B1B
:100710002968D3F890305E20984733E430B9264BEF
:100720001820D3F89430984728602BE401287FF4F0
:1007300029AC214B2968D3F890301820984721E440
:1007400030B91D4B1920D3F894309847286019E42C
:1007500001287FF417AC184B2968D3F89030192082
:1007600098470FE401287FF40DAC134B2968D3F8A8
:1007700090305C20984705E438B90F4B5F20D3F8E0
:10078000943098472860FFF7FDBB01287FF4FAAB4F
:10079000094B2968D3F890305F209847FFF7F2BBE8
:1007A00060B9054B0620D3F894309847C0F3074052
:1007B0002860FFF7E7BB00BF600F002001287FF42F
:1007C000E1AB6D4E0620D6F8943098472B6820F4A4
:1007D0007F011B0403F47F03D6F890201943062001
:1007E0009047FFF7CFBBD7F8943007209847D7F84A
:1007F000903020F4800107209847FFF7C3BB002802
:100800007FF4C0AB5C4B6520D3F8943098472860E8
:10081000FFF7B8BB00287FF4B5AB574B0720D3F8E0
:1008200094309847C0F38150431E58425841286085
:10083000FFF7A8BB01287FF4A5AB4F4B2968D3F87D
:10084000903052209847FFF79DBB38B94A4BD3F8F8
:10085000A83093F890312B60FFF794BB01287FF408
:1008600091AB454A2968D2F8A83001F00F01D3F8BE
:100870009031D2F8902023F0FF0319436320904772
:10088000FFF780BB48B93C4BD3F8A830D3F8903180
:10089000C3F303232B60FFF775BB01287FF472AB12
:1008A000354A6320D2F8A830D2F89020D3F89011BE
:1008B0002B6821F470611B0203F4706319439047A5
:1008C000FFF760BB01287FF45DAB2B4A6320D2F8B1
:1008D000A830D2F89020D3F890112B6821F47F0132
:1008E0001B0403F47F0319439047FFF74BBB40B948
:1008F000214B0620D3F894309847C0B22860FFF708
:1009000041BB01287FF43EAB1B4E0620D6F8943045
:100910009847297820F0FF000143D6F89030062050
:100920009847FFF72FBB30B9134BD3F8A830DB69DA
:100930002B60FFF727BB01287FF424AB0E4B2968FF
:10094000D3F8903053209847FFF71CBB38B90A4BB7
:100950001520D3F8943098472860FFF713BB01287F
:100960007FF410AB2A68044B0449D3F8903051430C
:1009700015209847FFF706BB600F002000710200AA
:1009800007B502AB43F8042D02460120FFF7F1FA48
:1009900003B05DF804FB134602460020FFF7E9BAF6
:1009A00000207047012070470022014B5A607047B9
:1009B0000400002010B5054C10B1D4F8E80010BDBB
:1009C00008460EF0ADFED4F8D40010BD040000209F
:1009D00010B5054C10B1D4F8E80010BD08460EF073
:1009E00085FED4F8D40010BD040000200021EFE7FC
:1009F0004942EDE7ECE710B50C460BF065FE2060D0
:100A000010BD0BF08DBE70B51E460546024B29B1D8
:100A1000D3F8E840204670BD04000020D3F8D4404D
:100A2000FF2A01F2548001A151F822F0150A0108B1
:100A3000CF1A0108CF1A0108CF1A01082D0E01089C
:100A4000CF1A0108CF1A0108CF1A0108CF1A0108DE
:100A5000CF1A0108CF1A0108490E0108530E0108E8
:100A6000CF1A01085D0E0108CF1A0108CF1A01083C
:100A7000CF1A0108CF1A0108CF1A0108CF1A0108AE
:100A8000CF1A0108CF1A0108CF1A0108CF1A01089E
:100A9000CF1A0108CF1A0108CF1A0108CF1A01088E
:100AA000CF1A0108CF1A0108CF1A0108CF1A01087E
:100AB000CF1A0108CF1A0108CF1A0108CF1A01086E
:100AC000CF1A0108CF1A0108CF1A0108CF1A01085E
:100AD000CF1A0108CF1A0108CF1A0108CF1A01084E
:100AE000CF1A0108CF1A0108CF1A0108CF1A01083E
:100AF000CF1A0108670E0108890E0108CF1A0108F4
:100B0000AB0E0108CD0E0108CF1A0108CF1A01085B
:100B1000CF1A0108CF1A0108CF1A0108CF1A01080D
:100B2000CF1A0108CF1A0108CF1A0108CF1A0108FD
:100B3000CF1A0108CF1A0108CF1A0108CF1A0108ED
:100B4000CF1A0108CF1A0108CF1A0108CF1A0108DD
:100B5000CF1A0108CF1A0108CF1A0108CF1A0108CD
:100B6000CF1A0108CF1A0108CF1A0108CF1A0108BD
:100B7000CF1A0108CF1A0108CF1A0108CF1A0108AD
:100B8000CF1A0108CF1A0108CF1A0108CF1A01089D
:100B9000CF1A0108CF1A0108CF1A0108CF1A01088D
:100BA000CF1A0108CF1A0108CF1A0108CF1A01087D
:100BB000CF1A0108CF1A0108CF1A0108EF0E010859
:100BC000090F0108230F01083D0F0108570F010805
:100BD000710F01088B0F0108A50F0108BF0F010855
:100BE000D90F0108F30F01080D10010827100108A3
:100BF000411001085B100108751001088F100108F1
:100C0000A3100108B7100108CF1A0108CB10010882
:100C1000DF100108F3100108071101081B1101087A
:100C200037110108531101086F11010881110108E2
:100C3000CF1A0108CF1A0108CF1A01089311010831
:100C4000A3110108B3110108C7110108DB11010844
:100C5000CF1A0108CF1A0108CF1A0108EB110108B9
:100C6000FB1101080B120108CF1A0108CF1A010865
:100C7000CF1A0108CF1A0108CF1A0108CF1A0108AC
:100C8000CF1A010821120108371201084D1201087C
:100C900063120108CF1A0108CF1A0108CF1A010800
:100CA000CF1A0108CF1A0108CF1A010879120108DA
:100CB0008F120108A5120108BB120108D112010808
:100CC000CF1A0108CF1A0108CF1A0108CF1A01085C
:100CD000CF1A0108E7120108FD12010823130108C9
:100CE000491301085B130108791301088F130108E8
:100CF0009F130108B5130108C5130108E11301088A
:100D0000FB130108151401082F14010849140108E8
:100D1000631401087D14010897140108CF1A010813
:100D2000B1140108CD140108E914010803150108E4
:100D30001F15010839150108531501086D15010823
:100D400087150108A1150108BF150108DD15010867
:100D5000FB15010819160108371601085516010878
:100D60007316010891160108AF160108CD16010887
:100D7000EB16010809170108271701084517010894
:100D800063170108811701089F170108BD170108A3
:100D9000DB170108F7170108CF1A0108CF1A01085D
:100DA000CF1A0108CF1A0108CF1A0108CF1A01087B
:100DB000CF1A0108CF1A0108CF1A0108CF1A01086B
:100DC000CF1A010813180108311801084F1801083B
:100DD0006D1801088B180108A9180108C718010827
:100DE000E5180108031901081F1901083B1901083A
:100DF00057190108731901088F190108AB19010867
:100E0000C7190108E3190108FD190108171A01089B
:100E1000311A01084B1A0108671A0108831A0108E0
:100E20009F1A0108AF1A0108BF1A010820B96020F3
:100E30000BF04AFC3060EDE501287FF4EBAD316842
:100E400060200BF06DFCE5E500287FF4E3AD306039
:100E5000E0E500287FF4DEAD3060DBE500287FF4BC
:100E6000D9AD3060D6E530B9014608200BF0B7FCAB
:100E700000B23060CEE501287FF4CCAD328800218D
:100E800008200BF0DDFCC5E530B9014609200BF068
:100E9000A6FC00B23060BDE501287FF4BBAD32880E
:100EA000002109200BF0CCFCB4E530B90121082069
:100EB0000BF095FC00B23060ACE501287FF4AAADE0
:100EC0000146328808200BF0BBFCA3E530B90121B4
:100ED00009200BF084FC00B230609BE501287FF410
:100EE00099AD0146328809200BF0AAFC92E5002852
:100EF0007FF490AD012103200BF012FC2946022063
:100F00000BF06DFC306085E500287FF483AD012196
:100F100003200BF005FC012102200BF060FC306087
:100F200078E500287FF476AD022103200BF0F8FB72
:100F3000294602200BF053FC30606BE500287FF45B
:100F400069AD014603200BF0EBFB294602200BF0B4
:100F500046FC30605EE500287FF45CAD014603206E
:100F60000BF0DEFB012102200BF039FC306051E573
:100F700000287FF44FAD032108460BF0D1FB294632
:100F800002200BF02CFC306044E500287FF442ADD9
:100F9000042103200BF0C4FB294602200BF01FFCA8
:100FA000306037E500287FF435AD042103200BF0D5
:100FB000B7FB012102200BF012FC30602AE500286B
:100FC0007FF428AD052103200BF0AAFB294602205F
:100FD0000BF005FC30601DE500287FF41BAD0521FA
:100FE00003200BF09DFB012102200BF0F8FB306089
:100FF00010E500287FF40EAD062103200BF090FBD6
:10100000294602200BF0EBFB306003E500287FF45B
:1010100001AD072103200BF083FB294602200BF0D2
:10102000DEFB3060F6E400287FF4F4AC07210320F7
:101030000BF076FB012102200BF0D1FB3060E9E4DC
:1010400000287FF4E7AC082103200BF069FB294658
:1010500002200BF0C4FB3060DCE400287FF4DAAC43
:10106000082103200BF05CFB012102200BF0B7FBF1
:101070003060CFE400287FF4CDAC092103200BF0D1
:101080004FFB294602200BF0AAFB3060C2E4002887
:101090007FF4C0AC014612200BF0A1FB00B230601F
:1010A000B8E400287FF4B6AC012112200BF097FBC6
:1010B00000B23060AEE400287FF4ACAC01461320EF
:1010C0000BF08DFB00B23060A4E400287FF4A2ACEA
:1010D000014615200BF083FB00B230609AE4002833
:1010E0007FF498AC012115200BF079FB00B2306041
:1010F00090E400287FF48EAC014616200BF06FFBC5
:1011000000B2306086E400287FF484AC0121162010
:101110000BF065FB00B230607CE400287FF47AAC11
:101120000A2103200BF0FCFA294602200BF057FBA2
:1011300000B230606EE400287FF46CAC0A2103201A
:101140000BF0EEFA012102200BF049FB00B23060F7
:1011500060E400287FF45EAC0B2103200BF0E0FA82
:10116000294602200BF03BFB00B2306052E400281D
:101170007FF450AC014606200BF031FB306049E4AF
:1011800000287FF447AC012106200BF028FB3060DB
:1011900040E400287FF43EAC41200BF095FA30602B
:1011A00038E400287FF436AC42200BF08DFA306032
:1011B00030E400287FF42EAC012146200BF00FFB19
:1011C00000B2306026E400287FF424AC01464620BB
:1011D0000BF005FB00B230601CE400287FF41AAC71
:1011E00047200BF071FA306014E400287FF412AC51
:1011F00021200BF069FA30600CE400287FF40AAC7F
:1012000022200BF061FA306004E400287FF402AC85
:10121000014623200BF0E3FA00B23060FFF7FABB7F
:1012200000287FF4F7AB27200BF04EFA20F07F4028
:101230003060FFF7EFBB00287FF4ECAB28200BF009
:1012400043FA20F07F403060FFF7E4BB00287FF4D2
:10125000E1AB01212A200BF0C2FA00B23060FFF7A7
:10126000D9BB00287FF4D6AB01462A200BF0B7FA91
:1012700000B23060FFF7CEBB00287FF4CBAB014655
:1012800039200BF0ACFA00B23060FFF7C3BB002886
:101290007FF4C0AB012139200BF0A1FA00B230601D
:1012A000FFF7B8BB00287FF4B5AB01463D200BF03B
:1012B00096FA00B23060FFF7ADBB00287FF4AAAB0E
:1012C00001463F200BF08BFA00B23060FFF7A2BB63
:1012D00000287FF49FAB01463A200BF080FA00B261
:1012E0003060FFF797BB00287FF494AB0146532092
:1012F0000BF075FA00B23060FFF78CBB38B90121F2
:1013000064200BF06CFA00B23060FFF783BB012859
:101310007FF480AB0146328864200BF091FAFFF72E
:1013200079BB38B9014664200BF059FA00B230603D
:10133000FFF770BB01287FF46DAB32880021642079
:101340000BF07EFAFFF766BB00287FF463AB6620E4
:101350000BF0BAF93060FFF75DBB28B968200BF0DD
:10136000B3F93060FFF756BB01287FF453AB306808
:101370000EF0D6F9FFF74EBB00287FF44BAB0121EE
:1013800069200BF02CFA00B23060FFF743BB002855
:101390007FF440AB0EF044F93060FFF73BBB002810
:1013A0007FF438AB014669200BF019FA00B23060C7
:1013B000FFF730BB00287FF42DAB0EF0ACF93060A6
:1013C000FFF728BB20B90EF0CBF93060FFF722BB46
:1013D00001287FF41FAB30680EF0BEF9FFF71ABB8F
:1013E00000287FF417AB01466D200BF099F96C20B3
:1013F0000BF06AF93060FFF70DBB00287FF40AABF1
:1014000001216D200BF08CF96C200BF05DF9306040
:10141000FFF700BB00287FF4FDAA02216D200BF02E
:101420007FF96C200BF050F93060FFF7F3BA002819
:101430007FF4F0AA03216D200BF072F96C200BF001
:1014400043F93060FFF7E6BA00287FF4E3AA0421ED
:101450006D200BF065F96C200BF036F93060FFF76A
:10146000D9BA00287FF4D6AA05216D200BF058F9CF
:101470006C200BF029F93060FFF7CCBA00287FF41C
:10148000C9AA06216D200BF04BF96C200BF01CF95A
:101490003060FFF7BFBA00287FF4BCAA07216D2097
:1014A0000BF03EF96C200BF00FF93060FFF7B2BA89
:1014B00020B90EF081F83060FFF7ACBA01287FF454
:1014C000A9AA30680EF06CF8FFF7A4BA20B90EF0A4
:1014D00099F83060FFF79EBA01287FF49BAA306824
:1014E0000EF07DF8FFF796BA00287FF493AA012149
:1014F0006F200BF015F96E200BF0E6F83060FFF767
:1015000089BA20B90EF0FDF83060FFF783BA0128E0
:101510007FF480AA30680EF0E9F8FFF77BBA002864
:101520007FF478AA03216F200BF0FAF86E200BF0FD
:10153000CBF83060FFF76EBA00287FF46BAA042165
:101540006F200BF0EDF86E200BF0BEF83060FFF767
:1015500061BA00287FF45EAA05216F200BF0E0F845
:101560006E200BF0B1F83060FFF754BA00287FF41A
:1015700051AA06216F200BF0D3F86E200BF0A4F8CF
:101580003060FFF747BA00287FF444AA07216F2094
:101590000BF0C6F86E200BF097F83060FFF73ABA00
:1015A00000287FF437AA08216F200BF0B9F82946EC
:1015B0006E200BF014F900B23060FFF72BBA002850
:1015C0007FF428AA08216F200BF0AAF801216E20D1
:1015D0000BF005F900B23060FFF71CBA00287FF469
:1015E00019AA09216F200BF09BF829466E200BF0F9
:1015F000F6F800B23060FFF70DBA00287FF40AAAAF
:101600000A216F200BF08CF829466E200BF0E7F8CA
:1016100000B23060FFF7FEB900287FF4FBA90A2171
:101620006F200BF07DF801216E200BF0D8F800B28E
:101630003060FFF7EFB900287FF4ECA90B216F2091
:101640000BF06EF829466E200BF0C9F800B230603E
:10165000FFF7E0B900287FF4DDA90B216F200BF024
:101660005FF801216E200BF0BAF800B23060FFF78E
:10167000D1B900287FF4CEA90C216F200BF050F8CF
:1016800029466E200BF0ABF800B23060FFF7C2B90C
:1016900000287FF4BFA90C216F200BF041F8012135
:1016A0006E200BF09CF800B23060FFF7B3B9002851
:1016B0007FF4B0A90D216F200BF032F829466E207F
:1016C0000BF08DF800B23060FFF7A4B900287FF46A
:1016D000A1A90D216F200BF023F801216E200BF042
:1016E0007EF800B23060FFF795B900287FF492A928
:1016F0000E216F200BF014F829466E200BF06FF8C6
:1017000000B23060FFF786B900287FF483A90E216C
:101710006F200BF005F801216E200BF060F800B28D
:101720003060FFF777B900287FF474A90F216F208C
:101730000AF0F6FF29466E200BF051F800B2306037
:10174000FFF768B900287FF465A90F216F200AF020
:10175000E7FF01216E200BF042F800B23060FFF786
:1017600059B900287FF456A910216F200AF0D8FF3C
:1017700029466E200BF033F800B23060FFF74AB90B
:1017800000287FF447A911216F200AF0C9FF2946DC
:101790006E200BF024F800B23060FFF73BB9002850
:1017A0007FF438A911216F200AF0BAFF01216E20C1
:1017B0000BF015F800B23060FFF72CB900287FF469
:1017C00029A912216F200AF0ABFF29466E200BF0E9
:1017D00006F800B23060FFF71DB900287FF41AA99F
:1017E00013216F200AF09CFF29466E200AF0F7FFB4
:1017F0003060FFF70FB900287FF40CA913216F2088
:101800000AF08EFF01216E200AF0E9FF3060FFF739
:1018100001B900287FF4FEA8C0216F200AF080FFE4
:1018200029466E200AF0DBFF00B23060FFF7F2B805
:1018300000287FF4EFA8C0216F200AF071FF01217A
:101840006E200AF0CCFF00B23060FFF7E3B800284A
:101850007FF4E0A8C1216F200AF062FF29466E20C4
:101860000AF0BDFF00B23060FFF7D4B800287FF463
:10187000D1A8C1216F200AF053FF01216E200AF088
:10188000AEFF00B23060FFF7C5B800287FF4C2A8F1
:10189000C2216F200AF044FF29466E200AF09FFF04
:1018A00000B23060FFF7B6B800287FF4B3A8C221B9
:1018B0006F200AF035FF01216E200AF090FF00B280
:1018C0003060FFF7A7B800287FF4A4A8C3216F20D9
:1018D0000AF026FF29466E200AF081FF00B2306030
:1018E000FFF798B800287FF495A8C3216F200AF06D
:1018F00017FF01216E200AF072FF00B23060FFF77F
:1019000089B800287FF486A8C4216F200AF008FF58
:1019100029466E200AF063FF3060FFF77BB800288D
:101920007FF478A8C4216F200AF0FAFE01216E200E
:101930000AF055FF3060FFF76DB800287FF46AA801
:10194000C5216F200AF0ECFE29466E200AF047FF01
:101950003060FFF75FB800287FF45CA8C5216F20D6
:101960000AF0DEFE01216E200AF039FF3060FFF739
:1019700051B800287FF44EA8C6216F200AF0D0FE8F
:1019800029466E200AF02BFF3060FFF743B800288D
:101990007FF440A8C6216F200AF0C2FE01216E200C
:1019A0000AF01DFF3060FFF735B800287FF432A839
:1019B000C7216F200AF0B4FE29466E200AF00FFFFF
:1019C0003060FFF727B800287FF424A8C7216F20D4
:1019D0000AF0A6FE01216E200AF001FF3060FFF739
:1019E00019B800287FF416A8C8216F200AF098FEC5
:1019F0006E200AF069FE3060FFF70CB800287FF413
:101A000009A8C9216F200AF08BFE6E200AF05CFE47
:101A10003060FEF7FFBF00287EF4FCAFCA216F20C4
:101A20000AF07EFE6E200AF04FFE3060FEF7F2BF35
:101A300000287EF4EFAFCB216F200AF071FE6E20FC
:101A40000AF042FE3060FEF7E5BF20B9224B1B686A
:101A50003360FEF7DFBF01287EF4DCAF32681E4B37
:101A60001A60FEF7D7BF20B90DF05CFF3060FEF7BB
:101A7000D1BF01287EF4CEAF30880DF04DFFFEF7C8
:101A8000C9BF20B90DF062FF3060FEF7C3BF012867
:101A90007EF4C0AF30780DF04BFFFEF7BBBF0028DF
:101AA0007EF4B8AF0DF058FF3060FEF7B3BF0028EA
:101AB0007EF4B0AF0DF056FF3060FEF7ABBF0028EC
:101AC0007EF4A8AF0DF014FC3060FEF7A3BFD3F88E
:101AD000E0000443FEF79EBF742A002007B502AB66
:101AE00043F8042D02460120FEF78DFF03B05DF898
:101AF00004FB134602460020FEF785BF0F4B9A7881
:101B0000824204BF0E4A92F8D1001A78824206D16E
:101B10000C4BDB681B689B690B4A106818475B78A5
:101B2000834209D1064B93F8D130834204D1054B4F
:101B3000DB681B685B69EFE7704700BF781A00201D
:101B4000040000208C4D0208604D002010B5064BAB
:101B50001878FFF7D3FFBDE81040044B044ADB6858
:101B600010681B689B691847781A00208C4D020882
:101B7000604D002038B5244B244DDC686068236834
:101B8000C8302860DB689847236828685B699847F5
:101B90001F4B20495A6901240A601F49C2F80412E8
:101BA0001E49C2F80C120021117051701C4A5C745D
:101BB0001A621C4A83F8D040DA611B4A9A611B4AB8
:101BC0005A621B4ADA641B4A9A631B4A5A631B4ACD
:101BD0009A621B4ADA621B4A9A641B4A5A641B4A7D
:101BE0005A651B4A1A651B4A5A661B4A1A661B4AE3
:101BF000DA653222DA6040F28A229A600DF0B2FC95
:101C00002046BDE8384079E78C4D0208604D002041
:101C100004000020E04D0020651D0108A509010811
:101C2000D1090108F5090108F1090108ED090108C8
:101C3000611C0108F31A0108DD1A0108B509010841
:101C4000491D0108030A0108F7090108811C010860
:101C5000A1090108FD1A0108A90901084D1B010885
:101C600038B50D46054C10B1D4F8E80038BD0DF07C
:101C700052FD2860D4F8D40038BD00BF0400002015
:101C80007FB5304C05466368C31A002BB8BF5B4272
:101C9000092B07DD6420A36858430DF065FB002382
:101CA0006560A360A36828460133A3600DF032FE8F
:101CB0000DF0B0FB60B10DF0B3FC05460DF02BFD4F
:101CC00006460DF04DFD3146024628460DF024FC37
:101CD0000DF09AFB90B10DF00DFC03280ED8DFE853
:101CE00000F0150F021B0DF034FD00900DF038FDD3
:101CF000019004AB13E90F000DF0A6FB04B070BD1A
:101D00000DF0FFFC00900DF006FDF1E70DF07AFC00
:101D100000900DF085FCEBE7236853B1012BE8D16F
:101D20004FF496736421C8228DE80E004FF4C873F7
:101D300005E014230A201E248DE8190028230393AC
:101D4000D7E700BF742A002010B5054C10B1D4F8B5
:101D5000E80010BD08680DF0EEFCD4F8D40010BD0A
:101D600004000020012070470AF0AEBC0AF0D8BC85
:101D70000AF035BD0AF064BD0020704701207047AD
:101D80000022014B5A6070470400002010B5054C3A
:101D900010B1D4F8E80010BD08460DF03EFFD4F8AD
:101DA000D40010BD0400002010B5054C10B1D4F8CB
:101DB000E80010BD08460DF01DFFD4F8D40010BD9A
:101DC000040000200021EFE74942EDE7ECE710B501
:101DD0000C460AF079FC206010BD0AF0A1BC70B579
:101DE0001E460546024B29B1D3F8E840204670BD97
:101DF00004000020D3F8D440FF2A01F2788101A129
:101E000051F822F0ED1D0108EF300108EF30010814
:101E1000EF30010805220108EF300108EF3001081A
:101E2000EF300108EF300108EF300108EF30010812
:101E3000212201082B220108EF3001083522010878
:101E4000EF300108EF300108EF300108EF300108F2
:101E5000EF300108EF300108EF300108EF300108E2
:101E6000EF300108EF300108EF300108EF300108D2
:101E7000EF300108EF300108EF300108EF300108C2
:101E8000EF300108EF300108EF300108EF300108B2
:101E9000EF300108EF300108EF300108EF300108A2
:101EA000EF300108EF300108EF300108EF30010892
:101EB000EF300108EF300108EF300108EF30010882
:101EC000EF300108EF300108EF3001083F22010830
:101ED00061220108EF30010883220108A5220108D0
:101EE000EF300108EF300108EF300108EF30010852
:101EF000EF300108EF300108EF300108EF30010842
:101F0000EF300108EF300108EF300108EF30010831
:101F1000EF300108EF300108EF300108EF30010821
:101F2000EF300108EF300108EF300108EF30010811
:101F3000EF300108EF300108EF300108EF30010801
:101F4000EF300108EF300108EF300108EF300108F1
:101F5000EF300108EF300108EF300108EF300108E1
:101F6000EF300108EF300108EF300108EF300108D1
:101F7000EF300108EF300108EF300108EF300108C1
:101F8000EF300108EF300108EF300108EF300108B1
:101F9000EF300108C7220108E1220108FB220108F5
:101FA000152301082F230108492301086323010891
:101FB0007D23010897230108B1230108CB230108E1
:101FC000E5230108FF23010819240108332401082F
:101FD0004D240108672401087B2401088F2401088F
:101FE000EF300108A3240108B7240108CB2401081D
:101FF000DF240108F32401080F2501082B2501081F
:102000004725010859250108EF300108EF30010884
:10201000EF3001086B2501087B2501088B2501089D
:102020009F250108B3250108EF300108EF300108B2
:10203000EF300108C3250108D3250108E325010875
:10204000EF300108EF300108EF300108EF300108F0
:10205000EF300108EF300108EF300108F9250108E1
:102060000F260108252601083B26010851260108F4
:1020700081260108B1260108E72601081D2701086D
:1020800053270108872701089D270108B327010866
:10209000C9270108DF270108EF300108EF300108E8
:1020A000EF300108EF300108EF300108F527010893
:1020B0000B28010831280108572801086928010860
:1020C0007B28010891280108A1280108B7280108E8
:1020D000C7280108E7280108012901081B29010870
:1020E000352901084F2901086929010883290108B8
:1020F0009D290108EF300108B7290108D3290108FB
:10210000EF290108092A0108232A01083D2A0108AC
:10211000572A0108712A01088B2A0108A52A0108FB
:10212000C32A0108E12A0108FF2A01081D2B010822
:102130003B2B0108592B0108772B0108952B01082F
:10214000B32B0108D12B0108EF2B01080D2C01083E
:102150002B2C0108492C0108672C0108852C01084B
:10216000A32C0108C12C0108DF2C0108FB2C01085D
:10217000EF300108172D0108472D0108772D0108C0
:10218000AD2D0108E32D0108192E0108EF300108DB
:10219000EF300108EF300108EF3001084F2E010841
:1021A0006D2E01088B2E0108A92E0108C72E0108EB
:1021B000E52E0108032F0108212F01083F2F0108F8
:1021C0005B2F0108772F0108932F0108AF2F01081B
:1021D000CB2F0108E72F0108033001081F30010849
:1021E00039300108533001086D300108EF30010823
:1021F00087300108A3300108BF300108CF30010843
:10220000DF30010820B960200AF05EFA3060EDE5A9
:1022100001287FF4EBAD316860200AF081FAE5E532
:1022200000287FF4E3AD3060E0E500287FF4DEAD08
:102230003060DBE500287FF4D9AD3060D6E530B9F9
:10224000014608200AF0CBFA00B23060CEE5012842
:102250007FF4CCAD3288002108200AF0F1FAC5E500
:1022600030B9014609200AF0BAFA00B23060BDE583
:1022700001287FF4BBAD3288002109200AF0E0FA82
:10228000B4E530B9012108200AF0A9FA00B23060A3
:10229000ACE501287FF4AAAD0146328808200AF097
:1022A000CFFAA3E530B9012109200AF098FA00B26B
:1022B00030609BE501287FF499AD01463288092002
:1022C0000AF0BEFA92E500287FF490AD01210320C8
:1022D0000AF026FA294602200AF081FA306085E5E4
:1022E00000287FF483AD012103200AF019FA0121AF
:1022F00002200AF074FA306078E500287FF476ADA9
:10230000022103200AF00CFA294602200AF067FA9B
:1023100030606BE500287FF469AD014603200AF0C8
:10232000FFF9294602200AF05AFA30605EE50028DB
:102330007FF45CAD014603200AF0F2F9012102208E
:102340000AF04DFA306051E500287FF44FAD0321CB
:1023500008460AF0E5F9294602200AF040FA306002
:1023600044E500287FF442AD042103200AF0D8F9A7
:10237000294602200AF033FA306037E500287FF45E
:1023800035AD042103200AF0CBF9012102200AF027
:1023900026FA30602AE500287FF428AD05210320C5
:1023A0000AF0BEF9294602200AF019FA30601DE54C
:1023B00000287FF41BAD052103200AF0B1F90121AB
:1023C00002200AF00CFA306010E500287FF40EAD10
:1023D000062103200AF0A4F9294602200AF0FFF999
:1023E000306003E500287FF401AD072103200AF0E7
:1023F00097F9294602200AF0F2F93060F6E4002845
:102400007FF4F4AC072103200AF08AF901210220AD
:102410000AF0E5F93060E9E400287FF4E7AC082130
:1024200003200AF07DF9294602200AF0D8F930602D
:10243000DCE400287FF4DAAC082103200AF070F90C
:10244000012102200AF0CBF93060CFE400287FF4AC
:10245000CDAC092103200AF063F9294602200AF0D5
:10246000BEF93060C2E400287FF4C0AC01461220FF
:102470000AF0B5F900B23060B8E400287FF4B6ACD9
:10248000012112200AF0ABF900B23060AEE400285E
:102490007FF4ACAC014613200AF0A1F900B2306021
:1024A000A4E400287FF4A2AC014615200AF097F9B5
:1024B00000B230609AE400287FF498AC0121152026
:1024C0000AF08DF900B2306090E400287FF48EAC01
:1024D000014616200AF083F900B2306086E4002835
:1024E0007FF484AC012116200AF079F900B2306043
:1024F0007CE400287FF47AAC0A2103200AF010F96A
:10250000294602200AF06BF900B230606EE4002820
:102510007FF46CAC0A2103200AF002F901210220A9
:102520000AF05DF900B2306060E400287FF45EAC30
:102530000B2103200AF0F4F8294602200AF04FF993
:1025400000B2306052E400287FF450AC014606200F
:102550000AF045F9306049E400287FF447AC0121D6
:1025600006200AF03CF9306040E400287FF43EACDD
:1025700041200AF0A9F8306038E400287FF436AC36
:1025800042200AF0A1F8306030E400287FF42EAC3D
:10259000012146200AF023F900B2306026E4002829
:1025A0007FF424AC014646200AF019F900B23060ED
:1025B0001CE400287FF41AAC47200AF085F830604C
:1025C00014E400287FF412AC21200AF07DF830607A
:1025D0000CE400287FF40AAC22200AF075F8306081
:1025E00004E400287FF402AC014623200AF0F7F847
:1025F00000B23060FFF7FABB00287FF4F7AB27206A
:102600000AF062F820F07F403060FFF7EFBB00284F
:102610007FF4ECAB28200AF057F820F07F403060C0
:10262000FFF7E4BB00287FF4E1AB01212A200AF088
:10263000D6F800B23060FFF7D9BB00287FF4D6ABE4
:1026400001462A200AF0CBF800B23060FFF7CEBB7B
:1026500048B9D4216F200AF063F86E200AF034F8EC
:102660003060FFF7C3BB01287FF4C0ABD4216F20DB
:102670000AF056F831686E200AF052F8FFF7B6BB40
:1026800048B9D5216F200AF04BF86E200AF01CF8EB
:102690003060FFF7ABBB01287FF4A8ABD5216F20DA
:1026A0000AF03EF831686E200AF03AF8FFF79EBB58
:1026B00058B9D6216F200AF033F829466E200AF067
:1026C0008EF800B23060FFF791BB01287FF48EAB2B
:1026D000D6216F200AF024F8328800216E200AF0FB
:1026E000AFF8FFF783BB58B9D6216F200AF018F86E
:1026F00001216E200AF073F800B23060FFF776BB5C
:1027000001287FF473ABD6216F200AF009F83288D4
:1027100029466E200AF094F8FFF768BB58B9D72114
:102720006F2009F0FDFF29466E200AF058F800B22C
:102730003060FFF75BBB01287FF458ABD7216F20D7
:1027400009F0EEFF328800216E200AF079F8FFF7D9
:102750004DBB50B9D7216F2009F0E2FF01216E2057
:102760000AF03DF83060FFF741BB01287FF43EAB33
:10277000D7216F2009F0D4FF328829466E200AF055
:102780005FF8FFF733BB00287FF430AB01463920F8
:102790000AF025F800B23060FFF728BB00287FF46C
:1027A00025AB012139200AF01AF800B23060FFF79A
:1027B0001DBB00287FF41AAB01463D200AF00FF83C
:1027C00000B23060FFF712BB00287FF40FAB014668
:1027D0003F200AF004F800B23060FFF707BB002882
:1027E0007FF404AB01463A2009F0F9FF00B23060F3
:1027F000FFF7FCBA00287FF4F9AA0146532009F03C
:10280000EEFF00B23060FFF7F1BA38B90121642061
:1028100009F0E5FF00B23060FFF7E8BA01287FF465
:10282000E5AA0146328864200AF00AF8FFF7DEBA0A
:1028300038B90146642009F0D2FF00B23060FFF7DA
:10284000D5BA01287FF4D2AA32880021642009F089
:10285000F7FFFFF7CBBA00287FF4C8AA662009F07B
:1028600033FF3060FFF7C2BA00287FF4BFAA6820A8
:1028700009F02AFF3060FFF7B9BA00287FF4B6AA42
:102880000121692009F0ABFF00B23060FFF7AEBA5A
:1028900000287FF4ABAA0DF047F93060FFF7A6BA25
:1028A00000287FF4A3AA0146692009F098FF00B22E
:1028B0003060FFF79BBA00287FF498AA0DF0A8F9C2
:1028C0003060FFF793BA28B96B2009F0FDFE306045
:1028D000FFF78CBA01287FF489AA31686B2009F0D0
:1028E0001FFFFFF783BA00287FF480AA01466D20FE
:1028F00009F016FF6C2009F0E7FE3060FFF776BAAA
:1029000000287FF473AA01216D2009F009FF6C20D3
:1029100009F0DAFE3060FFF769BA00287FF466AA92
:1029200002216D2009F0FCFE6C2009F0CDFE306024
:10293000FFF75CBA00287FF459AA03216D2009F043
:10294000EFFE6C2009F0C0FE3060FFF74FBA0028A0
:102950007FF44CAA04216D2009F0E2FE6C2009F0FE
:10296000B3FE3060FFF742BA00287FF43FAA05218A
:102970006D2009F0D5FE6C2009F0A6FE3060FFF74F
:1029800035BA00287FF432AA06216D2009F0C8FE6E
:102990006C2009F099FE3060FFF728BA00287FF418
:1029A00025AA07216D2009F0BBFE6C2009F08CFEE2
:1029B0003060FFF71BBA20B90DF082F83060FFF7E6
:1029C00015BA01287FF412AA30680DF06DF8FFF7F0
:1029D0000DBA20B90DF09AF83060FFF707BA012858
:1029E0007FF404AA30680DF07EF8FFF7FFB90028E5
:1029F0007FF4FCA901216F2009F092FE6E2009F0FE
:102A000063FE3060FFF7F2B900287FF4EFA90221DE
:102A10006F2009F085FE6E2009F056FE3060FFF74A
:102A2000E5B900287FF4E2A903216F2009F078FEC0
:102A30006E2009F049FE3060FFF7D8B900287FF416
:102A4000D5A904216F2009F06BFE6E2009F03CFE31
:102A50003060FFF7CBB900287FF4C8A905216F20AB
:102A600009F05EFE6E2009F02FFE3060FFF7BEB960
:102A700000287FF4BBA906216F2009F051FE6E20CB
:102A800009F022FE3060FFF7B1B900287FF4AEA94B
:102A900007216F2009F044FE6E2009F015FE30601A
:102AA000FFF7A4B900287FF4A1A908216F2009F03D
:102AB00037FE29466E2009F092FE00B23060FFF723
:102AC00095B900287FF492A908216F2009F028FE0B
:102AD00001216E2009F083FE00B23060FFF786B955
:102AE00000287FF483A909216F2009F019FE2946E7
:102AF0006E2009F074FE00B23060FFF777B900284D
:102B00007FF474A90A216F2009F00AFE29466E207D
:102B100009F065FE00B23060FFF768B900287FF465
:102B200065A90A216F2009F0FBFD01216E2009F043
:102B300056FE00B23060FFF759B900287FF456A95D
:102B40000B216F2009F0ECFD29466E2009F047FEAD
:102B500000B23060FFF74AB900287FF447A90B2183
:102B60006F2009F0DDFD01216E2009F038FE00B272
:102B70003060FFF73BB900287FF438A90C216F20A3
:102B800009F0CEFD29466E2009F029FE00B2306022
:102B9000FFF72CB900287FF429A90C216F2009F038
:102BA000BFFD01216E2009F01AFE00B23060FFF770
:102BB0001DB900287FF41AA90D216F2009F0B0FD7E
:102BC00029466E2009F00BFE00B23060FFF70EB907
:102BD00000287FF40BA90D216F2009F0A1FD012130
:102BE0006E2009F0FCFD00B23060FFF7FFB800284E
:102BF0007FF4FCA80E216F2009F092FD29466E207B
:102C000009F0EDFD00B23060FFF7F0B800287FF466
:102C1000EDA80E216F2009F083FD01216E2009F03F
:102C2000DEFD00B23060FFF7E1B800287FF4DEA8D7
:102C30000F216F2009F074FD29466E2009F0CFFDA9
:102C400000B23060FFF7D2B800287FF4CFA80F2180
:102C50006F2009F065FD01216E2009F0C0FD00B272
:102C60003060FFF7C3B800287FF4C0A810216F20A0
:102C700009F056FD29466E2009F0B1FD00B2306022
:102C8000FFF7B4B800287FF4B1A811216F2009F034
:102C900047FD29466E2009F0A2FD00B23060FFF723
:102CA000A5B800287FF4A2A811216F2009F038FDF3
:102CB00001216E2009F093FD00B23060FFF796B855
:102CC00000287FF493A812216F2009F029FD2946DE
:102CD0006E2009F084FD00B23060FFF787B800284D
:102CE0007FF484A813216F2009F01AFD29466E2075
:102CF00009F075FD3060FFF779B800287FF476A8F9
:102D000013216F2009F00CFD01216E2009F067FDF1
:102D10003060FFF76BB848B9D0216F2009F000FD93
:102D20006E2009F0D1FC3060FFF760B801287FF415
:102D30005DA8D0216F2009F0F3FC31686E2009F006
:102D4000EFFCFFF753B848B9D1216F2009F0E8FC38
:102D50006E2009F0B9FC3060FFF748B801287FF415
:102D600045A8D1216F2009F0DBFC31686E2009F005
:102D7000D7FCFFF73BB858B9D2216F2009F0D0FC3F
:102D800029466E2009F02BFD00B23060FFF72EB807
:102D900001287FF42BA8D2216F2009F0C1FC3288D2
:102DA00000216E2009F04CFDFFF720B858B9D22160
:102DB0006F2009F0B5FC01216E2009F010FD00B272
:102DC0003060FFF713B801287FF410A8D2216F20DC
:102DD00009F0A6FC328829466E2009F031FDFFF784
:102DE00005B858B9D3216F2009F09AFC29466E2006
:102DF00009F0F5FC00B23060FEF7F8BF01287EF460
:102E0000F5AFD3216F2009F08BFC328800216E20B2
:102E100009F016FDFEF7EABF58B9D3216F2009F07B
:102E20007FFC01216E2009F0DAFC00B23060FEF771
:102E3000DDBF01287EF4DAAFD3216F2009F070FCEA
:102E4000328829466E2009F0FBFCFEF7CFBF002830
:102E50007EF4CCAFC0216F2009F062FC29466E20C1
:102E600009F0BDFC00B23060FEF7C0BF00287EF460
:102E7000BDAFC0216F2009F053FC01216E2009F085
:102E8000AEFC00B23060FEF7B1BF00287EF4AEAFFA
:102E9000C1216F2009F044FC29466E2009F09FFCF7
:102EA00000B23060FEF7A2BF00287EF49FAFC121C0
:102EB0006F2009F035FC01216E2009F090FC00B272
:102EC0003060FEF793BF00287EF490AFC2216F20E0
:102ED00009F026FC29466E2009F081FC00B2306022
:102EE000FEF784BF00287EF481AFC2216F2009F075
:102EF00017FC01216E2009F072FC00B23060FEF771
:102F000075BF00287EF472AFC3216F2009F008FC62
:102F100029466E2009F063FC00B23060FEF766BF00
:102F200000287EF463AFC3216F2009F0F9FB012173
:102F30006E2009F054FC00B23060FEF757BF002845
:102F40007EF454AFC4216F2009F0EAFB29466E20BD
:102F500009F045FC3060FEF749BF00287EF446AF1B
:102F6000C4216F2009F0DCFB01216E2009F037FC41
:102F70003060FEF73BBF00287EF438AFC5216F20DC
:102F800009F0CEFB29466E2009F029FC3060FEF7DF
:102F90002DBF00287EF42AAFC5216F2009F0C0FBA9
:102FA00001216E2009F01BFC3060FEF71FBF0028D6
:102FB0007EF41CAFC6216F2009F0B2FB29466E20BB
:102FC00009F00DFC3060FEF711BF00287EF40EAF53
:102FD000C6216F2009F0A4FB01216E2009F0FFFB40
:102FE0003060FEF703BF00287EF400AFC7216F20DA
:102FF00009F096FB29466E2009F0F1FB3060FEF7E0
:10300000F5BE00287EF4F2AEC7216F2009F088FBE0
:1030100001216E2009F0E3FB3060FEF7E7BE0028D7
:103020007EF4E4AEC8216F2009F07AFB6E2009F02F
:103030004BFB3060FEF7DABE00287EF4D7AEC92124
:103040006F2009F06DFB6E2009F03EFB3060FEF74B
:10305000CDBE00287EF4CAAECA216F2009F060FB05
:103060006E2009F031FB3060FEF7C0BE00287EF410
:10307000BDAECB216F2009F053FB6E2009F024FB7D
:103080003060FEF7B3BE20B90CF0CAFE3060FEF728
:10309000ADBE01287EF4AAAE30880CF0BBFEFEF770
:1030A000A5BE20B90CF0D0FE3060FEF79FBE01280F
:1030B0007EF49CAE30780CF0B9FEFEF797BE002887
:1030C0007EF494AE0CF0C6FE3060FEF78FBE002892
:1030D0007EF48CAE0CF0C4FE3060FEF787BE002894
:1030E0007EF484AE0CF004F93060FEF77FBED3F8B6
:1030F000E0000443FEF77ABE07B502AB43F8042DA7
:1031000002460120FEF76BFE03B05DF804FB134698
:1031100002460020FEF763BE0F4B9A78824204BF3E
:103120000E4A92F8D1001A78824206D10C4BDB6825
:103130001B689B690B4A106818475B78834209D16A
:10314000064B93F8D130834204D1054BDB681B68F2
:103150005B69EFE7704700BF781A00200400002089
:103160008C4D0208604D002010B5064B1878FFF713
:10317000D3FFBDE81040044B044ADB6810681B68AD
:103180009B691847781A00208C4D0208604D00207A
:1031900038B5244B244DDC6860682368C83028604B
:1031A000DB689847236828685B6998471F4B20496C
:1031B0005A6901240A601F49C2F804121E49C2F864
:1031C0000C120021117051701C4A5C741A621C4A66
:1031D00083F8D040DA611B4A9A611B4A5A621B4A43
:1031E000DA641B4A9A631B4A5A631B4A9A621B4A57
:1031F000DA621B4A9A641B4A5A641B4A5A651B4A84
:103200001A651B4A5A661B4A1A661B4ADA6532223D
:10321000DA6040F28A229A600CF028FC2046BDE871
:10322000384079E78C4D0208604D002004000020F2
:10323000E44D0020893301087D1D0108A91D010806
:10324000CD1D0108C91D0108C51D010899320108DD
:103250000F310108F93001088D1D01087D32010888
:10326000DB1D0108CF1D0108B9320108791D0108D5
:1032700019310108811D01086931010810B5054C9B
:1032800010B1D4F8E80010BD08680CF0D1FCD4F8F7
:10329000D40010BD0400002038B50D46054C10B117
:1032A000D4F8E80038BD0CF0B3FC2860D4F8D400A2
:1032B00038BD00BF0400002030B5314C85B0236814
:1032C0000546C31A002BB8BF5B42092B07DD6420FB
:1032D000636858430CF048F8002325606360636816
:1032E0002846013363600CF093FD0CF093F820B195
:1032F0000022114610460CF00FF90CF085F880B151
:103300000CF0F8F803280CD8DFE800F0110D0227C4
:103310000A2300931423019304AB13E90F000CF06C
:1033200093F805B030BD1E2300932823F3E7002156
:103330006F2009F0F5F96E2009F0C6F9012100901F
:10334000692009F04CFA00210446692009F047FA87
:1033500024B200B204440194DEE701212A2009F0DE
:103360003EFA00210446232009F039FA24B200B2C3
:10337000044B0190001B009402900393CCE700BF24
:103380008C2A0020F0D8FFFF0120704709F09CB97B
:1033900009F0C6B909F023BA09F052BA2DE9F34190
:1033A0001D46C34B5C7C1E468C4205D8D3F8E840D2
:1033B000204602B0BDE8F0811C2AD3F8D44000F0CA
:1033C000DD8300F2AB800C2A00F08E824BD8052AF8
:1033D00000F00E821AD8022A00F0BB8109D8002A18
:1033E00000F08381012A00F09A81D6F8E0000443BE
:1033F000DEE7032A00F0CE81042AF6D1002840F04F
:10340000D781AC4B53F821302B60D1E7082A00F06C
:10341000488213D8062A00F00582072AE5D1002841
:1034200040F026822020A44B884040F01000D3F8C2
:103430009832C0B29847C0B22860B9E70A2A00F0B3
:1034400040820B2AD1D10028B2D120209A4B88404B
:1034500040F01500D3F89832C0B29847C04300F04E
:1034600001002860A4E7122A00F0EA8229D80F2A76
:1034700000F0A48212D80D2A00F061820E2AB4D185
:10348000002840F08D8220208B4B884040F01400B3
:10349000D3F89832C0B29847286089E7102A00F024
:1034A000A782112AA1D1002840F0BC822020824BA3
:1034B000884040F00800D3F89832C0B2984728609E
:1034C00076E7152A00F0FE8212D8132A00F0D28285
:1034D000142A8AD1002840F0E7822020764B8840C9
:1034E00040F00B00D3F89832C0B2984728605FE7ED
:1034F000172A00F01B83C0F0FF82182A7FF475AFF3
:10350000002840F02D8320206B4B884040F01300B2
:10351000D3F89832C0B29847286049E7AC2A00F047
:103520006B8566D8A52A00F00D8433D8A22A00F056
:10353000A28319D81D2A00F047838C2A7FF455AF47
:10354000002840F04D8308015B4B40F06C00D3F83D
:10355000983200F0FC0098474FF48073C0F303608A
:1035600043FA00F0286023E7A32A00F0AC83A42AE2
:103570007FF43BAF002840F0CD8308014E4B40F074
:103580006C00D3F8983200F0FC009847C0F300308C
:1035900028600DE7A82A00F09D8415D8A62A00F01F
:1035A0002D84A72A7FF421AF002840F07B840801F6
:1035B000414B40F06C00D3F8983200F0FC00984783
:1035C00000F00F002860F3E6AA2A00F0D48440F24D
:1035D000A884002840F0F7840801374B40F06D00C4
:1035E000D3F8983200F0FD009847C0F341102860EE
:1035F000DEE6B62A00F0C8853FD8B32A00F063851E
:103600001DD8AD2A00F01F85AE2A7FF4EEAE00284B
:1036100040F040850801284B40F06D00D3F8983207
:1036200000F0FD009847001410F0400F0CBF00237D
:103630006FF07F0300F07F0213432B60B8E6B42ADB
:1036400000F06885B52A7FF4D0AE002840F072857E
:103650002020884046B2184F46F01400D7F8983220
:10366000C0B2984741057FF5A3AE46F01100D7F8E8
:103670009832C0B2984728609AE6CE2A00F0E285D8
:103680001CD8B82A00F09C85B92A7FF4AEAE002879
:1036900040F0BD850801084B40F06C00D3F898322B
:1036A00000F0FC009847C0F30350286080E600BF9C
:1036B00004000020A02A002080010020D22A00F06F
:1036C000E085D32A00F0F985D12A7FF48EAE002858
:1036D00040F0C8852020AF4B884040F01900D3F857
:1036E0009832C0B29847286062E650B92020A94BB2
:1036F000884040F00D00D3F89832C0B29847286057
:1037000056E601287FF454AE2020A24B884040F0BA
:103710000D00D3F894322968C0B2984748E650B9F2
:1037200020209C4B884040F00100D3F89832C0B272
:10373000984728603CE601287FF43AAE2020954B5C
:10374000884040F00100D3F894322968C0B298470D
:103750002EE650B920208F4B884040F00700D3F868
:103760009832C0B29847286022E601287FF420AE44
:1037700001222020884B88405A542A68854B82EACF
:10378000E27140F00700D3F89432A1EBE271C0B2CD
:1037900098470DE600287FF40BAE20207D4B884033
:1037A00040F00200D3F89832C0B298472860FFE595
:1037B00001287FF4FDAD20202B68784A002B754F3F
:1037C000B8BF5B4200FA01F642F82130F0B2D7F8F8
:1037D0009832984700287FF4EBAD296846F007003F
:1037E0000029D7F89432B8BF4942C0B29847DFE504
:1037F00050B92020674B884040F00600D3F898323B
:10380000C0B298472860D3E501287FF4D1AD2020CD
:10381000604B884040F00600D3F894322968C0B26B
:103820009847C5E560B920205A4B884040F0100009
:10383000D3F89832C0B29847C0F307202860B7E5A4
:1038400001287FF4B5AD20208840524F40F010068B
:10385000F6B2D7F8983230469847C2B22B78009229
:10386000D7F89052C0F3074200213046A8479FE5A1
:1038700001287FF49DAD20208840464F40F010067F
:10388000F6B2D7F89832304698472B78C0F3074203
:103890000093D7F89052C0F3072300213046A84781
:1038A00086E500287FF484AD20203A4B884040F024
:1038B0001500D3F89832C0B29847C0F34020286072
:1038C00076E500287FF474AD2020324B884040F02C
:1038D0001500D3F89832C0B2984710F0020F0CBF11
:1038E000012300232B6063E560B92020294B884029
:1038F00040F01400D3F89832C0B29847C0F34000AB
:10390000286055E501287FF453AD2020884040F021
:103910001406204FF6B2D7F89832304698472B68F5
:1039200033B940F00201D7F89432304698473FE56A
:1039300020F00201D7F894323046984738E560B954
:103940002020144B884040F01400D3F89832C0B2C5
:10395000984700F0010028602AE501287FF428AD8F
:103960002020884040F014060A4FF6B2D7F898326B
:10397000304698472B6833B940F00101D7F89432AC
:103980003046984714E520F00101D7F894323046CC
:1039900098470DE5800100205C100020A02A00203F
:1039A00001287FF405AD2020A44B884040F014008E
:1039B000D3F894322968C0B29847F9E450B920206E
:1039C0009E4B884040F00400D3F89832C0B298472C
:1039D0002860EDE401287FF4EBAC2020974B884071
:1039E00040F00400D3F894322968C0B29847DFE46D
:1039F00050B92020914B884040F00500D3F8983210
:103A0000C0B298472860D3E401287FF4D1AC2020CD
:103A10008A4B884040F00500D3F894322968C0B240
:103A20009847C5E401287FF4C3AC2020834B88402D
:103A300040F00800D3F894322968C0B29847B7E440
:103A400050B920207D4B884040F00A00D3F89832CE
:103A5000C0B298472860ABE401287FF4A9AC2020CD
:103A6000764B884040F00A00D3F894322968C0B2FF
:103A700098479DE450B92020704B884040F00300E7
:103A8000D3F89832C0B29847286091E401287FF4B7
:103A90008FAC2020694B884040F00300D3F894326B
:103AA0002968C0B2984783E401287FF481AC2020C4
:103AB000624B884040F00B00D3F894322968C0B2C2
:103AC000984775E450B920205C4B884040F00C00CA
:103AD000D3F89832C0B29847286069E401287FF48F
:103AE00067AC2020554B884040F00C00D3F894324E
:103AF0002968C0B298475BE450B920204F4B8840FA
:103B000040F01100D3F89832C0B2984728604FE4D3
:103B100001287FF44DAC2020484B884040F0110034
:103B2000D3F894322968C0B2984741E450B92020B4
:103B3000424B884040F01200D3F89832C0B2984708
:103B4000286035E401287FF433AC20203B4B8840CB
:103B500040F01200D3F894322968C0B2984727E4A5
:103B600001287FF425AC2020344B884040F013001E
:103B7000D3F894322968C0B2984719E460B90801B3
:103B80002E4B40F06C00D3F8983200F0FC009847C0
:103B9000C0F3804028600BE401287FF409AC0801E1
:103BA00040F06C06254FF6B2D7F898323046984769
:103BB0002B6820F480210BB141F48021D7F8943296
:103BC00030469847FFF7F4BB00287FF4F1AB1B4A5F
:103BD00053689268002918BF13462B60FFF7E8BBB3
:103BE00001287FF4E5AB2B68102B23D00DDC022BD2
:103BF0001CD004DC012B16D04FF0FF3314E0042B53
:103C000016D0082BF8D105230EE0402B14D003DC8E
:103C1000202BF1D1032307E0802B11D0B3F5807F57
:103C2000EAD1002300E008232B600AE00723FBE72A
:103C30000623F9E70423F7E70223F5E780010020D4
:103C400028602B6801333FF4B3AB0801BC4F40F050
:103C50006C06F6B2D7F89832304698472B6820F0B9
:103C600070611B0603F07063D7F894221943304645
:103C70009047FFF79DBB68B90801B14B40F06C005D
:103C8000D3F8983200F0FC009847C0F3C1302860A8
:103C9000FFF78EBB01287FF48BAB0801A84F40F0E3
:103CA0006C06F6B2D7F89832304698472B6820F465
:103CB000C031DB0303F4C033D7F8942219433046F4
:103CC0009047FFF775BB68B908019D4B40F06C0049
:103CD000D3F8983200F0FC009847C0F38030286099
:103CE000FFF766BB01287FF463AB080140F06C0668
:103CF000934FF6B2D7F89832304698472B6820F4A5
:103D000080410BB141F48041D7F894323046984756
:103D1000FFF74EBB01287FF44BAB080140F06C0667
:103D2000874FF6B2D7F89832304698472B6820F480
:103D300080510BB141F48051D7F894323046984706
:103D4000FFF736BB20BB080140F06C067C4FF6B293
:103D5000D7F898323046984710F4804FD7F8983209
:103D6000304605D09847C0F3C3102860FFF720BB4A
:103D70009847D7F8983280463046984718F4006F35
:103D8000C0F3021018BF40F008002860FFF710BB16
:103D900001287FF40DAB080140F06C06684FF6B2C5
:103DA000D7F898323046984710F4804F10D0D7F8A3
:103DB0009832304698472B6820F4F061DB0103F419
:103DC000F063D7F89422194330469047FFF7F0BAD2
:103DD000D7F89832304698472968D7F894320D07BB
:103DE0004CBF40F4006020F40060090120F0700036
:103DF000C9B2014330469847FFF7DABA20BB080141
:103E000040F06C064E4FF6B2D7F8983230469847DD
:103E100010F4804FD7F89832304605D09847C0F359
:103E200002102860FFF7C4BA9847D7F89832804646
:103E30003046984718F4006FC0F3C31018BF40F025
:103E400008002860FFF7B4BA01287FF4B1AA08017E
:103E500040F06C063A4FF6B2D7F8983230469847A1
:103E600010F4804FD7F8983230460DD098472B6821
:103E700020F070011B0103F07003D7F8942219435E
:103E800030469047FFF794BA98472B6820F4F061CA
:103E9000DB0103F4F063D7F89422194330469047CE
:103EA000FFF786BA01287FF483AA0801244F40F067
:103EB0006C06F6B2D7F89832304698472B6820F057
:103EC0000F0103F00F03D7F89422194330469047AF
:103ED000FFF76EBA68B90801194B40F06D00D3F8CE
:103EE000983200F0FD009847C0F3C0302860FFF71B
:103EF0005FBA01287FF45CAA080140F06D06104FFC
:103F0000F6B2D7F89832304698472B6820F4004133
:103F10000BB141F40041D7F8943230469847FFF78F
:103F200047BA78B90801064B40F06D00D3F89832D3
:103F300000F0FD009847C0F341302860FFF738BA21
:103F40008001002001287FF433AA0801BC4F40F013
:103F50006D06F6B2D7F89832304698472B6820F4B1
:103F6000C0415B0303F4C043D7F8942219433046A1
:103F70009047FFF71DBA68B90801B14B40F06D00DA
:103F8000D3F8983200F0FD009847C0F30320286072
:103F9000FFF70EBA01287FF40BAA0801A84F40F0E2
:103FA0006D06F6B2D7F89832304698472B6820F461
:103FB00070611B0203F47063D7F8942219433046F2
:103FC0009047FFF7F5B901287FF4F2A908019C4F4B
:103FD00040F06D06F6B2D7F89832304698472B6815
:103FE00020F060015B0103F06003D7F894221943CD
:103FF00030469047FFF7DCB968B90801904B40F0B4
:104000006D00D3F8983200F0FD00984700F00F00E3
:104010002860FFF7CDB901287FF4CAA90801884FAD
:1040200040F06D06F6B2D7F89832304698472B68C4
:1040300020F00F0103F00F03D7F894221943304604
:104040009047FFF7B5B968B908017D4B40F06D00A6
:10405000D3F8983200F0FD009847C0F30060286064
:10406000FFF7A6B901287FF4A3A9080140F06D0667
:10407000734FF6B2D7F89832304698472B6820F045
:1040800080710BB141F08071D7F894323046984777
:10409000FFF78EB901287FF48BA90801684F40F023
:1040A0006D06F6B2D7F89832304698472B6820F460
:1040B000FE011B0403F4FE03D7F894221943304693
:1040C0009047FFF775B968B908015D4B40F06C0087
:1040D000D3F8983200F0FC009847C0F340402860C5
:1040E000FFF766B901287FF463A9080140F06C0668
:1040F000534FF6B2D7F89832304698472B6820F4E1
:1041000000310BB141F40031D7F894323046984772
:10411000FFF74EB900287FF44BA90801484B40F047
:104120006F00D3F89832C0B29847C0F307402860B8
:10413000FFF73EB901287FF43BA920208840404F7B
:1041400046B246F0110046F014062968F6B2D7F8D8
:104150009432C0B29847D7F898323046984720F446
:1041600080684146D7F89432304698472B683046ED
:10417000002B0CBF00214FF48061D7F8943241EA44
:1041800008019847FFF714B958B920202C4B8840F4
:1041900040F01100D3F89832C0B298472860FFF77A
:1041A00007B901287FF404A92020254B884040F05E
:1041B0001100D3F894322968C0B29847FFF7F8B8D5
:1041C00068B908011E4B40F06C00D3F8983200F03B
:1041D000FC009847C0F340302860FFF7E9B8012899
:1041E0007FF4E6A8080140F06C06154FF6B2D7F848
:1041F0009832304698472B6820F400510BB141F4B7
:104200000051D7F8943230469847FFF7D1B80128CB
:104210007FF4CEA808010A4F40F06C06F6B2D7F83A
:104220009832304698472B6820F470011B0503F440
:104230007003D7F89422194330469047FFF7B8B877
:104240008001002000287FF4B3A80801444B40F00F
:104250006F00D3F89832C0B29847C0F309002860C5
:10426000FFF7A6B801287FF4A3A820203C4B884084
:1042700040F01900D3F894322968C0B29847FFF78C
:1042800097B858B92020364B884040F01A00D3F830
:104290009832C0B298472860FFF78AB801287FF4A7
:1042A00087A820202E4B884040F01A00D3F8943283
:1042B0002968C0B29847FFF77BB8F0B979B10129F6
:1042C0007FF476A8264BD3F89832984700F0600028
:1042D000A0F12003584258412860FFF769B8204BED
:1042E0000846D3F89832984700F01800A0F1100261
:1042F000504250412860FFF75BB801287FF458A86E
:1043000099B101297FF454A8154E0020D6F89832AF
:1043100098472B68FBB120F0400141F02001D6F80E
:10432000943200209847FFF743B80D4E0846D6F860
:10433000983298472B684BB120F0080141F01001EA
:10434000D6F8943200209847FFF732B820F01001D9
:1043500041F00801F4E720F0200141F04001DEE7E0
:104360008001002007B502AB43F8042D024601206E
:10437000FFF714F803B05DF804FB13460246002073
:10438000FFF70CB8014BD3F8943218478001002096
:10439000034B10B5D3F898320C469847206010BDF7
:1043A00080010020014BD3F88C3218478001002097
:1043B0000022014B5A607047040000202DE9F341B0
:1043C000154B06465A7C884682421F4604D8D3F8CD
:1043D000E80002B0BDE8F0812024104D844044F094
:1043E000070081EAE171D5F89432A1EBE871C0B21F
:1043F000984701230A4AB8F1000F9355B8BF02232A
:1044000000930023E0B21A46D5F890421946A0471F
:10441000D7F8D400DDE700BF0400002080010020B1
:104420005C100020CAE74942C8E70021C6E72DE931
:10443000F3411A4B04465A7C0F4682421E4604D86A
:10444000D3F8E80002B0BDE8F081DFF85C80144DDD
:1044500018F800306BB12020124AA04040F007004D
:10446000D5F8943252F82410C0B29847002308F8C7
:104470000430202303FA04F444F00D00D5F89432FC
:104480003946C0B2984700230093E0B2D5F8905265
:104490001A461946A847D6F8D400D3E704000020EE
:1044A00080010020A02A00205C10002038B50446BE
:1044B0002020084BA0400D4640F00100D3F8983270
:1044C000C0B298472B68C11829602046BDE8384023
:1044D000ADE700BF80010020094B5A7C82421A469A
:1044E00002D8D3F8E800704720B10128F9D1054B74
:1044F0009B6801E0034B5B680B60D2F8D400704707
:104500000400002080010020012810B5144613D0BB
:1045100005D302281CD0124BD3F8E00010BD14685C
:10452000104A114BD268126824B1526958699047F9
:10453000002010BD9269F9E70A4B0B4ADB68D0688E
:104540001B681B6A9847003018BF01202060EFE706
:10455000044B054ADB6810691B681B6AF2E700BF61
:10456000040000208C4D0208A02A002038B50B4B17
:104570000B4D9C782CB1D5F8A032984701242046E9
:1045800038BDD5F89832222098470028F7D1D5F8C1
:104590009832422098470028EDD0F0E7341A0020E6
:1045A00080010020022804BF0B4B93F8D10030B9E2
:1045B0000A4BDB681B685B69094A90681847012849
:1045C00009D1054B93F8D130012B04D1034BDB68A3
:1045D0001B689B69F0E77047040000208C4D0208BF
:1045E000A02A002070B53D4E3D4CF5686B6803F580
:1045F000AA72E26003F5B872226103F56F7262611C
:1046000003F5767203F1C800A26103F57D7203F52C
:10461000826323622B68E261DB68A06098472B68A5
:104620006069DB6898472B6860699B6998472B68CD
:10463000E0681B6998472B6820691B6998472B68BD
:10464000206A1B6998472B68A0691B6998472B68EB
:10465000E0691B6998476B68326903F537735360EB
:104660002049214B0A605A692048C1F89C22D1F8A0
:10467000A412C2F80402C2F80C12002111701C4AE4
:1046800032211A621B4AD960DA611B4AB6219A614B
:104690001A4A99605A621A4A01209A63194A5A635F
:1046A000194A9A62194ADA62194A9A64194A5A648A
:1046B000194A5A65194A1A65194ADA64194A5A6632
:1046C000194A1A6602225A7483F8D020174A9A654A
:1046D000174ADA65BDE8704064E700BF8C4D0208F8
:1046E000A02A002080010020040000206D45010860
:1046F000BD43010825440108274401082B44010853
:104700007B430108654301082F440108AD440108BB
:104710008543010891430108A543010809450108A3
:10472000D9440108A5450108B1430108E545010840
:104730003547010870B50020FFF734FF104B114CCE
:10474000DD68A0682B689B6898472B68E0689B68C9
:1047500098472B6820699B6898472B68206A9B685C
:1047600098472B68A0699B6898472B68E0699B680D
:1047700098472B6860699B68BDE87040184700BF88
:104780008C4D0208A02A00202DE9F3411D46C64B9E
:104790005C7C1E468C4205D8D3F8E840204602B027
:1047A000BDE8F0811C2AD3F8D44000F0D18300F298
:1047B000AB800C2A00F07D824BD8052A00F0FD81E9
:1047C0001AD8022A00F0AA8109D8002A00F07281C2
:1047D000012A00F08981D6F8E0000443DEE7032ACD
:1047E00000F0BD81042AF6D1002840F0C681AF4B0D
:1047F00053F821302B60D1E7082A00F0378213D814
:10480000062A00F0F481072AE5D1002840F015823D
:104810002020A74B884040F01000D3F89832C0B257
:104820009847C0B22860B9E70A2A00F02F820B2A05
:10483000D1D10028B2D120209D4B884040F01500F6
:10484000D3F89832C0B29847C04300F00100286006
:10485000A4E7122A00F0DE8229D80F2A00F09882FD
:1048600012D80D2A00F053820E2AB4D1002840F04D
:104870007A8220208E4B884040F01400D3F8983282
:10488000C0B29847286089E7102A00F09B82112A5D
:10489000A1D1002840F0B0822020854B884040F014
:1048A0000800D3F89832C0B29847286076E7152AF6
:1048B00000F0F28212D8132A00F0C682142A8AD19C
:1048C000002840F0DB822020794B884040F00B002C
:1048D000D3F89832C0B2984728605FE7172A00F0F3
:1048E0000F83C0F0F382182A7FF475AF002840F0E0
:1048F000218320206E4B884040F01300D3F898327B
:10490000C0B29847286049E7AB2A00F0368567D8DF
:10491000A52A00F0008433D8A22A00F0958319D884
:104920001D2A00F03A838C2A7FF455AF002840F00E
:10493000408308015E4B40F06C00D3F8983200F0E1
:10494000FC0098474FF48073C0F3036043FA00F013
:10495000286023E7A32A00F09F83A42A7FF43BAFBB
:10496000002840F0C0830801514B40F06C00D3F8A0
:10497000983200F0FC009847C0F3003028600DE743
:10498000A82A00F0908415D8A62A00F02084A72A2F
:104990007FF421AF002840F06E840801444B40F0C2
:1049A0006C00D3F8983200F0FC00984700F00F003C
:1049B0002860F3E6A92A00F09D84AA2A7FF40BAFB1
:1049C000002840F0C1840801394B40F06D00D3F855
:1049D000983200F0FD009847C0F303202860DDE620
:1049E000B52A00F088852ED8AE2A00F02D8515D87E
:1049F000AC2A00F0EA84AD2A7FF4EDAE002840F046
:104A00000B8508012A4B40F06D00D3F8983200F076
:104A1000FD009847C0F300602860BFE6B32A00F0AD
:104A20004385B42A7FF4D7AE00287FF4B7AE0801DF
:104A30001F4B40F06F00D3F89832C0B29847C0F3D4
:104A400007402860AAE6CE2A00F0B38515D8B62A1A
:104A500000F07B85B82A7FF4BEAE002840F0918537
:104A60000801134B40F06C00D3F8983200F0FC00C2
:104A70009847C0F34030286090E6D22A00F0B8850D
:104A8000D32A00F0D185D12A7FF4A5AE002840F0CA
:104A9000A0852020064B884040F01900D3F89832BA
:104AA000C0B29847286079E604000020D02A002090
:104AB0002804002050B92020B24B884040F00D005F
:104AC000D3F89832C0B29847286067E601287FF48F
:104AD00065AE2020AB4B884040F00D00D3F89432F7
:104AE0002968C0B2984759E650B92020A54B8840A4
:104AF00040F00100D3F89832C0B2984728604DE6E4
:104B000001287FF44BAE20209E4B884040F00100EE
:104B1000D3F894322968C0B298473FE650B92020B4
:104B2000984B884040F00700D3F89832C0B29847BD
:104B3000286033E601287FF431AE01222020924B19
:104B400088405A542A688F4B82EAE27140F007008D
:104B5000D3F89432A1EBE271C0B298471EE6002868
:104B60007FF41CAE2020874B884040F00200D3F831
:104B70009832C0B29847286010E601287FF40EAE44
:104B800020202B68814A002B7E4FB8BF5B4200FA81
:104B900001F642F82130F0B2D7F898329847002851
:104BA0007FF4FCAD296846F007000029D7F894325D
:104BB000B8BF4942C0B29847F0E550B92020714BC8
:104BC000884040F00600D3F89832C0B29847286079
:104BD000E4E501287FF4E2AD20206A4B884040F0F4
:104BE0000600D3F894322968C0B29847D6E560B978
:104BF0002020644B884040F01000D3F89832C0B2B7
:104C00009847C0F307202860C8E501287FF4C6ADA7
:104C1000202088405B4F40F01006F6B2D7F898325B
:104C200030469847C2B22B780092D7F89052C0F322
:104C3000074200213046A847B0E501287FF4AEAD19
:104C4000202088404F4F40F01006F6B2D7F8983237
:104C5000304698472B78C0F307420093D7F890521C
:104C6000C0F3072300213046A84797E500287FF4CA
:104C700095AD2020434B884040F01500D3F8983282
:104C8000C0B29847C0F34020286087E500287FF431
:104C900085AD20203B4B884040F01500D3F898327A
:104CA000C0B2984710F0020F0CBF012300232B6005
:104CB00074E560B92020334B884040F01400D3F8ED
:104CC0009832C0B29847C0F34000286066E50128DA
:104CD0007FF464AD202088402A4F40F01406F6B2DD
:104CE000D7F89832304698472B6820F00A00002BFE
:104CF0000CBF00210221022B40EA010014BF002159
:104D00000821D7F8943201433046984746E560B908
:104D100020201C4B884040F01400D3F89832C0B2D9
:104D2000984700F00100286038E501287FF436AD8F
:104D300020208840134F40F01406F6B2D7F898327E
:104D4000304698472B6820F00500002B18BF40F034
:104D50000100022B14BF00210421D7F89432014333
:104D6000304698471AE501287FF418AD2020054BFE
:104D7000884040F01400D3F894322968C0B29847B4
:104D80000CE500BF2804002064100020D02A002079
:104D900050B92020AB4B884040F00400D3F8983243
:104DA000C0B298472860F9E401287FF4F7AC2020CE
:104DB000A44B884040F00400D3F894322968C0B274
:104DC0009847EBE450B920209E4B884040F0050006
:104DD000D3F89832C0B298472860DFE401287FF406
:104DE000DDAC2020974B884040F00500D3F894328A
:104DF0002968C0B29847D1E401287FF4CFAC2020C5
:104E0000904B884040F00800D3F894322968C0B233
:104E10009847C3E450B920208A4B884040F00A00EC
:104E2000D3F89832C0B298472860B7E401287FF4DD
:104E3000B5AC2020834B884040F00A00D3F8943270
:104E40002968C0B29847A9E450B920207D4B88401A
:104E500040F00300D3F89832C0B2984728609DE430
:104E600001287FF49BAC2020764B884040F0030063
:104E7000D3F894322968C0B298478FE401287FF4B0
:104E80008DAC20206F4B884040F00B00D3F894325B
:104E90002968C0B2984781E450B92020694B884006
:104EA00040F00C00D3F89832C0B29847286075E4FF
:104EB00001287FF473AC2020624B884040F00C0046
:104EC000D3F894322968C0B2984767E450B92020DB
:104ED0005C4B884040F01100D3F89832C0B298473C
:104EE00028605BE401287FF459AC2020554B8840B2
:104EF00040F01100D3F894322968C0B298474DE4CD
:104F000050B920204F4B884040F01200D3F898321F
:104F1000C0B29847286041E401287FF43FAC2020CC
:104F2000484B884040F01200D3F894322968C0B250
:104F3000984733E401287FF431AC2020414B88406E
:104F400040F01300D3F894322968C0B2984725E4A2
:104F500060B908013B4B40F06C00D3F8983200F088
:104F6000FC009847C0F38040286017E401287FF4D4
:104F700015AC080140F06C06324FF6B2D7F8983203
:104F8000304698472B6820F480210BB141F48021F2
:104F9000D7F894323046984700E400287FF4FEABFF
:104FA000284A53689268002918BF13462B60FFF700
:104FB000F5BB01287FF4F2AB2B68102B23D00DDC5E
:104FC000022B1CD004DC012B16D04FF0FF3314E071
:104FD000042B16D0082BF8D105230EE0402B14D05B
:104FE00003DC202BF1D1032307E0802B0FD0B3F596
:104FF000807FEAD1002300E008232B6008E007232C
:10500000FBE70623F9E70423F7E70223F5E7286027
:105010002B6801333FF4C2AB08010A4F40F06C0625
:10502000F6B2D7F89832304698472B6820F0706176
:105030001B0603F07063D7F894221943304690475B
:10504000FFF7ACBB2804002068B90801BD4B40F055
:105050006C00D3F8983200F0FC009847C0F3C130E0
:105060002860FFF79BBB01287FF498AB0801B54F80
:1050700040F06C06F6B2D7F89832304698472B6865
:1050800020F4C031DB0303F4C033D7F89422194372
:1050900030469047FFF782BB68B90801A94B40F042
:1050A0006C00D3F8983200F0FC009847C0F38030D1
:1050B0002860FFF773BB01287FF470AB080140F054
:1050C0006C06A04FF6B2D7F89832304698472B6856
:1050D00020F480410BB141F48041D7F8943230463E
:1050E0009847FFF75BBB01287FF458AB080140F0FD
:1050F0006C06944FF6B2D7F89832304698472B6832
:1051000020F480510BB141F48051D7F894323046ED
:105110009847FFF743BB20BB080140F06C06894F5E
:10512000F6B2D7F898323046984710F4804FD7F847
:105130009832304605D09847C0F3C3102860FFF777
:105140002DBB9847D7F8983280463046984718F4D8
:10515000006FC0F3021018BF40F008002860FFF78E
:105160001DBB01287FF41AAB080140F06C06754F97
:10517000F6B2D7F898323046984710F4804F10D0E6
:10518000D7F89832304698472B6820F4F061DB015D
:1051900003F4F063D7F89422194330469047FFF7A1
:1051A000FDBAD7F89832304698472968D7F8943234
:1051B0000D074CBF40F4006020F40060090120F0AE
:1051C0007000C9B2014330469847FFF7E7BA20BBE9
:1051D000080140F06C065B4FF6B2D7F898323046C3
:1051E000984710F4804FD7F89832304605D098474A
:1051F000C0F302102860FFF7D1BA9847D7F8983269
:1052000080463046984718F4006FC0F3C31018BFAB
:1052100040F008002860FFF7C1BA01287FF4BEAA59
:10522000080140F06C06474FF6B2D7F89832304686
:10523000984710F4804FD7F8983230460DD09847F1
:105240002B6820F070011B0103F07003D7F8942243
:10525000194330469047FFF7A1BA98472B6820F4CE
:10526000F061DB0103F4F063D7F894221943304670
:105270009047FFF793BA01287FF490AA0801314FB5
:1052800040F06C06F6B2D7F89832304698472B6853
:1052900020F00F0103F00F03D7F894221943304692
:1052A0009047FFF77BBA68B90801264B40F06D00C4
:1052B000D3F8983200F0FD009847C0F3C030286062
:1052C000FFF76CBA01287FF469AA080140F06D0667
:1052D0001C4FF6B2D7F89832304698472B6820F426
:1052E00000410BB141F40041D7F894323046984761
:1052F000FFF754BA68B90801124B40F06D00D3F8BB
:10530000983200F0FD009847C0F341302860FFF765
:1053100045BA01287FF442AA08010A4F40F06D0601
:10532000F6B2D7F89832304698472B6820F4C0413F
:105330005B0303F4C043D7F89422194330469047E7
:10534000FFF72CBA2804002001287FF427AA0801BF
:10535000BE4F40F06D06F6B2D7F898323046984707
:105360002B6820F470611B0203F47063D7F8942259
:10537000194330469047FFF711BA68B90801B34B9B
:1053800040F06D00D3F8983200F0FD009847C0F36C
:1053900041102860FFF702BA01287FF4FFA9080135
:1053A000AA4F40F06D06F6B2D7F8983230469847CB
:1053B0002B6820F060015B0103F06003D7F89422B2
:1053C000194330469047FFF7E9B968B908019F4B88
:1053D00040F06D00D3F8983200F0FD00984700F0DF
:1053E0000F002860FFF7DAB901287FF4D7A9080178
:1053F000964F40F06D06F6B2D7F89832304698478F
:105400002B6820F00F0103F00F03D7F89422194303
:1054100030469047FFF7C2B901287FF4BFA90801C1
:1054200040F06D06894FF6B2D7F89832304698476B
:105430002B6820F080710BB141F08071D7F8943265
:1054400030469847FFF7AAB9A8B908017F4B40F04A
:105450006D00D3F8983200F0FD009847001410F06A
:10546000400F0CBF00236FF07F0300F07F02134357
:105470002B60FFF793B901287FF490A90801734FBF
:1054800040F06D06F6B2D7F89832304698472B6850
:1054900020F4FE011B0403F4FE03D7F89422194301
:1054A00030469047FFF77AB968B90801674B40F07A
:1054B0006C00D3F8983200F0FC009847C0F34040ED
:1054C0002860FFF76BB901287FF468A9080140F054
:1054D0006C065E4FF6B2D7F89832304698472B6884
:1054E00020F400310BB141F40031D7F8943230464A
:1054F0009847FFF753B901287FF450A9202088402E
:10550000524F46B246F0110046F014062968F6B232
:10551000D7F89432C0B29847D7F8983230469847B7
:1055200020F480684146D7F89432304698472B687B
:105530003046002B0CBF00214FF48061D7F8943225
:1055400041EA08019847FFF729B958B920203F4B95
:10555000884040F01100D3F89832C0B298472860D4
:10556000FFF71CB901287FF419A92020374B884088
:1055700040F01100D3F894322968C0B29847FFF781
:105580000DB901287FF40AA9080140F06C062F4FDD
:10559000F6B2D7F89832304698472B6820F400517D
:1055A0000BB141F40051D7F8943230469847FFF7D9
:1055B000F5B800287FF4F2A80801244B40F06F00F2
:1055C000D3F89832C0B29847C0F309002860FFF7BB
:1055D000E5B801287FF4E2A820201C4B884040F069
:1055E0001900D3F894322968C0B29847FFF7D6B8AB
:1055F00058B92020154B884040F01A00D3F8983253
:10560000C0B298472860FFF7C9B801287FF4C6A840
:1056100020200E4B884040F01A00D3F894322968BD
:10562000C0B29847FFF7BAB800BB89B101297FF42F
:10563000B5A8064BD3F89832984700F06000A0F167
:105640002003584258412860FFF7A8B828040020DA
:10565000204B0846D3F89832984700F01800A0F184
:105660001002504250412860FFF798B801287FF49B
:1056700095A899B101297FF491A8164E0020D6F87B
:10568000983298472B68FBB120F0400141F020018F
:10569000D6F8943200209847FFF780B80D4E0846A0
:1056A000D6F8983298472B684BB120F0080141F0AA
:1056B0001001D6F8943200209847FFF76FB820F019
:1056C000100141F00801F4E720F0A00141F0400191
:1056D000DEE700BF2804002007B502AB43F8042D25
:1056E00002460120FFF750F803B05DF804FB1346B3
:1056F00002460020FFF748B8014BD3F89432184710
:1057000028040020034B10B5D3F898320C46984774
:10571000206010BD28040020014BD3F88C321847BC
:10572000280400200022014B5A607047040000202A
:105730002DE9F341154B06465A7C884682421F46A6
:1057400004D8D3F8E80002B0BDE8F0812024104D61
:10575000844044F0070081EAE171D5F89432A1EB6E
:10576000E871C0B2984701230A4AB8F1000F935577
:10577000B8BF022300930023E0B21A46D5F8904246
:105780001946A047D7F8D400DDE700BF0400002089
:105790002804002064100020CAE74942C8E700211D
:1057A000C6E72DE9F3411A4B04465A7C0F46824264
:1057B0001E4604D8D3F8E80002B0BDE8F081DFF857
:1057C0005C80144D18F800306BB12020124AA040C4
:1057D00040F00700D5F8943252F82410C0B2984730
:1057E000002308F80430202303FA04F444F00D00E9
:1057F000D5F894323946C0B2984700230093E0B2FE
:10580000D5F890521A461946A847D6F8D400D3E7DF
:105810000400002028040020D02A0020641000206A
:1058200038B504462020084BA0400D4640F001004A
:10583000D3F89832C0B298472B68C1182960204627
:10584000BDE83840ADE700BF28040020094B5A7C72
:1058500082421A4602D8D3F8E800704720B10128E6
:10586000F9D1054B9B6801E0034B5B680B60D2F8F4
:10587000D40070470400002028040020012810B53F
:10588000144605D0022810D00B4BD3F8E00010BD11
:105890000A4B0B4ADB68D0681B681B6A98470030CC
:1058A00018BF01202060002010BD044B044ADB68B3
:1058B00010691B681B6AF1E7040000208C4D020888
:1058C000D02A002038B50B4B0B4D9C782CB1D5F865
:1058D000A03298470124204638BDD5F898322220BE
:1058E00098470028F7D1D5F89832422098470028E9
:1058F000EDD0F0E7341A002028040020022804BF6D
:105900000B4B93F8D10030B90A4BDB681B685B691D
:10591000094A90681847012809D1054B93F8D130FE
:10592000012B04D1034BDB681B689B69F0E77047D0
:10593000040000208C4D0208D02A002070B52D4EA6
:105940002D4DF468636803F5AA7203F1C80003F5EE
:10595000B8732B612368EA60DB68A8609847236806
:10596000E8681B699847236828691B69984763683A
:10597000326903F5377353602049214B0A605A6935
:105980002048C1F89C22D1F8A412C2F80402C2F83F
:105990000C12002111701C4A02201A621B4A587412
:1059A000DA611B4A83F8D0009A611A4A5A621A4A8D
:1059B0009A631A4A5A631A4A9A621A4ADA621A4A65
:1059C0009A641A4A5A641A4A5A651A4A1A651A4A4D
:1059D000DA641A4A5A661A4A1A663222DA604FF4B0
:1059E0008C729A60174A9A65174ADA65BDE870406A
:1059F00084E700BF8C4D0208D02A00202804002034
:105A000004000020C55801083157010899570108C2
:105A10009B5701089F570108EF560108D956010806
:105A2000A357010821580108F95601080557010834
:105A3000195701087D5801084D580108FD58010803
:105A4000255701083D5901084D5A010870B500203D
:105A5000FFF754FF084B094CDD68A0682B689B6872
:105A600098472B68E0689B6898472B6820699B687B
:105A7000BDE87040184700BF8C4D0208D02A0020B6
:105A80002DE9F3411D46C34B5C7C1E468C4205D874
:105A9000D3F8E840204602B0BDE8F0811C2AD3F8D4
:105AA000D44000F0DD8300F2AB800C2A00F08E823F
:105AB0004BD8052A00F00E821AD8022A00F0BB81CA
:105AC00009D8002A00F08381012A00F09A81D6F8D3
:105AD000E0000443DEE7032A00F0CE81042AF6D179
:105AE000002840F0D781AC4B53F821302B60D1E730
:105AF000082A00F0488213D8062A00F00582072AF7
:105B0000E5D1002840F026822020A44B884040F0B8
:105B10001000D3F89832C0B29847C0B22860B9E7F5
:105B20000A2A00F040820B2AD1D10028B2D12020CD
:105B30009A4B884040F01500D3F89832C0B298478D
:105B4000C04300F001002860A4E7122A00F0EA82B6
:105B500029D80F2A00F0A48212D80D2A00F0618201
:105B60000E2AB4D1002840F08D8220208B4B884033
:105B700040F01400D3F89832C0B29847286089E703
:105B8000102A00F0A782112AA1D1002840F0BC827F
:105B90002020824B884040F00800D3F89832C0B2F1
:105BA0009847286076E7152A00F0FE8212D8132A5B
:105BB00000F0D282142A8AD1002840F0E782202007
:105BC000764B884040F00B00D3F89832C0B298472B
:105BD00028605FE7172A00F01B83C0F0FF82182AB5
:105BE0007FF475AF002840F02D8320206B4B884058
:105BF00040F01300D3F89832C0B29847286049E7C4
:105C0000AC2A00F06B8566D8A52A00F00D8433D845
:105C1000A22A00F0A28319D81D2A00F047838C2AFB
:105C20007FF455AF002840F04D8308015B4B40F0F6
:105C30006C00D3F8983200F0FC0098474FF4807362
:105C4000C0F3036043FA00F0286023E7A32A00F0C2
:105C5000AC83A42A7FF43BAF002840F0CD83080139
:105C60004E4B40F06C00D3F8983200F0FC0098479F
:105C7000C0F3003028600DE7A82A00F09D8415D8F5
:105C8000A62A00F02D84A72A7FF421AF002840F037
:105C90007B840801414B40F06C00D3F8983200F04F
:105CA000FC00984700F00F002860F3E6AA2A00F0F5
:105CB000D48440F2A884002840F0F7840801374BD0
:105CC00040F06D00D3F8983200F0FD009847C0F323
:105CD00041102860DEE6B62A00F0C8853FD8B32A16
:105CE00000F063851DD8AD2A00F01F85AE2A7FF431
:105CF000EEAE002840F040850801284B40F06D00D2
:105D0000D3F8983200F0FD009847001410F0400FCF
:105D10000CBF00236FF07F0300F07F0213432B6062
:105D2000B8E6B42A00F06885B52A7FF4D0AE002822
:105D300040F072852020884046B2184F46F014008B
:105D4000D7F89832C0B2984741057FF5A3AE46F028
:105D50001100D7F89832C0B2984728609AE6CE2A48
:105D600000F0E2851CD8B82A00F09C85B92A7FF49F
:105D7000AEAE002840F0BD850801084B40F06C0035
:105D8000D3F8983200F0FC009847C0F30350286025
:105D900080E600BF04000020F02A002080010020DF
:105DA000D22A00F0E085D32A00F0F985D12A7FF4C9
:105DB0008EAE002840F0C8852020AF4B884040F0D0
:105DC0001900D3F89832C0B29847286062E650B9FB
:105DD0002020A94B884040F00D00D3F89832C0B283
:105DE0009847286056E601287FF454AE2020A24B45
:105DF000884040F00D00D3F894322968C0B298472B
:105E000048E650B920209C4B884040F00100D3F870
:105E10009832C0B2984728603CE601287FF43AAE39
:105E20002020954B884040F00100D3F89432296837
:105E3000C0B298472EE650B920208F4B884040F0E2
:105E40000700D3F89832C0B29847286022E60128AC
:105E50007FF420AE01222020884B88405A542A68C3
:105E6000854B82EAE27140F00700D3F89432A1EB4F
:105E7000E271C0B298470DE600287FF40BAE2020F7
:105E80007D4B884040F00200D3F89832C0B298476A
:105E90002860FFE501287FF4FDAD20202B68784ABB
:105EA000002B754FB8BF5B4200FA01F642F8213073
:105EB000F0B2D7F89832984700287FF4EBAD296804
:105EC00046F007000029D7F89432B8BF4942C0B263
:105ED0009847DFE550B92020674B884040F0060026
:105EE000D3F89832C0B298472860D3E501287FF4F0
:105EF000D1AD2020604B884040F00600D3F89432AA
:105F00002968C0B29847C5E560B920205A4B88403F
:105F100040F01000D3F89832C0B29847C0F3072081
:105F20002860B7E501287FF4B5AD20208840524FA6
:105F300040F01006F6B2D7F8983230469847C2B211
:105F40002B780092D7F89052C0F3074200213046D8
:105F5000A8479FE501287FF49DAD20208840464F4B
:105F600040F01006F6B2D7F89832304698472B78B2
:105F7000C0F307420093D7F89052C0F307230021E3
:105F80003046A84786E500287FF484AD20203A4BB0
:105F9000884040F01500D3F89832C0B29847C0F35B
:105FA0004020286076E500287FF474AD2020324B35
:105FB000884040F01500D3F89832C0B2984710F0EE
:105FC000020F0CBF012300232B6063E560B9202082
:105FD000294B884040F01400D3F89832C0B298475B
:105FE000C0F34000286055E501287FF453AD202020
:105FF000884040F01406204FF6B2D7F89832304669
:1060000098472B6833B940F00201D7F894323046F4
:1060100098473FE520F00201D7F894323046984780
:1060200038E560B92020144B884040F01400D3F8C4
:106030009832C0B2984700F0010028602AE5012894
:106040007FF428AD2020884040F014060A4FF6B2B5
:10605000D7F89832304698472B6833B940F00101A1
:10606000D7F894323046984714E520F00101D7F86C
:106070009432304698470DE5800100206C100020D6
:10608000F02A002001287FF405AD2020A44B884091
:1060900040F01400D3F894322968C0B29847F9E46C
:1060A00050B920209E4B884040F00400D3F898322D
:1060B000C0B298472860EDE401287FF4EBAC2020C3
:1060C000974B884040F00400D3F894322968C0B25E
:1060D0009847DFE450B92020914B884040F00500FC
:1060E000D3F89832C0B298472860D3E401287FF4EF
:1060F000D1AC20208A4B884040F00500D3F8943280
:106100002968C0B29847C5E401287FF4C3AC2020B9
:10611000834B884040F00800D3F894322968C0B21D
:106120009847B7E450B920207D4B884040F00A00E2
:10613000D3F89832C0B298472860ABE401287FF4C6
:10614000A9AC2020764B884040F00A00D3F8943266
:106150002968C0B298479DE450B92020704B884010
:1061600040F00300D3F89832C0B29847286091E419
:1061700001287FF48FAC2020694B884040F0030059
:10618000D3F894322968C0B2984783E401287FF499
:1061900081AC2020624B884040F00B00D3F8943251
:1061A0002968C0B2984775E450B920205C4B8840FC
:1061B00040F00C00D3F89832C0B29847286069E4E8
:1061C00001287FF467AC2020554B884040F00C003C
:1061D000D3F894322968C0B298475BE450B92020C4
:1061E0004F4B884040F01100D3F89832C0B2984726
:1061F00028604FE401287FF44DAC2020484B8840B4
:1062000040F01100D3F894322968C0B2984741E4B5
:1062100050B92020424B884040F01200D3F8983209
:10622000C0B29847286035E401287FF433AC2020C1
:106230003B4B884040F01200D3F894322968C0B23A
:10624000984727E401287FF425AC2020344B884070
:1062500040F01300D3F894322968C0B2984719E48B
:1062600060B908012E4B40F06C00D3F8983200F072
:10627000FC009847C0F3804028600BE401287FF4BD
:1062800009AC080140F06C06254FF6B2D7F89832F9
:10629000304698472B6820F480210BB141F48021CF
:1062A000D7F8943230469847FFF7F4BB00287FF4C4
:1062B000F1AB1B4A53689268002918BF13462B6044
:1062C000FFF7E8BB01287FF4E5AB2B68102B23D048
:1062D0000DDC022B1CD004DC012B16D04FF0FF3359
:1062E00014E0042B16D0082BF8D105230EE0402B28
:1062F00014D003DC202BF1D1032307E0802B11D035
:10630000B3F5807FEAD1002300E008232B600AE088
:106310000723FBE70623F9E70423F7E70223F5E762
:106320008001002028602B6801333FF4B3AB0801E3
:10633000BC4F40F06C06F6B2D7F89832304698471A
:106340002B6820F070611B0603F07063D7F894226D
:10635000194330469047FFF79DBB68B90801B14B20
:1063600040F06C00D3F8983200F0FC009847C0F37E
:10637000C1302860FFF78EBB01287FF48BAB08018A
:10638000A84F40F06C06F6B2D7F8983230469847DE
:106390002B6820F4C031DB0303F4C033D7F8942218
:1063A000194330469047FFF775BB68B908019D4B0C
:1063B00040F06C00D3F8983200F0FC009847C0F32E
:1063C00080302860FFF766BB01287FF463AB0801CB
:1063D00040F06C06934FF6B2D7F8983230469847A3
:1063E0002B6820F480410BB141F48041D7F89432FE
:1063F00030469847FFF74EBB01287FF44BAB0801AE
:1064000040F06C06874FF6B2D7F89832304698477E
:106410002B6820F480510BB141F48051D7F89432AD
:1064200030469847FFF736BB20BB080140F06C06AA
:106430007C4FF6B2D7F898323046984710F4804F28
:10644000D7F89832304605D09847C0F3C31028607B
:10645000FFF720BB9847D7F89832804630469847D8
:1064600018F4006FC0F3021018BF40F00800286055
:10647000FFF710BB01287FF40DAB080140F06C065C
:10648000684FF6B2D7F898323046984710F4804FEC
:1064900010D0D7F89832304698472B6820F4F06136
:1064A000DB0103F4F063D7F8942219433046904798
:1064B000FFF7F0BAD7F89832304698472968D7F8EE
:1064C00094320D074CBF40F4006020F400600901D5
:1064D00020F07000C9B2014330469847FFF7DABA9E
:1064E00020BB080140F06C064E4FF6B2D7F8983248
:1064F0003046984710F4804FD7F89832304605D090
:106500009847C0F302102860FFF7C4BA9847D7F83D
:10651000983280463046984718F4006FC0F3C31095
:1065200018BF40F008002860FFF7B4BA01287FF4D4
:10653000B1AA080140F06C063A4FF6B2D7F898328B
:106540003046984710F4804FD7F8983230460DD037
:1065500098472B6820F070011B0103F07003D7F8F7
:106560009422194330469047FFF794BA98472B6816
:1065700020F4F061DB0103F4F063D7F894221943AF
:1065800030469047FFF786BA01287FF483AA0801B6
:10659000244F40F06C06F6B2D7F898323046984750
:1065A0002B6820F00F0103F00F03D7F89422194352
:1065B00030469047FFF76EBA68B90801194B40F0B2
:1065C0006D00D3F8983200F0FD009847C0F3C0305A
:1065D0002860FFF75FBA01287FF45CAA080140F049
:1065E0006D06104FF6B2D7F89832304698472B68B0
:1065F00020F400410BB141F40041D7F89432304609
:106600009847FFF747BA78B90801064B40F06D008C
:10661000D3F8983200F0FD009847C0F3413028606D
:10662000FFF738BA8001002001287FF433AA08015F
:10663000BC4F40F06D06F6B2D7F898323046984716
:106640002B6820F4C0415B0303F4C043D7F89422C5
:10665000194330469047FFF71DBA68B90801B14B9E
:1066600040F06D00D3F8983200F0FD009847C0F379
:1066700003202860FFF70EBA01287FF40BAA080157
:10668000A84F40F06D06F6B2D7F8983230469847DA
:106690002B6820F470611B0203F47063D7F8942216
:1066A000194330469047FFF7F5B901287FF4F2A966
:1066B00008019C4F40F06D06F6B2D7F8983230468C
:1066C00098472B6820F060015B0103F06003D7F866
:1066D0009422194330469047FFF7DCB968B90801A6
:1066E000904B40F06D00D3F8983200F0FD009847D1
:1066F00000F00F002860FFF7CDB901287FF4CAA988
:106700000801884F40F06D06F6B2D7F8983230464F
:1067100098472B6820F00F0103F00F03D7F894225D
:10672000194330469047FFF7B5B968B908017D4B6A
:1067300040F06D00D3F8983200F0FD009847C0F3A8
:1067400000602860FFF7A6B901287FF4A3A908011B
:1067500040F06D06734FF6B2D7F89832304698473E
:106760002B6820F080710BB141F08071D7F8943222
:1067700030469847FFF78EB901287FF48BA90801AE
:10678000684F40F06D06F6B2D7F898323046984719
:106790002B6820F4FE011B0403F4FE03D7F89422B7
:1067A000194330469047FFF775B968B908015D4B4A
:1067B00040F06C00D3F8983200F0FC009847C0F32A
:1067C00040402860FFF766B901287FF463A90801FB
:1067D00040F06C06534FF6B2D7F8983230469847DF
:1067E0002B6820F400310BB141F40031D7F894321A
:1067F00030469847FFF74EB900287FF44BA90801AF
:10680000484B40F06F00D3F89832C0B29847C0F3BD
:1068100007402860FFF73EB901287FF43BA92020FC
:106820008840404F46B246F0110046F014062968F1
:10683000F6B2D7F89432C0B29847D7F898323046BB
:10684000984720F480684146D7F8943230469847FC
:106850002B683046002B0CBF00214FF48061D7F825
:10686000943241EA08019847FFF714B958B920203B
:106870002C4B884040F01100D3F89832C0B29847B2
:106880002860FFF707B901287FF404A92020254BD1
:10689000884040F01100D3F894322968C0B298477C
:1068A000FFF7F8B868B908011E4B40F06C00D3F848
:1068B000983200F0FC009847C0F340302860FFF7A2
:1068C000E9B801287FF4E6A8080140F06C06154FEE
:1068D000F6B2D7F89832304698472B6820F400512A
:1068E0000BB141F40051D7F8943230469847FFF786
:1068F000D1B801287FF4CEA808010A4F40F06C06F9
:10690000F6B2D7F89832304698472B6820F47001D9
:106910001B0503F47003D7F89422194330469047BF
:10692000FFF7B8B88001002000287FF4B3A8080161
:10693000444B40F06F00D3F89832C0B29847C0F390
:1069400009002860FFF7A6B801287FF4A3A820203B
:106950003C4B884040F01900D3F894322968C0B20B
:106960009847FFF797B858B92020364B884040F039
:106970001A00D3F89832C0B298472860FFF78AB857
:1069800001287FF487A820202E4B884040F01A0071
:10699000D3F894322968C0B29847FFF77BB8F0B9B2
:1069A00079B101297FF476A8264BD3F8983298471D
:1069B00000F06000A0F12003584258412860FFF722
:1069C00069B8204B0846D3F89832984700F0180071
:1069D000A0F11002504250412860FFF75BB8012837
:1069E0007FF458A899B101297FF454A8154E0020CE
:1069F000D6F8983298472B68FBB120F0400141F05F
:106A00002001D6F8943200209847FFF743B80D4E86
:106A10000846D6F8983298472B684BB120F0080109
:106A200041F01001D6F8943200209847FFF732B8B1
:106A300020F0100141F00801F4E720F0200141F0BE
:106A40004001DEE78001002007B502AB43F8042DCA
:106A500002460120FFF714F803B05DF804FB13466B
:106A600002460020FFF70CB8014BD3F894321847C8
:106A700080010020034B10B5D3F898320C4698479C
:106A8000206010BD80010020014BD3F88C321847E4
:106A9000800100200022014B5A6070470400002052
:106AA0002DE9F341154B06465A7C884682421F4623
:106AB00004D8D3F8E80002B0BDE8F0812024104DDE
:106AC000844044F0070081EAE171D5F89432A1EBEB
:106AD000E871C0B2984701230A4AB8F1000F9355F4
:106AE000B8BF022300930023E0B21A46D5F89042C3
:106AF0001946A047D7F8D400DDE700BF0400002006
:106B0000800100206C100020CAE74942C8E700213C
:106B1000C6E72DE9F3411A4B04465A7C0F468242E0
:106B20001E4604D8D3F8E80002B0BDE8F081DFF8D3
:106B30005C80144D18F800306BB12020124AA04040
:106B400040F00700D5F8943252F82410C0B29847AC
:106B5000002308F80430202303FA04F444F00D0065
:106B6000D5F894323946C0B2984700230093E0B27A
:106B7000D5F890521A461946A847D6F8D400D3E75C
:106B80000400002080010020F02A00206C1000206A
:106B900038B504462020084BA0400D4640F00100C7
:106BA000D3F89832C0B298472B68C11829602046A4
:106BB000BDE83840ADE700BF80010020094B5A7C9A
:106BC00082421A4602D8D3F8E800704720B1012863
:106BD000F9D1054B9B6801E0034B5B680B60D2F871
:106BE000D40070470400002080010020012810B567
:106BF000144613D005D302281CD0124BD3F8E00062
:106C000010BD1468104A114BD268126824B1526941
:106C100058699047002010BD9269F9E70A4B0B4A6A
:106C2000DB68D0681B681B6A9847003018BF0120DA
:106C30002060EFE7044B054ADB6810691B681B6A9C
:106C4000F2E700BF040000208C4D0208F02A00206B
:106C500038B50B4B0B4D9C782CB1D5F8A03298472A
:106C60000124204638BDD5F89832222098470028C4
:106C7000F7D1D5F89832422098470028EDD0F0E7B8
:106C8000341A002080010020022804BF0B4B93F827
:106C9000D10030B90A4BDB681B685B69094A906810
:106CA0001847012809D1054B93F8D130012B04D1A5
:106CB000034BDB681B689B69F0E77047040000200A
:106CC0008C4D0208F02A002070B53D4E3D4CF56811
:106CD0006B6803F5AA72E26003F5B872226103F5EE
:106CE0006F72626103F5767203F1C800A26103F569
:106CF0007D7203F5826323622B68E261DB68A0602A
:106D000098472B686069DB6898472B6860699B69C6
:106D100098472B68E0681B6998472B6820691B69B6
:106D200098472B68206A1B6998472B68A0691B69E4
:106D300098472B68E0691B6998476B68326903F5CF
:106D4000377353602049214B0A605A692048C1F8C3
:106D50009C22D1F8A412C2F80402C2F80C1200213D
:106D600011701C4A32211A621B4AD960DA611B4A2F
:106D7000DE219A611A4A99605A621A4A01209A637E
:106D8000194A5A63194A9A62194ADA62194A9A6484
:106D9000194A5A64194A5A65194A1A65194ADA642D
:106DA000194A5A66194A1A6602225A7483F8D02080
:106DB000174A9A65174ADA65BDE8704064E700BF74
:106DC0008C4D0208F02A00208001002004000020E1
:106DD000516C0108A16A0108096B01080B6B0108DD
:106DE0000F6B01085F6A0108496A0108136B01080B
:106DF000916B0108696A0108756A0108896A0108CE
:106E0000ED6B0108BD6B0108896C0108956A0108EA
:106E1000C96C0108196E010870B50020FFF734FF36
:106E2000104B114CDD68A0682B689B6898472B6855
:106E3000E0689B6898472B6820699B6898472B6897
:106E4000206A9B6898472B68A0699B6898472B68C5
:106E5000E0699B6898472B6860699B68BDE8704053
:106E6000184700BF8C4D0208F02A00202DE9F3419D
:106E70001D46C64B5C7C1E468C4205D8D3F8E840C4
:106E8000204602B0BDE8F0811C2AD3F8D44000F0BF
:106E9000D18300F2AB800C2A00F07D824BD8052A0A
:106EA00000F0FD811AD8022A00F0AA8109D8002A30
:106EB00000F07281012A00F08981D6F8E0000443D5
:106EC000DEE7032A00F0BD81042AF6D1002840F055
:106ED000C681AF4B53F821302B60D1E7082A00F070
:106EE000378213D8062A00F0F481072AE5D100285A
:106EF00040F015822020A74B884040F01000D3F8C6
:106F00009832C0B29847C0B22860B9E70A2A00F0A8
:106F10002F820B2AD1D10028B2D120209D4B88404E
:106F200040F01500D3F89832C0B29847C04300F043
:106F300001002860A4E7122A00F0DE8229D80F2A77
:106F400000F0988212D80D2A00F053820E2AB4D194
:106F5000002840F07A8220208E4B884040F01400B8
:106F6000D3F89832C0B29847286089E7102A00F019
:106F70009B82112AA1D1002840F0B0822020854BAD
:106F8000884040F00800D3F89832C0B29847286093
:106F900076E7152A00F0F28212D8132A00F0C68292
:106FA000142A8AD1002840F0DB822020794B8840C7
:106FB00040F00B00D3F89832C0B2984728605FE7E2
:106FC000172A00F00F83C0F0F382182A7FF475AF00
:106FD000002840F0218320206E4B884040F01300B1
:106FE000D3F89832C0B29847286049E7AB2A00F03E
:106FF000368567D8A52A00F0008433D8A22A00F08D
:10700000958319D81D2A00F03A838C2A7FF455AF56
:10701000002840F0408308015E4B40F06C00D3F83C
:10702000983200F0FC0098474FF48073C0F303607F
:1070300043FA00F0286023E7A32A00F09F83A42AE4
:107040007FF43BAF002840F0C0830801514B40F073
:107050006C00D3F8983200F0FC009847C0F3003081
:1070600028600DE7A82A00F0908415D8A62A00F021
:107070002084A72A7FF421AF002840F06E84080105
:10708000444B40F06C00D3F8983200F0FC00984775
:1070900000F00F002860F3E6A92A00F09D84AA2AD8
:1070A0007FF40BAF002840F0C1840801394B40F059
:1070B0006D00D3F8983200F0FD009847C0F303202C
:1070C0002860DDE6B52A00F088852ED8AE2A00F0CB
:1070D0002D8515D8AC2A00F0EA84AD2A7FF4EDAEF8
:1070E000002840F00B8508012A4B40F06D00D3F8D2
:1070F000983200F0FD009847C0F300602860BFE6BA
:10710000B32A00F04385B42A7FF4D7AE00287FF479
:10711000B7AE08011F4B40F06F00D3F89832C0B2F1
:107120009847C0F307402860AAE6CE2A00F0CD8534
:1071300015D8B62A00F09585B82A7FF4BEAE00288F
:1071400040F0AB850801134B40F06C00D3F8983247
:1071500000F0FC009847C0F34030286090E6D22A47
:1071600000F0D285D32A00F0EE85D12A7FF4A5AEB7
:10717000002840F0BA852020064B884040F01900D6
:10718000D3F89832C0B29847286079E6040000200E
:10719000202B00202804002050B92020B24B88402A
:1071A00040F00D00D3F89832C0B29847286067E6E7
:1071B00001287FF465AE2020AB4B884040F00D00E5
:1071C000D3F894322968C0B2984759E650B92020C4
:1071D000A54B884040F00100D3F89832C0B29847E0
:1071E00028604DE601287FF44BAE20209E4B88405E
:1071F00040F00100D3F894322968C0B298473FE6C6
:1072000050B92020984B884040F00700D3F89832BE
:10721000C0B29847286033E601287FF431AE0122DE
:107220002020924B88405A542A688F4B82EAE271A0
:1072300040F00700D3F89432A1EBE271C0B2984756
:107240001EE600287FF41CAE2020874B884040F0CB
:107250000200D3F89832C0B29847286010E601289F
:107260007FF40EAE20202B68814A002B7E4FB8BFE2
:107270005B4200FA01F642F82130F0B2D7F89832BA
:10728000984700287FF4FCAD296846F007000029E4
:10729000D7F89432B8BF4942C0B29847F0E550B928
:1072A0002020714B884040F00600D3F89832C0B2DD
:1072B00098472860E4E501287FF4E2AD20206A4B7E
:1072C000884040F00600D3F894322968C0B298474D
:1072D000D6E560B92020644B884040F01000D3F818
:1072E0009832C0B29847C0F307202860C8E501284B
:1072F0007FF4C6AD202088405B4F40F01006F6B208
:10730000D7F8983230469847C2B22B780092D7F817
:107310009052C0F3074200213046A847B0E501284B
:107320007FF4AEAD202088404F4F40F01006F6B2FB
:10733000D7F89832304698472B78C0F3074200932D
:10734000D7F89052C0F3072300213046A84797E5AD
:1073500000287FF495AD2020434B884040F0150075
:10736000D3F89832C0B29847C0F34020286087E530
:1073700000287FF485AD20203B4B884040F015006D
:10738000D3F89832C0B2984710F0020F0CBF012317
:1073900000232B6074E560B92020334B884040F017
:1073A0001400D3F89832C0B29847C0F34000286068
:1073B00066E501287FF464AD202088402A4F40F024
:1073C0001406F6B2D7F89832304698472B6820F06A
:1073D0000A00002B0CBF00210221022B40EA010011
:1073E00014BF00210821D7F8943201433046984752
:1073F00046E560B920201C4B884040F01400D3F8CB
:107400009832C0B2984700F00100286038E50128A2
:107410007FF436AD20208840134F40F01406F6B2BA
:10742000D7F89832304698472B6820F00500002B9B
:1074300018BF40F00100022B14BF00210421D7F82F
:1074400094320143304698471AE501287FF418AD7D
:107450002020054B884040F01400D3F8943229686E
:10746000C0B298470CE500BF28040020741000202B
:10747000202B002050B92020AB4B884040F0040066
:10748000D3F89832C0B298472860F9E401287FF415
:10749000F7AC2020A44B884040F00400D3F894328D
:1074A0002968C0B29847EBE450B920209E4B884031
:1074B00040F00500D3F89832C0B298472860DFE466
:1074C00001287FF4DDAC2020974B884040F0050078
:1074D000D3F894322968C0B29847D1E401287FF4E8
:1074E000CFAC2020904B884040F00800D3F8943275
:1074F0002968C0B29847C3E450B920208A4B88401D
:1075000040F00A00D3F89832C0B298472860B7E438
:1075100001287FF4B5AC2020834B884040F00A005E
:10752000D3F894322968C0B29847A9E450B9202012
:107530007D4B884040F00300D3F89832C0B29847A2
:1075400028609DE401287FF49BAC2020764B884086
:1075500040F00300D3F894322968C0B298478FE412
:1075600001287FF48DAC20206F4B884040F00B0049
:10757000D3F894322968C0B2984781E450B92020EA
:10758000694B884040F00C00D3F89832C0B298475D
:10759000286075E401287FF473AC2020624B88409A
:1075A00040F00C00D3F894322968C0B2984767E4E1
:1075B00050B920205C4B884040F01100D3F898323D
:1075C000C0B2984728605BE401287FF459AC2020C2
:1075D000554B884040F01100D3F894322968C0B26E
:1075E00098474DE450B920204F4B884040F012009E
:1075F000D3F89832C0B29847286041E401287FF45C
:107600003FAC2020484B884040F01200D3F8943221
:107610002968C0B2984733E401287FF431AC2020B8
:10762000414B884040F01300D3F894322968C0B22F
:10763000984725E460B908013B4B40F06C00D3F853
:10764000983200F0FC009847C0F38040286017E4AF
:1076500001287FF415AC080140F06C06324FF6B2F9
:10766000D7F89832304698472B6820F480210BB128
:1076700041F48021D7F894323046984700E400283E
:107680007FF4FEAB284A53689268002918BF13465E
:107690002B60FFF7F5BB01287FF4F2AB2B68102BB2
:1076A00023D00DDC022B1CD004DC012B16D04FF0B4
:1076B000FF3314E0042B16D0082BF8D105230EE07D
:1076C000402B14D003DC202BF1D1032307E0802BC7
:1076D0000FD0B3F5807FEAD1002300E008232B60B0
:1076E00008E00723FBE70623F9E70423F7E7022373
:1076F000F5E728602B6801333FF4C2AB08010A4F5D
:1077000040F06C06F6B2D7F89832304698472B68AE
:1077100020F070611B0603F07063D7F894221943C0
:1077200030469047FFF7ACBB2804002068B9080139
:10773000BD4B40F06C00D3F8983200F0FC00984745
:10774000C0F3C1302860FFF79BBB01287FF498ABE2
:107750000801B54F40F06C06F6B2D7F898323046C3
:1077600098472B6820F4C031DB0303F4C033D7F80B
:107770009422194330469047FFF782BB68B908014D
:10778000A94B40F06C00D3F8983200F0FC00984709
:10779000C0F380302860FFF773BB01287FF470AB23
:1077A000080140F06C06A04FF6B2D7F89832304688
:1077B00098472B6820F480410BB141F48041D7F801
:1077C000943230469847FFF75BBB01287FF458ABF3
:1077D000080140F06C06944FF6B2D7F89832304664
:1077E00098472B6820F480510BB141F48051D7F8B1
:1077F000943230469847FFF743BB20BB080140F066
:107800006C06894FF6B2D7F898323046984710F494
:10781000804FD7F89832304605D09847C0F3C31050
:107820002860FFF72DBB9847D7F89832804630463E
:10783000984718F4006FC0F3021018BF40F008001A
:107840002860FFF71DBB01287FF41AAB080140F048
:107850006C06754FF6B2D7F898323046984710F458
:10786000804F10D0D7F89832304698472B6820F4D4
:10787000F061DB0103F4F063D7F89422194330463A
:107880009047FFF7FDBAD7F89832304698472968F5
:10789000D7F894320D074CBF40F4006020F400602C
:1078A000090120F07000C9B2014330469847FFF744
:1078B000E7BA20BB080140F06C065B4FF6B2D7F880
:1078C00098323046984710F4804FD7F898323046B7
:1078D00005D09847C0F302102860FFF7D1BA984747
:1078E000D7F8983280463046984718F4006FC0F3B6
:1078F000C31018BF40F008002860FFF7C1BA012884
:107900007FF4BEAA080140F06C06474FF6B2D7F8E4
:1079100098323046984710F4804FD7F89832304666
:107920000DD098472B6820F070011B0103F0700305
:10793000D7F89422194330469047FFF7A1BA9847E9
:107940002B6820F4F061DB0103F4F063D7F8942294
:10795000194330469047FFF793BA01287FF490AA65
:107960000801314F40F06C06F6B2D7F89832304635
:1079700098472B6820F00F0103F00F03D7F89422EB
:10798000194330469047FFF77BBA68B90801264B88
:1079900040F06D00D3F8983200F0FD009847C0F336
:1079A000C0302860FFF76CBA01287FF469AA08018B
:1079B00040F06D061C4FF6B2D7F898323046984723
:1079C0002B6820F400410BB141F40041D7F8943208
:1079D00030469847FFF754BA68B90801124B40F097
:1079E0006D00D3F8983200F0FD009847C0F34130A5
:1079F0002860FFF745BA01287FF442AA08010A4F20
:107A000040F06D06F6B2D7F89832304698472B68AA
:107A100020F4C0415B0303F4C043D7F89422194318
:107A200030469047FFF72CBA2804002001287FF445
:107A300027AA0801BB4F40F06D06F6B2D7F898327E
:107A4000304698472B6820F470611B0203F4706382
:107A5000D7F89422194330469047FFF711BA68B916
:107A60000801B04B40F06D00D3F8983200F0FD00F3
:107A70009847C0F341102860FFF702BA01287FF44D
:107A8000FFA90801A74F40F06D06F6B2D7F898326B
:107A9000304698472B6820F060015B0103F06003DB
:107AA000D7F89422194330469047FFF7E9B968B9EF
:107AB00008019C4B40F06D00D3F8983200F0FD00B7
:107AC000984700F00F002860FFF7DAB901287FF42B
:107AD000D7A90801934F40F06D06F6B2D7F8983257
:107AE000304698472B6820F00F0103F00F03D7F8BA
:107AF0009422194330469047FFF7C2B901287FF41A
:107B0000BFA9080140F06D06864FF6B2D7F898324B
:107B1000304698472B6820F080710BB141F080719E
:107B2000D7F8943230469847FFF7AAB9A8B90801A8
:107B30007C4B40F06D00D3F8983200F0FD00984780
:107B4000001410F0400F0CBF00236FF07F0300F013
:107B50007F0213432B60FFF793B901287FF490A9AC
:107B60000801704F40F06D06F6B2D7F898323046F3
:107B700098472B6820F4FE011B0403F4FE03D7F89A
:107B80009422194330469047FFF77AB968B9080143
:107B9000644B40F06C00D3F8983200F0FC0098473A
:107BA000C0F340402860FFF76BB901287FF468A953
:107BB000080140F06C065B4FF6B2D7F898323046B9
:107BC00098472B6820F400310BB141F40031D7F80D
:107BD000943230469847FFF753B9C0B92020884007
:107BE00046B2504F46F01400D7F89832C0B29847CA
:107BF00010F4806008D046F01100D7F89832C0B277
:107C000098472860FFF73CB92860FFF739B9012889
:107C10007FF436A920208840424F46B246F011003A
:107C200046F014062968F6B2D7F89432C0B29847E5
:107C3000D7F898323046984720F480684146D7F804
:107C40009432304698472B683046002B0CBF0021F9
:107C50004FF48061D7F8943241EA08019847FFF762
:107C60000FB958B920202F4B884040F01100D3F8AD
:107C70009832C0B298472860FFF702B901287FF414
:107C8000FFA82020274B884040F01100D3F8943201
:107C90002968C0B29847FFF7F3B801287FF4F0A82D
:107CA000080140F06C061F4FF6B2D7F89832304604
:107CB00098472B6820F400510BB141F40051D7F8DC
:107CC000943230469847FFF7DBB800287FF4D8A8F5
:107CD0000801144B40F06F00D3F89832C0B29847B7
:107CE000C0F309002860FFF7CBB801287FF4C8A8CB
:107CF00020200C4B884040F01900D3F894322968BA
:107D0000C0B29847FFF7BCB870B92020054B884037
:107D100040F01A00D3F89832C0B298472860FFF7B5
:107D2000AFB800BF2804002001287FF4A9A82020B4
:107D30002E4B884040F01A00D3F894322968C0B224
:107D40009847FFF79DB8F0B979B101297FF498A859
:107D5000264BD3F89832984700F06000A0F120033A
:107D6000584258412860FFF78BB8204B0846D3F89B
:107D70009832984700F01800A0F11002504250418C
:107D80002860FFF77DB801287FF47AA899B101290E
:107D90007FF476A8154E0020D6F8983298472B68C5
:107DA000FBB120F0400141F02001D6F894320020D0
:107DB0009847FFF765B80D4E0846D6F898329847B1
:107DC0002B684BB120F0080141F01001D6F8943235
:107DD00000209847FFF754B820F0100141F0080147
:107DE000F4E720F0A00141F04001DEE72804002084
:107DF00007B502AB43F8042D02460120FFF736F821
:107E000003B05DF804FB134602460020FFF72EB8CE
:107E1000014BD3F89432184728040020034B10B5C7
:107E2000D3F898320C469847206010BD28040020F3
:107E3000014BD3F88C321847280400200022014B54
:107E40005A607047040000202DE9F341154B0646A7
:107E50005A7C884682421F4604D8D3F8E80002B014
:107E6000BDE8F0812024104D844044F0070081EAF1
:107E7000E171D5F89432A1EBE871C0B298470123C3
:107E80000A4AB8F1000F9355B8BF022300930023AC
:107E9000E0B21A46D5F890421946A047D7F8D40068
:107EA000DDE700BF0400002028040020741000203B
:107EB000CAE74942C8E70021C6E72DE9F3411A4B5A
:107EC00004465A7C0F4682421E4604D8D3F8E80086
:107ED00002B0BDE8F081DFF85C80144D18F8003086
:107EE0006BB12020124AA04040F00700D5F8943230
:107EF00052F82410C0B29847002308F80430202319
:107F000003FA04F444F00D00D5F894323946C0B2B7
:107F1000984700230093E0B2D5F890521A461946CC
:107F2000A847D6F8D400D3E7040000202804002096
:107F3000202B00207410002038B504462020084B68
:107F4000A0400D4640F00100D3F89832C0B29847E7
:107F50002B68C11829602046BDE83840ADE700BF56
:107F600028040020094B5A7C82421A4602D8D3F8D2
:107F7000E800704720B10128F9D1054B9B6801E06A
:107F8000034B5B680B60D2F8D400704704000020FC
:107F900028040020012810B5144613D005D3022868
:107FA0001CD0124BD3F8E00010BD1468104A114BDE
:107FB000D268126824B1526958699047002010BDF8
:107FC0009269F9E70A4B0B4ADB68D0681B681B6AA9
:107FD0009847003018BF01202060EFE7044B054AA6
:107FE000DB6810691B681B6AF2E700BF0400002011
:107FF0008C4D0208202B002038B50B4B0B4D9C7884
:108000002CB1D5F8A03298470124204638BDD5F8C8
:108010009832222098470028F7D1D5F8983242208C
:1080200098470028EDD0F0E7341A002028040020FB
:10803000022804BF0B4B93F8D10030B90A4BDB6820
:108040001B685B69094A90681847012809D1054BEC
:1080500093F8D130012B04D1034BDB681B689B697B
:10806000F0E77047040000208C4D0208202B002010
:1080700070B53D4E3D4CF5686B6803F5AA72E26041
:1080800003F5B872226103F56F72626103F57672CF
:1080900003F1C800A26103F57D7203F582632362D8
:1080A0002B68E261DB68A06098472B686069DB6839
:1080B00098472B6860699B6998472B68E0681B6943
:1080C00098472B6820691B6998472B68206A1B69B1
:1080D00098472B68A0691B6998472B68E0691B6962
:1080E00098476B68326903F5377353602049214B19
:1080F0000A605A692048C1F89C22D1F8A412C2F83B
:108100000402C2F80C12002111701C4A02201A62EB
:108110001B4A5874DA611B4A83F8D0009A611A4AE4
:108120005A621A4A9A631A4A5A631A4A9A621A4A4D
:10813000DA621A4A9A641A4A5A641A4A5A651A4AF8
:108140001A651A4ADA641A4A5A661A4A1A663222B2
:10815000DA604FF48C729A60174A9A65174ADA65AA
:10816000BDE8704064E700BF8C4D0208202B002062
:108170002804002004000020F97F0108497E01083E
:10818000B17E0108B37E0108B77E0108077E0108B1
:10819000F17D0108BB7E0108397F0108117E0108CD
:1081A0001D7E0108317E0108957F0108657F010869
:1081B000318001083D7E010871800108C1810108FC
:1081C00070B50020FFF734FF104B114CDD68A0683C
:1081D0002B689B6898472B68E0689B6898472B68DA
:1081E00020699B6898472B68206A9B6898472B6892
:1081F000A0699B6898472B68E0699B6898472B6843
:1082000060699B68BDE87040184700BF8C4D02084C
:10821000202B00202DE9F3410F4606461D46C1499B
:108220002FB1D1F8E840204602B0BDE8F0818C2A99
:10823000D1F8D44000F09D8300F2A1800E2A00F016
:10824000728245D8062A00F0DA811CD8022A00F092
:108250008B8109D8002A00F05D81012A00F072812B
:10826000D1F8E0000443DEE7042A00F09F8140F2E9
:108270009381002840F0B981AB4B2620D3F894328B
:1082800098472860CFE70A2A00F0F7810FD8072A1D
:1082900000F0D481082AE3D10028C4D1A24B3520B4
:1082A000D3F894329847C0F340202860BBE70C2AEB
:1082B00000F0FF8140F2F081002840F01C829A4BD0
:1082C0003420D3F89432984700F001002860AAE7E0
:1082D000152A00F09D8221D8112A00F052820ED872
:1082E0000F2A00F03282102ABAD1002840F03F82D3
:1082F0008D4B2520D3F894329847286093E7132AB2
:1083000000F06A8240F24F82002840F07782864B6C
:108310002B20D3F894329847286084E71C2A00F079
:10832000CF821CD8182A00F09C821B2A00F0AB8256
:10833000172A95D1002840F07D827B4B1520D3F879
:10834000943298474FF08073002808BF0120B3FB98
:10835000F0F0764B984294BF28602B6063E7212AA7
:1083600000F0CB82222A00F0E6821D2A7FF478AF4B
:1083700000287FF458AF6C4B5B682B6053E7B32A3F
:1083800000F021855CD8A82A00F0548426D8A42ABD
:1083900000F07C8311D8A22A00F04083A32A7FF446
:1083A0005FAF002840F05A835F4B6C20D3F89432C3
:1083B0009847C0F38030286035E7A62A00F0D983BB
:1083C00040F28383002840F02184574B6C20D3F87F
:1083D0009432984700F00F00286024E7AB2A00F0A1
:1083E0007D8411D8A92A00F04484AA2A7FF438AFEA
:1083F000002840F05E844C4B6D20D3F894329847AF
:10840000C0F3032028600EE7AD2A00F0A684C0F078
:108410008584AE2A7FF424AF002840F0BF84424B0D
:108420006D20D3F894329847001410F0400F0CBF21
:1084300000236FF07F0300F07F0213432B60F2E60E
:10844000BB2A00F0A78538D8B62A00F0178520D8B7
:10845000B42A00F0D784B52A7FF402AF002840F098
:10846000DE84314F3420D7F89432984743050ED537
:10847000D7F89432142098474FF08076002808BF30
:108480000120B6FBF0F62948864228BF06462E603A
:10849000C9E6B92A00F0328500F25085B82A7FF487
:1084A000DFAE002840F016851F4B6C20D3F89432C5
:1084B0009847C0F340302860B5E6CC2A00F0078624
:1084C00013D8BF2A00F0AA85C02A00F0D185BC2AA3
:1084D0007FF4C6AE002840F08D85134B7020D3F892
:1084E00094329847C0B228609DE6D12A00F01186E8
:1084F000D22A00F02286CE2A7FF4B2AE00287FF482
:1085000092AE094B6F20D3F894329847C0F309001C
:10851000286088E660B9044B2D20D3F89432984740
:10852000286080E604000020100A0020FFFF0F00F2
:1085300001287FF478AEA54B2968D3F890322D201E
:10854000984770E630B9A14B2120D3F89432984770
:10855000286068E601287FF466AE9C4B2968D3F852
:108560009032212098475EE630B9984B2720D3F807
:1085700094329847286056E601287FF454AE196873
:10858000924B0029D3F89032B8BF49422720984730
:1085900001228F4B1A6046E600287FF444AE8B4BD5
:1085A0002220D3F89432984728603CE618B9894BCA
:1085B0001B682B6037E601287FF435AE1B68854ABF
:1085C000002B824EB8BF5B4213602020D6F8943255
:1085D000984700287FF427AE2968D6F89032002902
:1085E000B8BF4942272098471DE601287FF41BAEFB
:1085F000764B2968D3F890322620984713E640B985
:10860000724B1020D3F894329847C0F304202860AE
:1086100009E601287FF407AE6C4E1020D6F894329C
:1086200098472B68C2B20092D6F88C52C0F307422A
:1086300003F01F0339461020A847F4E538B9634B0F
:108640001020D3F894329847C0B22860EBE5012897
:108650007FF4E9AD5D4E1020D6F8943298472B6830
:10866000C0F3074203F01F030093D6F88C52C0F307
:10867000072300211020A847D5E500287FF4D3ADBB
:10868000524B3520D3F89432984710F0020F0CBFAC
:10869000012300232B60C6E500287FF4C4AD4B4BBB
:1086A0003520D3F894329847C04300F00100286089
:1086B000B9E540B9454B3420D3F894329847C0F31C
:1086C00040002860AFE501287FF4ADAD3F4E342077
:1086D000D6F8943298472B6833B940F00201D6F8A7
:1086E0009032342098479EE520F00201D6F890326F
:1086F0003420984797E501287FF495AD334E342018
:10870000D6F8943298472B6833B940F00101D6F877
:1087100090323420984786E520F00101D6F8903257
:10872000342098477FE530B9284B3420D3F8943271
:108730009847286077E501287FF475AD234B2968B9
:10874000D3F89032342098476DE530B91F4B242080
:10875000D3F894329847286065E501287FF463AD2B
:108760001A4B2968D3F89032242098475BE50128FA
:108770007FF459AD154B2968D3F8903225209847DE
:1087800051E530B9114B2820D3F89432984728602E
:1087900049E501287FF447AD0C4B2968D3F89032A6
:1087A000282098473FE530B9084B2A20D3F8943267
:1087B0009847286037E501287FF435AD034B2968D9
:1087C000D3F890322A2098472DE500BF100A0020E8
:1087D000502B00207C10002030B9AA4B2320D3F866
:1087E0009432984728601EE501287FF41CADA54B04
:1087F0002968D3F890322320984714E501287FF4A4
:1088000012ADA04B2968D3F890322B2098470AE587
:1088100030B99C4B2C20D3F894329847286002E55D
:1088200001287FF400AD974B2968D3F890322C20B3
:108830009847F8E401287FF4F6AC1B684FF0807687
:10884000002B08BF0123B6FBF3F68F4B15209E4289
:1088500028BF1E468B4B3146D3F8903298472E6086
:10886000E1E430B9874B3320D3F89432984728603D
:10887000D9E401287FF4D7AC824B2968D3F8903231
:1088800033209847CFE440B97E4B6C20D3F8943224
:108890009847C0F3C0402860C5E401287FF4C3AC0A
:1088A000784E6C20D6F8943298472B6820F400213B
:1088B0000BB141F40021D6F890326C209847B2E415
:1088C00040B9704B6C20D3F894329847C0F3804085
:1088D0002860A8E401287FF4A6AC6A4E6C20D6F884
:1088E000943298472B6820F480210BB141F4802109
:1088F000D6F890326C20984795E438B9614BD3F89C
:108900009432984700F0010028608CE401287FF43D
:108910008AAC5C4E0020D6F894329847296820F043
:10892000010000290CBF014640F00101D6F8903249
:108930000020984777E438B9524BD3F894329847DF
:10894000C0F3400028606EE401287FF46CAC4D4E0B
:108950000020D6F894329847296820F002000029B8
:108960000CBF014640F00101D6F890320020984734
:1089700059E460B9434B6C20D3F8943298474FF4D4
:108980008073C0F3036043FA00F028604BE40128D1
:108990007FF449AC1B68102B23D00DDC022B1CD0BC
:1089A00004DC012B16D04FF0FF3314E0042B16D05B
:1089B000082BF8D105230EE0402B14D003DC202B2C
:1089C000F1D1032307E0802B0FD0B3F5807FEAD1EC
:1089D000002300E008232B6008E00723FBE70623C1
:1089E000F9E70423F7E70223F5E728602B68013352
:1089F00010D0244E6C20D6F8943298472B6820F083
:108A000070611B0603F07063D6F8902219436C2046
:108A1000904708E4D1F8EC00044304E448B9194B4A
:108A20006C20D3F894329847C0F3C1302860FFF728
:108A3000FABB01287FF4F7AB124E6C20D6F89432C3
:108A400098472B6820F4C031DB0303F4C033D6F819
:108A5000902219436C209047FFF7E5BB01287FF473
:108A6000E2AB084E6C20D6F8943298472B6820F47D
:108A700080410BB141F48041D6F890326C20984788
:108A8000FFF7D1BB100A0020FFFF0F0048B9C24B0F
:108A90006C20D3F894329847C0F300302860FFF779
:108AA000C2BB01287FF4BFABBB4E6C20D6F894321A
:108AB00098472B6820F480510BB141F48051D6F8CF
:108AC00090326C209847FFF7AEBB00BBB24E6C20D3
:108AD000D6F89432984710F4804FD6F894324FF07D
:108AE0006C0005D09847C0F3C3102860FFF79BBB0C
:108AF0009847D6F8943207466C2098473E05C0F355
:108B0000021048BF40F008002860FFF78CBB012826
:108B10007FF489ABA04E6C20D6F89432984710F4BD
:108B2000804F10D0D6F894326C2098472B6820F4F0
:108B3000F061DB0103F4F063D6F8902219436C2056
:108B40009047FFF770BBD6F894326C20984729689D
:108B5000D6F890320D074CBF40F4006020F400605E
:108B6000090120F07000C9B201436C209847FFF75B
:108B70005ABB00BB884E6C20D6F89432984710F44C
:108B8000804FD6F894324FF06C0005D09847C0F370
:108B900002102860FFF747BB9847D6F89432074683
:108BA0006C2098473A05C0F3C31048BF40F0080056
:108BB0002860FFF738BB01287FF435AB764E6C2078
:108BC000D6F89432984710F4804FD6F894324FF08C
:108BD0006C000DD098472B6820F070011B0103F04A
:108BE0007003D6F8902219436C209047FFF71BBB07
:108BF00098472B6820F4F061DB0103F4F063D6F8AA
:108C0000902219436C209047FFF70DBB01287FF499
:108C10000AAB614E6C20D6F8943298472B6820F04E
:108C20000F0103F00F03D6F8902219436C209047F0
:108C3000FFF7F9BA48B9584B6D20D3F894329847EA
:108C4000C0F3C0302860FFF7EEBA01287FF4EBAA2A
:108C5000514E6D20D6F8943298472B6820F400418D
:108C60000BB141F40041D6F890326D209847FFF7E0
:108C7000DABA48B9484B6D20D3F894329847C0F31C
:108C800041302860FFF7CFBA01287FF4CCAA424ECA
:108C90006D20D6F8943298472B6820F4C0415B03CE
:108CA00003F4C043D6F8902219436D209047FFF794
:108CB000BABA01287FF4B7AA374E6D20D6F894329D
:108CC00098472B6820F470611B0203F47063D6F898
:108CD000902219436D209047FFF7A5BA48B92E4B53
:108CE0006D20D3F894329847C0F341102860FFF705
:108CF0009ABA01287FF497AA274E6D20D6F89432AD
:108D000098472B6820F060015B0103F06003D6F800
:108D1000902219436D209047FFF785BA48B91E4B42
:108D20006D20D3F89432984700F00F002860FFF7C9
:108D30007ABA01287FF477AA174E6D20D6F89432BC
:108D400098472B6820F00F0103F00F03D6F890220C
:108D500019436D209047FFF766BA48B90E4B6D2056
:108D6000D3F894329847C0F300602860FFF75BBAED
:108D700001287FF458AA084E6D20D6F894329847FF
:108D80002B6820F080710BB141F08071D6F89032E1
:108D90006D209847FFF747BA100A002001287FF49A
:108DA00042AAB94E6D20D6F8943298472B6820F429
:108DB000FE011B0403F4FE03D6F8902219436D2034
:108DC0009047FFF730BA48B9AF4B6C20D3F89432D4
:108DD0009847C0F340402860FFF725BA01287FF488
:108DE00022AAA94E6C20D6F8943298472B6820F41A
:108DF00000310BB141F40031D6F890326C20984725
:108E0000FFF711BA00287FF40EAA9F4B6F20D3F80A
:108E100094329847C0F304402860FFF704BA012851
:108E20007FF401AA1B684FF08076002B08BF012356
:108E3000B6FBF3F6954B944F9E4228BF1E46142076
:108E40003146D7F890329847D7F894323420984773
:108E500020F480684146D7F89032342098472B6838
:108E60003420002B0CBF00214FF480612E60D7F816
:108E7000903241EA08019847FFF7D5B990B9824B83
:108E80001420D3F8943298474FF08073002808BF1D
:108E90000120B3FBF0F07D4B984294BF28602B601B
:108EA000FFF7C1B901287FF4BEA91B684FF0807697
:108EB000002B08BF0123B6FBF3F6744B14209E422F
:108EC00028BF1E46704B3146D3F8903298472E602B
:108ED000FFF7A9B901287FF4A6A96B4E6C20D6F83C
:108EE000943298472B6820F400510BB141F40051A3
:108EF000D6F890326C209847FFF795B948B9624B85
:108F00006C20D3F894329847C0F303502860FFF7E1
:108F10008AB901287FF487A95B4E6C20D6F8943279
:108F200098472B6820F470011B0503F47003D6F8F2
:108F3000902219436C209047FFF775B990B9524BB6
:108F40001320D3F8943298474FF08073002808BF5D
:108F50000120B3FBF0F04D4B984294BF28602B608A
:108F6000FFF761B901287FF45EA91B684FF0807696
:108F7000002B08BF0123B6FBF3F6444B13209E429F
:108F800028BF1E46404B3146D3F8903298472E609A
:108F9000FFF749B948B93C4B7020D3F89432984751
:108FA000C0F307202860FFF73EB901287FF43BA9F2
:108FB000354E7020D6F894329847296820F47F40C7
:108FC00040EA0121D6F8903270209847D6F89432C2
:108FD000384698472A6833464AB140F00406D3F829
:108FE00090323146002098472E60FFF71CB920F0E0
:108FF0000406F4E701287FF416A9234F7020D7F860
:10900000943298472E7820F0FF000643D7F890322C
:109010003146702098472E60FFF705B948B91A4BC2
:109020007020D3F894329847C0F301402860FFF7CE
:10903000FAB801287FF4F7A81B68032B13D8124F46
:109040007020D7F8943298472B6820F440301E04E3
:1090500006F440360643D7F89032314670209847E0
:109060002E60FFF7E0B8D1F8EC000443FFF7DBB85F
:1090700070B9054B7020D3F894329847C0F3804004
:109080002860FFF7D0B800BF100A0020FFFF0F00D4
:1090900001287FF4C8A81B68012B13D8314F70201A
:1090A000D7F8943298472B6820F480209E0406F469
:1090B00080260643D7F890323146702098472E60BC
:1090C000FFF7B1B8D1F8EC000443FFF7ACB848B9EA
:1090D000244B7020D3F894329847C0F30150286095
:1090E000FFF7A1B801287FF49EA81E4F7020D7F883
:1090F000943298472B6820F440101E0506F4401661
:109100000643D7F890323146702098472E60FFF71B
:109110008AB838B9134B3920D3F89432984728606D
:10912000FFF781B801287FF47EA80E4B2968D3F899
:10913000903239209847FFF776B838B9094B3A2072
:10914000D3F8943298472860FFF76DB801287FF470
:109150006AA8044B2968D3F890323A209847FFF761
:1091600062B800BF100A002007B502AB43F8042D17
:1091700002460120FFF74EF803B05DF804FB1346EA
:1091800002460020FFF746B8054B10B1D3F8E800BF
:109190007047044A52680A60D3F8D400704700BF91
:1091A00004000020100A0020014BD3F89032184729
:1091B000100A0020034B10B5D3F894320C469847A0
:1091C000206010BD100A0020014BD3F888321847E8
:1091D000100A00200022014B5A6070470400002052
:1091E0000528F8B50D46144600F0C28023D80228A1
:1091F00000F0888007D8002838D0012865D06E4B51
:10920000D3F8E0405FE0032800F093800428F6D113
:1092100015686A4E6A4B002D00F09780012D00F012
:109220009F80DD6870692B681B6998472B6870699F
:109230001B6A984787E0FC2800F0AC8010D806280D
:1092400000F0A1800728DAD113685D4A012BD268AB
:109250005A4B1268D8690CBF5269926990474FE027
:10926000FD284DD11268544B1A7449E0136833F04D
:10927000030225D113F0010F504D514E0ED0F3686B
:109280001B681B69A8689847246814F002040DD075
:10929000F36868681B681B69984731E0F768A8683D
:1092A0003B68DB6898473B689B69EBE7F668686852
:1092B0003368DB689847336868689B69984702E0C1
:1092C0003D4BD3F8EC402046F8BD44F620631468CB
:1092D0009C42F5D842F21073394A9C42D268374B0F
:1092E0001268986A8CBF52699269904742F2117372
:1092F000B4FBF3F003FB1040324B80B29B689847FD
:109300000024E0E714682E4B64B1DC6860682368D1
:1093100000F50670DB6898476068236800F5067002
:109320009B69B9E7DB6858681B6800F506709B68A5
:10933000C4E7254E2846D6F8903211689847D6F8EB
:109340009432284698472060DAE7DF6870693B6806
:10935000DB6898473B689B69706998472846F2E745
:10936000DF6870693B68DB6898473B685B69F3E7D7
:10937000134B124ADB68106A1B681B6A984700305F
:1093800018BF0120DFE70E4B0C4ADB68506A1B68F0
:109390001B6AF3E71468094D094B44B1DC6868693E
:1093A0002368DB689847236868699B6974E7DB6812
:1093B00068691B681B6981E704000020502B0020AE
:1093C0008C4D0208AC190020100A00201C4B70B50F
:1093D000DD681C4C2B68E0689B6998472B68E06A45
:1093E0009B6898472B68A06A9B6898472B68206900
:1093F0009B6898472B6860699B6898472B68A069B1
:109400009B6898472B6860689B6898472B68A068A2
:109410009B6898472B68206A9B6898472B68606A0E
:109420009B6898472B68E0699B6898472B68E068C1
:109430009B689847BDE87040034B5B68184700BFC6
:109440008C4D0208502B0020AC19002038B5124B6F
:10945000124D9C78C4B1D5F89C329847104B00202F
:109460009B6898470F4B104CDD68A06A2B689B697E
:1094700098472B6860681B6998472B68A0681B6930
:1094800098470124204638BDD5F8943222209847C9
:109490000028E0D0F6E700BF341A0020100A0020B0
:1094A000AC1900208C4D0208502B0020012873B508
:1094B0000D46104C03D9D4F8E80002B070BD01226B
:1094C0000D4B0E4E81EAE1711A60A1EBE571D6F801
:1094D000903227209847002DACBF01230223D6F8F5
:1094E0008C620093002320201A461946B047D4F816
:1094F000D400E2E704000020502B0020100A0020D6
:10950000D4E74942D2E70021D0E72DE9F34188466C
:109510000746114D20B1D5F8E80002B0BDE8F08152
:109520000E4E0F4C336833B10E4AD4F890321168A6
:10953000272098473760D4F8903241462D2098472D
:10954000002300932020D4F88C421A461946A047E5
:10955000D5F8D400E1E700BF04000020502B002024
:10956000100A00207C10002038B5074B0C46054639
:10957000D3F89432212098472368C11821602846E7
:10958000BDE83840C1E700BF100A00200F4B9A78B1
:10959000824204BF0E4A92F8D1001A78824206D164
:1095A0000C4BDB681B685B690B4AD06818475B781B
:1095B000834209D1064B93F8D130834204D1054B45
:1095C000DB681B689B69EFE7704700BF781A0020D3
:1095D000040000208C4D0208502B00202DE9F041A2
:1095E000544E554CF56801276B6803F1C802E260E0
:1095F00003F58072226103F58E72626103F5B87221
:10960000626003F5C672A26003F5F072A26203F510
:10961000FE72E26203F5617203F1E400E26103F5B8
:10962000687203F56F7323622B6862621B69A06125
:1096300098472B6860691B6998472B6820691B69EC
:1096400098472B68206A1B6998472B68606A1B69DA
:1096500098472B68E069DB6898472B6860681B694E
:1096600098472B68A0681B6998472B68E068DB68FF
:1096700098472B68A06ADB6898472B68E06ADB682C
:1096800098472B68E0699B699847326900266B68A8
:109690002A4903F537735360294B0A605A692948F0
:1096A000C1F89822D1F8A012C2F8040216705670C0
:1096B000C2F80C12244A02201A62244A5F74DA614A
:1096C000234A83F8D0709A61224A5A62224A9A63E6
:1096D000224A5A63224A9A62224ADA62224A9A64E7
:1096E000224A5A64224A5A65224A1A65224ADA6490
:1096F000224A5A66224A1A663222DA604FF4F0721F
:109700009A60204ADA65FFF741FF0222E36A197C7A
:109710005A7418683A4607F005FA2B68E06A1A4C42
:109720001B68984723689847A3683046BDE8F04116
:10973000184700BF8C4D0208502B0020100A002053
:10974000040000204D940108AD9401080195010822
:1097500003950108079501087F91010869910108A7
:109760000B95010869950108A9910108B5910108B7
:10977000C9910108E1910108899101088D950108BD
:10978000D5910108CD930108AC19002002F09CBFCF
:1097900002F0C6BF03F023B803F052B8F7B50F4686
:1097A00006461D46C04927B1D1F8E840204603B01F
:1097B000F0BD8C2AD1F8D44000F09D8300F2A18046
:1097C0000E2A00F0728245D8062A00F0DA811CD8F1
:1097D000022A00F08B8109D8002A00F05D81012A5D
:1097E00000F07281D1F8E0000443DFE7042A00F0C2
:1097F0009F8140F29381002840F0B981AB4B262035
:10980000D3F8943298472860D0E70A2A00F0F7810D
:109810000FD8072A00F0D481082AE3D10028C5D147
:10982000A24B3520D3F894329847C0F340202860EB
:10983000BCE70C2A00F0FF8140F2F081002840F0E4
:109840001C829A4B3420D3F89432984700F00100E0
:109850002860ABE7152A00F09D8221D8112A00F07C
:1098600052820ED80F2A00F03282102ABAD1002874
:1098700040F03F828D4B2520D3F8943298472860E2
:1098800094E7132A00F06A8240F24F82002840F0E9
:109890007782864B2B20D3F894329847286085E74F
:1098A0001C2A00F0CF821CD8182A00F09C821B2AA8
:1098B00000F0AB82172A95D1002840F07D827B4BC7
:1098C0001520D3F8943298474FF08073002808BFD2
:1098D0000120B3FBF0F0764B984294BF28602B60D8
:1098E00064E7212A00F0CB82222A00F0E6821D2ABA
:1098F0007FF478AF00287FF459AF6C4B5B682B6026
:1099000054E7B32A00F021855CD8A82A00F05484DB
:1099100026D8A42A00F07C8311D8A22A00F0408324
:10992000A32A7FF45FAF002840F05A835F4B6C207E
:10993000D3F894329847C0F38030286036E7A62ADF
:1099400000F0D98340F28383002840F02184574BF4
:109950006C20D3F89432984700F00F00286025E778
:10996000AB2A00F07D8411D8A92A00F04484AA2AE9
:109970007FF438AF002840F05E844C4B6D20D3F864
:1099800094329847C0F3032028600FE7AD2A00F017
:10999000A684C0F08584AE2A7FF424AF002840F06E
:1099A000BF84424B6D20D3F894329847001410F0D6
:1099B000400F0CBF00236FF07F0300F07F021343C2
:1099C0002B60F3E6BB2A00F0A68538D8B62A00F053
:1099D000168520D8B42A00F0D784B52A7FF402AFC8
:1099E000002840F0DE84314F3420D7F89432984775
:1099F00043050ED5D7F89432142098474FF080765F
:109A0000002808BF0120B6FBF0F62948864228BF8F
:109A100006462E60CAE6B92A00F0318500F24F856D
:109A2000B82A7FF4DFAE002840F015851F4B6C206C
:109A3000D3F894329847C0F340302860B6E6CC2A79
:109A400000F0058613D8BF2A00F0A985C02A00F0CF
:109A5000D085BC2A7FF4C6AE002840F08C85134B1D
:109A60007020D3F894329847C0B228609EE6D12A7D
:109A700000F00F86D22A00F02086CE2A7FF4B2AE04
:109A800000287FF493AE094B6F20D3F894329847A7
:109A9000C0F30900286089E660B9044B2D20D3F893
:109AA00094329847286081E604000020B80C00201A
:109AB000FFFF0F0001287FF479AEA54B2968D3F88A
:109AC00090322D20984771E630B9A14B2120D3F870
:109AD00094329847286069E601287FF467AE9C4B72
:109AE0002968D3F89032212098475FE630B9984B27
:109AF0002720D3F894329847286057E601287FF44E
:109B000055AE1968924B0029D3F89032B8BF49423C
:109B10002720984701228F4B1A6047E600287FF4E0
:109B200045AE8B4B2220D3F89432984728603DE60F
:109B300018B9894B1B682B6038E601287FF436AED4
:109B40001B68854A002B824EB8BF5B421360202001
:109B5000D6F89432984700287FF428AE2968D6F8C2
:109B600090320029B8BF4942272098471EE60128B5
:109B70007FF41CAE764B2968D3F8903226209847A4
:109B800014E640B9724B1020D3F894329847C0F3D2
:109B9000042028600AE601287FF408AE6C4E1020ED
:109BA000D6F8943298472B68C2B20092D6F88C52FD
:109BB000C0F3074203F01F0339461020A847F5E51C
:109BC00038B9634B1020D3F894329847C0B228605C
:109BD000ECE501287FF4EAAD5D4E1020D6F8943212
:109BE00098472B68C0F3074203F01F030093D6F891
:109BF0008C52C0F3072300211020A847D6E5002887
